:020000040800F2
:10000000F0FF012049A305088DE60008457C04089F
:10001000C1A30508C1A30508C1A30508000000008D
:1000200000000000000000000000000089E6000859
:1000300085E600080000000081E60008B13F0408E2
:10004000C1A30508C1A30508C1A30508C1A30508EC
:10005000C1A30508C1A3050835920408FD91040851
:10006000C59104088D91040855910408198A050862
:10007000098A0508F9890508E9890508D589050867
:10008000C1890508AD890508C1A305080000000065
:100090000000000000000000000000001D910408A6
:1000A000112604086126040801260408892604088C
:1000B000512604084126040831260408C1A3050876
:1000C000C1A30508C1A30508C1A30508C1A305086C
:1000D000C1A30508D1400408154004080000000031
:1000E000E5900408C1A30508450D010800000000C3
:1000F00000000000000000000000000099890508D1
:1001000000000000C1A3050821260408C1A30508BA
:1001100000000000000000000000000000000000DF
:1001200085890508718905085D89050849890508DB
:1001300035890508000000000000000000000000F4
:1001400000000000000000000000000001FD0008A9
:10015000218905080D890508F9880508C1A3050846
:10016000C1A30508C1A305080000000000000000AD
:10017000000000000000000000000000000000007F
:1001800000000000C1A305080000000000000000FE
:08019000C1A30508C1A3050885
:08019800E89E050001000000D3
:1001A0000B3001001A00000050360020F4700020CF
:1001B00000000000E4C50608F07000201F50010098
:1001C0002400000010360020147100200000000000
:1001D00000C606081071002005020100040000009E
:1001E000547000203C7100200000000024C6060866
:1001F000387100201302010004000000F42A0020DE
:10020000447100200000000028C60608407100204C
:10021000031101000A000000403500204C7100204D
:1002200000000000698E0008487100200D100100D8
:1002300034000000946200205C7100200000000087
:100240001FB70308587100200902010001000000D7
:10025000B46F002094710020000000002CC6060836
:1002600090710020F9010100040000005462002098
:100270009C710020000000009D110408987100206E
:10028000FB01010001000000685D0020A471002056
:100290000000000035310508A0710020FC010100BC
:1002A00009000000345C0020AC7100200000000058
:1002B00045310508A8710020F70101000600000083
:1002C000285C0020BC710020000000002EC606083B
:1002D000B8710020160215003F00000044330020D2
:1002E000C871002000000000E5310508C47100203D
:1002F0003400010010000000585B00200C72002048
:100300000000000079430208087200201102010079
:1003100008000000305B0020207200200000000078
:1003200034C606081C7200201212010004000000EE
:10033000285B00202C720020000000003CC606084C
:10034000287200201830010038000000F05A002008
:100350003472002000000000553205083072002081
:10036000000201000B000000745700207072002092
:1003700000000000512805086C720020FD010100FA
:10038000210000005C51002080720020000000006D
:10039000F71004087C7200202A0201000800000007
:1003A00068430020A87200200000000040C6060834
:1003B000A472002020520100080000001043002019
:1003C000B47200200000000069330208B0720020FF
:1003D00006100100240000000C320020C072002032
:1003E0000000000061310508BC7200200C02010011
:1003F00004000000C83B0020E8720020000000005C
:1004000009280508E4720020FE0101001400000024
:1004100020670020F0720020000000005928050825
:10042000EC7200201B2001000C000000CC8C00208E
:10043000C09F00200000000021960108BC9F002002
:1004400021020100F0000000FC8A0020D09F002063
:100450000000000005350108CC9F00203710010086
:1004600030000000D89C0020C4A000200000000044
:1004700048C60608C0A000200E02010002000000CD
:1004800044910020F8A000200000000078C6060873
:10049000F4A0002016100100060000003C9100208E
:1004A00000A10020000000007AC60608FCA0002081
:1004B0002F10010022000000989F00200CA10020B6
:1004C0000000000080C6060808A1002023220100C9
:1004D000100000009490002034A1002000000000D3
:1004E000A4C6060830A100201E000100090000007B
:1004F0007C90002048A1002000000000B4C606083F
:1005000044A10020052001000C000000DC90002028
:1005100058A1002000000000C0C6060854A1002019
:10052000FD0701007C000000C089002068A10020B8
:10053000000000006114010864A10020F591010091
:100540006C000000808A0020E8A10020000000006C
:10055000E5330108E4A10020232001001000000081
:100560003A9C002058A2002000000000BD110208A3
:1005700054A20020123001001000000064900020FE
:100580006CA2002000000000CCC6060868A2002073
:10059000140001000500000088C60020B0C600203D
:1005A00000000000DCC60608ACC6002001200100E7
:1005B0000C00000018BA0020BCC60020000000009B
:1005C000E2C60608B8C600200C400600E4000000A1
:1005D0003CB80020CCC60020000000001D5F0308CE
:1005E000C8C600200A90010024000000F8B70020CF
:1005F000B4C700200000000075110208B0C7002039
:100600000E300300BC01000034B60020DCC700201F
:100610000000000081330208D8C700201310010039
:100620000400000030C400209CC90020000000002D
:10063000F0C6060898C9002001010100040000006E
:100640006CB50020A4C900200000000000000000DC
:10065000A0C90020000101000400000064B50020D2
:10066000ACC9002000000000F4C60608A8C900209C
:10067000020101000300000060B50020B4C90020A1
:10068000000000005D5F0308B0C9002022020100E5
:100690001C01000018C20020BCC90020000000009E
:1006A000C9330508B8C90020010201000B00000091
:1006B00078B50020DCCA00200000000041280508B1
:1006C000D8CA00200202010003000000BCBA0020CA
:1006D000ECCA00200000000000000000E8CA002072
:1006E0001B020100100000006CBA0020F4CA0020B8
:1006F00000000000E9280508F0CA002015001000DD
:100700007000000040D7002044D900200000000005
:100710000000000040D900202A000800600000000E
:1007200050D60020B8D90020000000004133020854
:10073000B4D900202C000400100000002CDA0020A6
:100740001CDA0020000000000931020818DA00203D
:10075000292014007800000040D3002040DA002057
:1007600000000000000000003CDA00201A00010038
:100770000E00000098D20020BCDA0020000000002B
:10078000F8C60608B8DA00202B001200240000008A
:1007900074D20020D0DA002000000000DD30020812
:1007A000CCDA0020190201001000000060D2002005
:1007B000F8DA00200000000021280508F4DA002003
:1007C000F62101000C00000044D100200CDB0020C9
:1007D0000000000008C7060808DB00201C02020019
:1007E0001C0000005CD1002060DB00200000000045
:1007F0003D3305085CDB0020F831010006000000F5
:10080000C4DD0020F4E000200000000014C706084A
:10081000F0E000200300010001000000D4DD002012
:1008200000E100200000000000000000FCE00020CB
:100830001010010002000000C0E0002008E10020CC
:10084000000000001AC7060804E10020190001009A
:100850000500000020DD002010E100200000000065
:100860001CC706080CE1002029020100400000001E
:1008700050E300200CE800200000000022C706081A
:1008800008E800202C0201000400000004E500201C
:1008900050E800200000000062C706084CE8002075
:1008A0000A02010014000000B0E3002078E80020F4
:1008B00000000000C568030874E8002025201E0021
:1008C0002C01000024E5002090E80020000000003A
:1008D000000000008CE80020031201003D00000031
:1008E000BCE70020C0E900200000000066C7060841
:1008F000BCE90020020001000C00000034EA0020E6
:10090000CCEA00200000000000000000C8EA00203F
:100910000400080080000000E8F2002068F30020D6
:100920000000000000000000ECF4002008120300AA
:100930000F000000D8F20020F4F4002000000000B6
:1009400081280508F0F400202802040004000000BB
:1009500044F2002008F5002000000000E52805080A
:1009600004F50020270204000400000040F20020EB
:1009700010F5002000000000D92805080CF5002023
:100980001F020800100000007CEF002018F5002076
:1009900000000000E927050814F500201A020100F4
:1009A0003C00000020EB00202CF50020000000009F
:1009B000B132050828F500203820010003000000AE
:1009C000E4EA00206CF5002000000000A4C706083F
:1009D00068F50020270001000400000094F50020C5
:1009E000F8F5002000000000A8C70608F4F5002074
:1009F0001002010001000000980D0120940D01205B
:100A000000000000ACC70608900D01202B02010079
:100A10000C00000004F70020AC0D012000000000D5
:100A2000AEC70608A80D01201D0202000600000046
:100A3000880D0120BC0D0120000000000000000016
:040A4000B80D0120CC
:100A44000403090412010002EF0201408304563238
:100A54000002010203010000120100020202004030
:100A640083044057000201020301000009026400EC
:100A7400030100C032090400000103000000092141
:100A8400110100012236000705830309000A080B3F
:100A94000102020201000904010001020201000531
:100AA4002400100105240100020424020205240686
:100AB4000102070582030800FF09040200020A007C
:100AC4000000070501024000000705810240000004
:100AD40009024300020100C03209040000010202BD
:100AE4000100052400100105240100010424020270
:100AF4000524060001070582030800FF090401001C
:100B0400020A0000000705010240000007058102F7
:100B140040000000FF000000140000FF000000007F
:100B240000000000AA550701000001AA55050100B4
:100B3400002D202D2D202D2D2D2D202D2D2D2D0062
:100B440000000000000000000000000000000000A1
:100B540008000000B0C60508FF1FFF1F7D0000004D
:100B640001840008FD830008F9830008ED83000870
:100B7400E9830008F5830008F18300087584000800
:100B84006984000841840008558400082D84000805
:100B94001984000805840008010000000000803F5B
:100BA40005010905A101A100050109300931093236
:100BB400093309350934093609371581257F750844
:100BC40095088102050919012908150025019508D0
:100BD40075018102C0C0000009022200010100E089
:100BE400320904000001030102000921110100017E
:100BF4002236000705830309000A00000060024052
:100C0400106002400000000000000000000000002E
:100C1400000B0000000000000000000000000000C5
:100C24000060024028600240010000000000000053
:100C340000000000060C000000000000000000009E
:100C4400000000000060024040600240020000001A
:100C54000000000000000000100D00000000000073
:100C640000000000000000000060024058600240E4
:100C7400030000000000000000000000160E000049
:100C840000000000000000000000000000600240BE
:100C9400706002400400000000000000000000003A
:100CA400200F000000000000000000000000000011
:100CB400006002408860024005000000000000005F
:100CC40000000000261000000000000000000000EA
:100CD4000000000000600240A06002400600000026
:100CE40000000000000000003011000000000000BF
:100CF400000000000000000000600240B8600240F4
:100D0400070000000000000000000000362F000073
:100D14000000000000000000000000000064024029
:100D24001064024000000000000000000000000009
:100D34000038000000000000000000000000000077
:100D4400006402402864024001000000000000002A
:100D54000000000006390000000000000000000050
:100D640000000000006402404064024002000000F1
:100D74000000000000000000103A00000000000025
:100D840000000000000000000064024058640240BB
:100D9400030000000000000000000000163B0000FB
:100DA4000000000000000000000000000064024099
:100DB4007064024004000000000000000000000015
:100DC400203C0000000000000000000000000000C3
:100DD4000064024088640240050000000000000036
:100DE4000000000026440000000000000000000095
:100DF4000000000000640240A064024006000000FD
:100E04000000000000000000304500000000000069
:100E1400000000000000000000640240B8640240CA
:100E2400070000000000000000000000364600003B
:100E340000000000000000000000000000000000AE
:100E440001020304010203040607080939E8000843
:100E5400F1EE000869EA000819850008F98A00081B
:100E64002985000845850008F1840008E18400080C
:100E74000000000000000000AA550B010000AA5564
:100E840005010000AA550902000000AA5503009FAD
:100E940001000000C0120000010000000000010079
:100EA400FFFFFFFF7EFF0000FFFFFFFFFF000000CA
:100EB400FFFFFFFFA4A20020000000007CA200208E
:100EC400000000000101FF01E00101007D8B010829
:100ED4000000000000000000D0CD050808FF00005D
:100EE400000000000000000000000000C4E4050849
:100EF4000000000000000000000000007CE5050880
:100F040000000000000000000000000028E50508C3
:100F14000000000000000000A9A6010856BD002042
:100F24000101000061E00108000000000000000071
:100F340044E60508C5E301080000000000000000C5
:100F4400FCE505082D202D2D202D2D2D2D202D2DBA
:100F54002D00000000000000000000000000000060
:100F640000000000FFFFFFFFC1B101080000000006
:100F74000000000054E4050801000000FA0000002D
:100F8400010000000100000082B900200000F4010B
:100F94000100000080B900200000F40101000000FD
:100FA4007EB900200000F401010000007CB900209B
:100FB4000000F401010000007AB900200000F401EF
:100FC4000100000078B900200000F40101000000D5
:100FD40076B900200000F4010100000039940108F2
:100FE400FD930108000000003CCF050866B900200D
:100FF4000532010074B900206400F401010000000E
:1010040072B900206400C4090100000064B9002022
:10101400E803D0070100000062B90020E803D0070C
:101024000100000060B90020E803D00701000000BF
:101034005EB900201E00B80B010000006CB900204E
:1010440005000F00010000006EB9002003000A0033
:10105400010000005CB900201E00F4010100000042
:1010640070B9002002000000C8CF05085AB900205A
:10107400140064000100000068B900203200E80395
:101084000100000058B900200000C8000100000061
:1010940039B8002000C8010038B800200050010011
:1010A40037B80020005A010035B8002002000000C3
:1010B40030CF0508404406084844060854BD0020C3
:1010C4000100C4090000000052BD00200100C40951
:1010D4000000000050BD00200100C4090000000011
:1010E4004EBD00200100C409000000004ABD0020DC
:1010F4000100C409000000004CBD00200100C40927
:101104000000000048BD00200100C40900000000E8
:1011140046BD00200100C4090000000099B500206C
:1011240000C8010098B5002000C8010096B5002051
:101134000000FFFF0A00000094B500200100C80071
:101144000100000092B5002032003075320000002A
:1011540090B500207EFF1400050000008EB500202D
:1011640005002C01050000008CB50020055A05007F
:1011740089B5002000FF01008BB5002002000000AB
:101184000C08002087B5002003000000E4C7050810
:1011940088B5002000FF01008AB50020020000008D
:1011A4000C08002086B5002003000000E4C70508F1
:1011B400D8B40020FF7F0100D4B400200000000058
:1011C400FFFFFFFF01000000D0B40020000000007A
:1011D400FFFFFFFF01000000CCB40020000000006E
:1011E400FFFFFFFF010000008D9301081D9301081C
:1011F4000000000018D0050828BA0020EE02CA0832
:101204000100000026BA002000C8010064000000AC
:1012140025BA002002C801006400000024BA00209E
:1012240002000000D4CF050872B500200000803E03
:101234000500000070B5002080C1803E050000005C
:101244006AB500200083007D0500000068B5002019
:1012540080C1803E0500000063B5002000FF01004E
:101264005CB500206400F401010000005AB50020C0
:101274006400F4010100000058B500206400F4018A
:101284000100000056B500200400000024D1050828
:1012940055B500200200000038D1050825B600200D
:1012A4000D00000044D1050822B6002000640100AE
:1012B40020B60020320010270A0000001EB60020CD
:1012C4000D00000044D105081DB600200D000000EB
:1012D40044D105081CB6002002000000E0CF050838
:1012E4002DBA0020460000007CD105082BBA00204E
:1012F4000300000098D205082CBA00200400000066
:10130400ECCF050827B6002003000000A8D205088A
:1013140026B6002003000000A8D2050826B8002045
:10132400000A010024B800200000E80301000000C6
:1013340022B800200000E8030100000020B80020CB
:10134400000A01001EB800200000E80301000000AC
:101354001CB800200000E80301000000F0B70020E2
:10136400C800E80301000000F6B700203C00FA00C2
:1013740001000000F4B700200100E80301000000B0
:10138400F2B700200005010034B80020020000007C
:1013940000D0050832B800200000F401010000006C
:1013A40030B800200000F401010000002EB8002035
:1013B4000000F401010000002CB800200000F4013A
:1013C400010000002AB800200000E803010000002A
:1013D40028B800200000E8030100000046B90020FE
:1013E400006401000A00000045B900200064010007
:1013F4000A00000033B900201964010032B900204A
:10140400020000000CD0050830B90020E803D00722
:101414000A0000002EB90020006401000A00000048
:1014240023B900200064010022B9002000640100F7
:101434002AB90020006401000A00000029B9002034
:10144400006401000A00000028B9002000640100C3
:101454000A0000002DB9002000FF01000A0000006E
:101464002CB9002000FF01000A0000002BB9002065
:1014740000FF01000A00000027B9002001FF01005D
:101484000A00000026B9002001FF01000A00000044
:1014940025B9002001FF01000A00000030B6002039
:1014A4000000F401010000002EB600200000E80353
:1014B400010000002CB600200000E8030100000039
:1014C4002AB600200000E8030100000028B600202E
:1014D4000000E80301000000A7BD00200096010001
:1014E4009EBD002000C801009DBD002000640100D5
:1014F4009CBD0020006401009BBD0020006401002D
:101504009ABD00200064010099BD0020FF0801007D
:1015140098BD0020016401000D920108D1910108D9
:1015240000000000B8D20508A1BD0020013201006E
:10153400A0BD00200100000028D305089FBD0020A5
:101544000400000030D3050897BD00200096010078
:1015540096BD00200064010094BD00201400E8033F
:101564000100000092BD0020000030750A00000058
:1015740090BD002000C801008FBD002000C80100FC
:101584008EBD002000C80100A4BD0020003201006F
:10159400A6BD002000140100A5BD0020004B0100E1
:1015A400A3BD00200400000044D30508A2BD002010
:1015B400006401000A00000052B900200AC80500B6
:1015C4000A00000051B900200100000054D30508AE
:1015D40054B900200AC805000A00000053B90020CD
:1015E4000100000054D3050849B9002000C80500D3
:1015F4000A00000050B9002000C805000A000000DD
:101604004AB9002000C805000A0000004BB90020B8
:1016140000C805000A0000004EB9002000C80500FB
:101624000A0000004FB9002000C805000A000000AD
:101634004DB9002000C805000A0000004CB9002084
:1016440000C805000A00000048B90020020000009C
:101654005CD30508B6BD00200000D00701000000DF
:10166400B0BD002000C80100AFBD002000C80100CB
:10167400AEBD002000C80100B4BD00200000D007AA
:1016840001000000ADBD002000C80100ACBD002079
:1016940000C80100ABBD002000C80100B2BD00209D
:1016A4000000D00701000000AABD002000C801000E
:1016B400A9BD002000C80100A8BD002000C8010089
:1016C400585506080000000000008FC6002064552D
:1016D4000608070800000000100E00206C550608DC
:1016E400070800000000080E0020745506080708CB
:1016F40000000000000E00207C55060808080000C9
:101704000000F40D0020A03F0608070800000000B8
:10171400EC0D0020A83F0608070800000000E40DB7
:101724000020B03F0608070800000000DC0D002080
:101734005C400608080800000000D00D0020845515
:101744000608071000000000C80D00208C5506088C
:10175400071000000000C00D002094550608071073
:1017640000000000B80D00209C5506080810000079
:101774000000AC0D0020A843060801000000000092
:101784000000000000000000100000000000000045
:1017940000000000A18F0108858F01089DB1010898
:1017A40068D3050819B60020005A010018B60020B5
:1017B40000C8010016B60020E803D00701000000AD
:1017C4000000000000000000E9A6010804D4050898
:1017D40085B50020030000004CD4050884B5002022
:1017E4000003010083B5002000030100C18E01083D
:1017F400758E0108000000005CD40508358E0108D0
:10180400ED8D010800000000F8D405080D8F0108D3
:1018140081B101080000000078D5050874B50020E6
:1018240001030100418B0108198B0108000000002D
:10183400ECD80508F9940108CD94010800000000D3
:101844006CD905085D8D0108058D010800000000B4
:10185400DCD90508B18F0108C9EB010800000000BC
:1018640094DA050895A701082595010800000000F1
:101874003CDB0508019001080000000000000000A6
:10188400C8DB0508E5900108859001080000000008
:101894002CDC05088D910108499101080000000025
:1018A400E4DC0508DD0F020849920108000000008D
:1018B40070DD050856B900200106010049900108B1
:1018C400159001080000000088DE0508F90E0208E2
:1018D40049B3010800000000F8DE05087992010808
:1018E40069B401080000000074E005082110020832
:1018F40029B4010800000000180E002055B900208A
:1019040001030100558F0108258F01080000000024
:1019140080E1050821B1010800000000000000007A
:10192400E4E10508B58D010869B101080000000073
:1019340080E2050800000000000000000000000034
:101944001CE30508F5920108B5B501080000000084
:101954009CE30508000000000000000000000000F7
:10196400C4E50508D43500209CFF2C0100000000CC
:10197400C8C30020E0150C1700000000CAC30020F3
:1019840002000000FCE8050850B5002088136F171A
:101994000100000052B5002088136F1700000000FA
:1019A40074350020000000000000000072350020A3
:1019B400000000000000000070350020000000005E
:1019C400000000006E350020000000000000000050
:1019D4006C35002000000000000000006A35002083
:1019E4000000000000000000EC05002000000000E2
:1019F40000000000D9B4002003000000E0E6050860
:101A040048B5002088136F17010000004A700020B9
:101A140088136F1700000000458C010800000000C7
:101A240000000000F0E6050811BD002001000000E0
:101A340044E705084C7000200100000050E7050849
:101A4400427000200200000058E705080000000072
:101A5400000000000000000064E705082D8C010868
:101A6400000000000000000000E80508000000007D
:101A7400000000000000000054E805080000000019
:101A84000000000000000000C4E8050854B5002070
:101A940002000000FCE8050846700020E0150C1761
:101AA4000000000080CC0020D4CC002001F11F3FB6
:101AB400D60101010001010100FF00003D2F0208D1
:101AC40004730020FFFFFFFF0000803F00000000C0
:101AD4000000000000000000000000000000000002
:101AE40000000000000000000000000000000000F2
:101AF4000000803F00000000000000000000000023
:101B04000000803F00000000000000000000000012
:101B14000000803F00000000000000000000000002
:101B2400010000000000FA430000FA430000803F77
:101B340095D703080000000000000000000000002A
:101B440060FECD000000000064E8002008000000F2
:101B54000000000054E8002008000000FFFFFFFF21
:101B6400FF000000C58A0008A589000849EA0008AA
:101B740000000000DD84000805E800081D89000855
:101B840079E7000800000000000000009D840008C0
:101B9400358A00086589000899E9000800000000FA
:101BA400B58400087DE70008F1880008D5E6000840
:101BB4000000000000000000A98400082C6A060848
:101BC400FC40060800000000E55F0308A086010051
:101BD400040000002C6A0608346A060800000000AD
:101BE400590F0408E8030000040000003C4A0608FA
:101BF400000000000000000051F602087D00000013
:101C0400FF0000004048060800000000000000003B
:101C1400E5DA02087D000000FF0000006C4D0608B4
:101C24000000000000000000F11B03087D0000001C
:101C3400FF000000D44A0608000000000000000075
:101C440015130408E8030000030000003C6A0608BA
:101C54000000000000000000BDFF02081027000083
:101C64000300000030730608000000004D2F020836
:101C7400A97C04085F76000005000000E4760608ED
:101C840000000000000000001DA904081027000047
:101C940002000000486A060800000000000000007E
:101CA4005D0F0408E803000005000000546A0608FC
:101CB4000000000000000000196B0308204E000023
:101CC40003000000646A0608000000000000000031
:101CD40001690308204E000003000000746A06082E
:101CE400000000000000000059180408400D030023
:101CF40003000000A06806080000000000000000C7
:101D040011D503081027000002000000284106082E
:101D14000000000000000000ADC40108102700000E
:101D240003000000944606080000000000000000C4
:101D3400ED0D0408A861000002000000BC6806085C
:101D44000000000000000000A9460408A00F0000E5
:101D540002000000846A0608000000000000000081
:101D6400217C0108102700000200000068570608C3
:101D74000000000015140108516F01088545010099
:101D840002000000544606080000000000000000A5
:101D94009D8E000810270000020000001041060874
:101DA400000000000000000015F5010850C3000009
:101DB40002000000906A0608000000000000000015
:101DC400E19C0008400D030001000000986A060829
:101DD4000000000000000000C1B50308400D03002E
:101DE40002000000A06A06080000000000000000D5
:101DF400E5D3010850C3000003000000AC6A0608E4
:101E04000000000000000000597F030840420F005A
:101E140001000000B86A060800000000000000008D
:101E240035B8030850C3000001000000C46A060866
:101E34000000000000000000055801081027000001
:101E44000200000065B70308000000000000000065
:101E540000000000D90D040800000000000000008C
:101E64000000000001000000A00F0000B80B0000FB
:101E74000102FFFF010000000C73060800000802C5
:101E8400050303000000000018730608010008029F
:101E94000504030000000000247306080000080283
:101EA40005030300000000002C730608010008026B
:101EB4000504030000000000106806080200FE018B
:101EC4000110030000000000884706080300140204
:101ED40000030000000000003473060804001F0221
:101EE40002000800000000003C73060805001F0201
:101EF4000201080000000000FFFF0000FFFFFFFFD9
:101F040000010000204E000000000000000000005E
:101F14000000185006000000D007000001040C0067
:101F24000101186007000000A00F000002040E0069
:101F340002031870070000000A1A000003040C00D2
:101F44000305189006000000204E000000020C005B
:101F54000000000097FFFFFF81060000C409000095
:101F6400C409000003000000881300000101000000
:101F740094FFFFFFE40C0000B80B0000C40900004C
:101F840006000000881300000203000090FFFFFF1A
:101F9400EF160000AC0D0000C40900000A000000A8
:101FA40088130000030500008BFFFFFF0B480000AF
:101FB400A00F0000C4090000000000008813000006
:101FC400541900200000000004000000000000007C
:101FD4001542050800000000000000000000000099
:101FE4000100000000000000501900200000000063
:101FF40002000000000000000000000000000000DB
:102004000000000008000000010000006541050810
:1020140000000000000000000000000001000000BB
:1020240000000000860000007C1700200000000073
:102034000400000000000000454305080000000003
:10204400000000000000000001000000000000008B
:102054003C1900209C0D0120040000000000000039
:10206400B941050800000000000000000000000065
:1020740001000000000000004C19002000000000D6
:1020840004000000000000001542050800000000E4
:10209400000000000000000001000000000000003B
:1020A40048190020A40D01200400000000000000D5
:1020B40021470508000000000000000000000000A7
:1020C40001000000000000001B0000002018002098
:1020D40000000000030000000000000000000000F9
:1020E40000000000000000000800000001000000E3
:1020F4007541050800000000000000000000000019
:10210400010000000000000044190020A00D01207F
:1021140004000000000000008541050800000000E4
:1021240000000000000000000100000000000000AA
:10213400401900200000000004000000000000001E
:102144001542050800000000000000000000000027
:10215400010000000000000097000000B0180020FB
:10216400000000000300000000000000A941050871
:10217400000000000000000000000000010000005A
:102184000000000001010100000004010000020041
:1021940001000002100000000700FF000000000022
:1021A400000000000000000001000000000000002A
:1021B400000000000000000000000000010000001A
:1021C40000000000FF000000F401000030390608A0
:1021D40000000000000000000102030406070809D3
:1021E40001000000150000008200FFFF170000003E
:1021F4001D0000008200FFFF1A0000008300FFFFA3
:10220400FF00000060190020000000000000000032
:1022140000000000000000000000000000000000BA
:1022240000000000000000000000000000000000AA
:10223400000000000000000000000000000000009A
:10224400000000000000000000000000000000008A
:10225400000000000000000000000000000000007A
:08226400000000000000000072
:082800000000000000000000D0
:10800000134B0268196821EA02011960596821EAD4
:108010000201596019680A431A609968026821EAE6
:1080200002019960D96821EA0201D96041791029D9
:1080300007D001F1804303F59E3319680A431A60A3
:108040007047996811439960D9680A43DA607047AC
:10805000003C01402DE9F04700230F6801264FF056
:10806000030C02E00133102B41D006FA03F232EA8E
:108070000704F7D1D0F800E05C000CFA04F52EEA12
:10808000050EC0F800E091F80490D0F800A009FABD
:1080900004FE09F1FF394EEA0A0EB9F1010FA846B4
:1080A000C0F800E06FEA050515D8D0F808E005EA49
:1080B0000E0585604D79D0F808E0A54045EA0E052B
:1080C0008560456825EA020242608A7945689A40DF
:1080D00092B22A434260C26822EA0802C260CA79A8
:1080E000C568A24001332A43102BC260BDD1BDE850
:1080F000F08700BF037830B403B30246C0F1010536
:10810000531912F8014FDBB2002CF9D101335B0097
:10811000DAB20C4C0B80032322706370017859B1E2
:10812000022300255A1CD2B2E154A55410F8011FB5
:108130000233DBB20029F5D130BC7047022213466E
:10814000E7E700BFC0190020084AD2E94031994250
:108150000AD0D118013391F808110170C3F30A0352
:10816000C2F800310120704700207047C01900207C
:10817000064AD2F80839D2F80C29934294BF4FF43A
:1081800000600020013B9B1A18447047C019002072
:10819000012380F85130704707B501A8FFF7D4FFDD
:1081A0000028FAD09DF8040003B05DF804FB044BEE
:1081B000D3E94003984288BF03F50063181A70475B
:1081C000C019002001207047024BC3F81029C3F8E2
:1081D00014197047C0190020024BC3F81829C3F8BE
:1081E0001C197047C01900207047704730B4134DF8
:1081F000D5E940239A4286BF03F50064A21A9A1A71
:108200000A44B2F5006F13D8A9B101444A1E0138DF
:1082100010F8014FE918824203F1010381F8084187
:10822000C3F30A03F4D1C5F80431002030BC704711
:10823000022030BC70470846F8E700BFC019002094
:10824000F8B51A4C94F82039002BFBD159B30144EE
:108250004E1E451ED4F80C29D4F8081915F8017FD4
:10826000531CC3F30A038B422CBF4FF40060002061
:10827000C91A224401440129C4F80C3982F824792E
:108280000FD101203BF0F0FDD4F80839D4F80C19D7
:108290008B4294BF4FF4006200225B1A1344012BFF
:1082A000EFD0B542D6D10020F8BD00BFC0190020E4
:1082B00010B5074CE36A0846114643B1E36A052B43
:1082C00005D1002A236B02DDFFF7BAFF236B10BD37
:1082D000B82A002010B590F85010002380F85030D4
:1082E00061B1094CE26A5AB1E26A052A0AD13C300E
:1082F000236BFFF7A5FF236B012010BD0120FCE7D6
:108300001046FAE71846F8E7B82A0020002280F85D
:108310005120DFE790F85020531C0244DBB280F874
:10832000503082F83C1090F851200AB1132B00D93C
:10833000D0E77047212838B50C4605D022282DD02B
:10834000202812D0002038BD0029FBD0072AF9D1FF
:10835000194B586B93F8381093F8392093F83A304A
:10836000206021716271A371ECE70029EAD0072A2D
:10837000E8D1124AD2F814391BB1D2F810090968B1
:1083800098470D4B256820796179A2795D6383F860
:10839000380083F8391083F83A20D3E70029D1D088
:1083A000022ACFD1054AD2F81C39002BCAD009883D
:1083B000D2F818099847C5E7B82A0020C01900204C
:1083C000014B0020D8627047B82A0020044B054AB0
:1083D00000200521D162C3F81C09C3F814097047B5
:1083E000C0190020B82A0020704700BF704700BFA6
:1083F000704700BF704700BF704700BF704700BFA5
:10840000704700BF08B50248FFF774FE014808BD79
:1084100064390608C019002008B50248FFF76AFE53
:10842000014808BD74390608C019002008B5024883
:10843000FFF760FE014808BD80390608C01900201A
:1084400008B50248FFF756FE014808BD8C390608FA
:10845000C019002008B50248FFF74CFE014808BDCE
:1084600098390608C0190020042301480B80704782
:108470009801002010B4074A074B92F83C001224E0
:1084800003F114020C8001280CBF184610465DF859
:10849000044B7047B82A00209C0100206423014847
:1084A0000B807047C4010020432301480B807047B4
:1084B0002802002010B5074CD4F8D400FF2807D0BC
:1084C00005490A6C4431FFF735FFFF23C4F8D43067
:1084D000002010BD98010020B82A0020EAE700BF64
:1084E00008B5D0F8E4355B6A9847002008BD00BFA6
:1084F00008B5D0F8E4351B6A9847002008BD00BFD6
:10850000D0F8E43510B504461B689847D4F8E83530
:108510009B689847002010BD08B5D0F8E435DB69AA
:1085200003B19847002008BD08B5042290F8121145
:10853000D0F8E83580F8131180F81221DB689847ED
:10854000002008BD10B5D0F8E83504461B699847EF
:10855000032384F81231002010BD00BF0B0617D48E
:1085600001EB810300EBC30310B400EB8100012495
:10857000002283F8764383F8741383F87523426DE1
:108580005DF8044B136843F4001300201360704738
:1085900001F07F0101EB810300EBC303012200EB3B
:1085A000810083F81C1183F81E2183F81D21826944
:1085B0001368002B01DA43F0804343F40013136087
:1085C0000020704782B00023016801930B6901937A
:1085D0000E4B03E00A690192013B13D0019A002A75
:1085E000F8DA019A094B42F001020192019A0A61FC
:1085F0000A69019203E00A690192013B02D0019AE3
:10860000D207F8D4002002B0704700BF400D03002D
:10861000436D064A1A61C278012A06D100F2CC5095
:1086200058614FF0802219681A607047180008607E
:1086300010B580210446FFF791FF20460021FFF787
:108640008DFF2046BDE81040E2E700BF70B44B78D4
:10865000012B26D00B784A6900EB83035C6D2568FB
:108660002369D2B18A684A6102F07F0223F40023B1
:1086700023F07F0342F4002213432361C378012BCC
:1086800004BF0B696361C5F3076363F07B0363F3A6
:108690001F652560002070BC70478A6802F07F0269
:1086A000E4E782694C691568136944B38E68B44283
:1086B0008CBF06F07F0404F07F0423F4002323F032
:1086C0007F0344F4002443EA040388BF4E6113612E
:1086D000C378012B1DD0C5F3076464F07B0464F3F9
:1086E0001F651560002BD5D14B69002BD2D00269D4
:1086F0000878516B012383400B435363CAE723F48B
:10870000002323F07F0343F400231361C378012B7C
:10871000E1D10B780C6900EB8300C5F30763816935
:1087200063F07B0363F31F654C610020156070BC30
:10873000704700BF2DE9F0434B78012B30D00B7808
:108740004C6900EB83035E6D356837691CB38B6839
:108750001C44013CB4FBF3F4C4F3090203FB02F331
:10876000C3F312034B61144643EAC44363F31C078B
:108770003761C378012B04BF0B697361CB78012B80
:1087800044D0C5F3076363F07B0363F31F65356073
:108790000020BDE8F0838A680124C2F31203E3E7F6
:1087A00091F800804E6900EB880EDEF818C0DCF806
:1087B0000050DCF8107076B3D1F80890384A06EB18
:1087C0000904013CB4FBF9F402EAC444C6F3120202
:1087D0002243CC7807F060473A43012C174649D032
:1087E000CCF81020C278012A55D00269516B03FAE7
:1087F00008F30B435363C5F3076363F07B0363F331
:108800001F65CCF800500020BDE8F0834B7973B3AE
:1088100045F00055B5E707F0604747F40027CC78EE
:10882000CCF81070C378012B2FD0012CE3D1026952
:108830009268D20554BF45F0005545F08055C5F308
:10884000076262F07B0262F31F65CCF80050002BD8
:108850009ED1B0B203308010DEF8D04098D0CA6804
:1088600052F8041B216001339842F9D190E745F09A
:10887000805586E764F35E77CCF81070C378012BDF
:10888000D5D10A69CCF81420D1E70A69CCF81420B4
:10889000012CB0D1CBE70B69CCF81430ABE700BFAB
:1088A0000000F81F38B501EB810400EBC4040D464D
:1088B000002184F87453C4F88C1384F87513C4F839
:1088C0008833C4F88023C3782821012B01FB0501DC
:1088D00008BFEDB201F55D7108BFC4F884231DB96E
:1088E000FFF7B4FE002038BDFFF724FF002038BD9D
:1088F00010B501EB8101084A00EBC1010446B1F853
:108900008C131046FFF772FC034A204640230121D6
:10891000FFF7C8FF002010BD042B0020E8E700BFD0
:1089200030B44C780022012C154612D0097800EBA7
:10893000810401238B40646D63F31F4501696FF36C
:10894000CF322260CB6923EA0503002030BCCB6123
:1089500070470B7800EB83019C4064F30F058C6932
:10896000ECE700BF40F2011310B500F5A271044618
:10897000A0F84431FFF7D4FF0123A4F89C3304F599
:1089800067712046FFF7CCFF4FF48173A4F86C3178
:1089900004F5B6712046FFF7C3FFFFF711FD002075
:1089A00010BD00BF38B540F2031304460D46A0F8D1
:1089B000943100F5CA71FFF7B3FF29462046FFF74F
:1089C000D1FF002038BD00BFF0B44B780A78012BEE
:1089D0004FF0000400EB820524D0012393406D6D1D
:1089E00063F31F442E68330415D48A6891F803C0DA
:1089F000CF880F49C2F30A0242F0805343F4004388
:108A00000CF0030243EA824307F00F0243EA825369
:108A100031400B432B600369DA691443DC610020A9
:108A2000F0BC70479340AD6963F30F04DAE700BF11
:108A3000007833EC2DE9F04140F2011304460225A1
:108A40004FF0400801270026A0F84431C0F84C81BF
:108A500080F84751A0F84A7180F8486100F5A2718A
:108A6000FFF7B2FF04F56771A4F89C73C4F8A48300
:108A700084F89F5384F8A0632046FFF7A5FF0822DF
:108A800003234FF48171C4F87421A4F86C1184F8A5
:108A90006F3104F5B671A4F872512046FFF794FFC8
:108AA000064B9D83FFF792FC054A43462046394614
:108AB000FFF7F8FE3046BDE8F08100BF98010020C6
:108AC000042B002070B50323092240F2031604464C
:108AD0000D46C0F89C2180F89731A0F89A31A0F893
:108AE000946100F5CA71FFF76FFF29462046FFF732
:108AF000A1FF002070BD00BF70B5002540260446D0
:108B0000A0F8745380F87753C0F87C6300F55D716A
:108B1000FFF75AFF4FF48073A4F81C3104F58E71EF
:108B2000C4F8246184F81F51A4F822512046FFF7AD
:108B30004BFFD4F8E835A078012284F812215B6855
:108B40009847284670BD00BF82B000230193019A68
:108B5000094B42F010020192C168019A0A610A6948
:108B6000019203E00A690192013B02D0019AD20608
:108B7000F8D4002002B07047400D030082B00023FB
:108B80000193019A0B4B42F020020192019A61F38A
:108B90008A120192C168019A0A610A69019203E08E
:108BA0000A690192013B02D0019A9206F8D4002092
:108BB00002B07047400D03000E4BDA68D20310D4A8
:108BC000DA68D1060FD4DA68D20510D4DA6812F068
:108BD000E00F0AD1DB6813F0020F14BF0820092050
:108BE0007047012070470620704707207047022019
:108BF000704700BF003C024000207047134AD2F883
:108C00008C00C8B1D2F89030B3B1884212D88B42F0
:108C100034BF00230123DBB25BB1D2F89830C2F835
:108C20009410994205D00A4BC2F89810142083F88A
:108C3000D80070470023EEE7A1F59C53083BB3F53D
:108C40007A7F2CBF00230123E6E700BFB82A00206B
:108C500098010020064B93F89D2083F89C108A42CF
:108C600005D0044A83F89D10142082F8D80070477C
:108C7000B82A002098010020704730B1034B93F8C8
:108C80009E00012894BF002001207047B82A0020D0
:108C900008B5FFF7F2FF60B1064A92F89F3092F8EC
:108CA0009C205B0003F00203002A18BF43F001037D
:108CB0000B6008BDB82A002008B5FFF7DEFF18B129
:108CC000024BD3F8A0300B8008BD00BFB82A0020AB
:108CD00070B5FFF7D2FF60B10B4AB2F8A4503DB1B6
:108CE000D2F8A8600023B3421C4603DB002000E05A
:108CF0000D7070BD02EB44040133B4F8AC40AC42DB
:108D0000DBB2F0D10B70F4E7B82A002008B5FFF70A
:108D1000B4FF10B100230B70137008BD042070471E
:108D200028B1034B93F9DA00003818BF01207047CF
:108D30009801002008B5FFF7F3FF50B1054B93F9F8
:108D4000DA20012AC3BF93F8DD30C3F340030B6080
:108D5000002008BD9801002008B5FFF7E1FF18B119
:108D6000024B93F8DC300B7008BD00BF9801002067
:108D700070B5FFF7D5FF38B10E4C94F8DD30DB0746
:108D800003D500230B70137070BD0B4D94F9DB30CD
:108D900095F8BC6093FBF6F301330B7094F9DB405C
:108DA00095F8BC1094FBF1F301FB134301331370EE
:108DB000EAE700BF98010020B82A0020032070478E
:108DC00070B50A4A92F8C03006255E1CB6FBF5F471
:108DD00005FB146492F8C150AC4205D002EBC3030A
:108DE000C3E9310182F8C04070BD00BFB82A00203D
:108DF000002230B504461046914200DC30BDA35C31
:108E00000825584010F0800F4FEA400318BF83F048
:108E1000D503013DD8B2F5D10132EDE710B5E9B186
:108E20000F4BD3F8F400814218DCBAB1D3F8BC3050
:108E30009A4213DC0B4C013A013903FB012184F8FF
:108E4000E81004F1E4000521FFF7D2FF062184F8C1
:108E5000E90004F1E400BDE81040B1E710BD00BF37
:108E6000B82A0020980100200023038083708380AB
:108E7000C3800381704700BF074A92F8F83092F828
:108E8000FC100133DBB2994282F8F83004BF0023B2
:108E900082F8F830704700BFB82A0020F8B5794C46
:108EA000D4F8483283B1D4F84C3293F82E305BB109
:108EB000754B94F85022A3FB0013012A4FEA931339
:108EC00030D0022A08D002B1F8BD704B9842FBD9CD
:108ED000012384F85032F8BDD4F8542264329A4207
:108EE0003ED894F8F83004EB031393F8D426FF2A05
:108EF00006D067490132012083F8D42681F8EA00C0
:108F0000FFF7BAFF94F8C8360122092B84F85022E3
:108F1000DAD1B4F87A3713449BB2A4F87A37A4F8BC
:108F2000CE36F8BD94F8F810C4F854328C2303FB05
:108F3000014394F8C80683F86A22002604F51775E1
:108F40000A220223092884F86662C4F8585284F879
:108F5000672284F85032B7D10131A4F8CC16F8BD9D
:108F600094F8662294F867329A42ADD104F25B20FD
:108F700004F51975002310F8012F082153405A00F9
:108F800013F0800F08BF5B0082F0070214BFD3B25A
:108F9000DBB20139F3D18542EDD194F865229A42D2
:108FA00039D194F8F860B4F85F5294F86372B4F869
:108FB000610294F8643294F85DC204EB06126DBA53
:108FC00040BA43EA0723ADB294F85E7282F8D41631
:108FD000C2F8D85681B22E4D94F95C02C2F8DC1664
:108FE00047EA0C271BB20121032EA2F8D676A2F87D
:108FF000E03682F8D50685F8EA1009D894F8C82634
:109000000C2A2AD00D2A03D104EB4606A6F8CC067A
:10901000FFF732FF5CE794F8F83004EB031393F8A2
:10902000D426FF2A06D01A490132012083F8D4261B
:1090300081F8EA00FFF720FF94F8C8360122092BD7
:1090400084F850227FF440AFB4F8783713449BB2D1
:10905000A4F87837A4F8D036F8BD94F876170D4AFE
:1090600003EB830303EB830349089B0004EB4606F1
:1090700093FBF1F382FB0312DB17C3EBA203A6F809
:10908000CC36C5E7B82A0020D34D62103F4B4C00C8
:1090900098010020676666660B4B93F8661293F89A
:1090A000672291420ED010B493F86622D3F858424A
:1090B000511CD2B2C0B2C9B283F86612A0545DF896
:1090C000044B7047704700BFB82A0020FD2870B5D8
:1090D00022D0F02804D0EF2822D00224204670BDF0
:1090E000114D0320052641282E444FF0000405F1C0
:1090F000010580F080030DD0042B0BD9FFF7E6FFAC
:109100002044B542C4B2E9D015F8010B412880F0E3
:109110008003F1D10420F3E7044D0B200426E2E79D
:10912000034D0C200626DEE7F4390608FC39060854
:10913000EC390608144B30B4D3F87C4714B3002242
:109140000F2583F88217090A83F8810783F88317AC
:10915000C3F88427C3F88827C3F88C2783F880577F
:1091600003F5F060012110F8015F01312A440E2956
:10917000D2B2F8D183F88E272046044930BC1022A1
:109180003BF05ABA30BC7047B82A00203832002071
:10919000034B002183F89017C3F89417CAE700BF68
:1091A000B82A00202DE9F04FDFF88CA3D34D5646A6
:1091B00086468C4617460FCE05F5F3642DED068BDB
:1091C0000FC40FCE0FC496E807008BB095F8563742
:1091D000059784E80700CDE906EC042B00F24681F0
:1091E000DFE813F0B90144013F010500C9019FED1B
:1091F000C48ADFEDC48AC449C5F8B417C349C44B57
:10920000C44AC5F8B0170599002918BF134638EEAF
:10921000887AF5EE006AC6EE879ABF4EC5F8BC376D
:10922000A6F1660B06F1C0080027DFEDBC7A9FEDC2
:10923000BC9A28EE278AB0EE67AA079BBB4200F0D3
:109240000A811BF8012BAB1893F85B47002C00F048
:109250001281002102E0152900F00D8101EB41008F
:109260004B0018F800C0A44501F10101F3D12844D6
:1092700090F88D18002900F06C812046CDE9032379
:1092800039F02CFDDDE9032381464846CDE903236F
:1092900039F06AFE90F800C0BCF1000F40F0EB809E
:1092A000039A049B01322B44D2B2032183F8CD28C8
:1092B00083F8CC18B9F1000F00F0DD802309013BE1
:1092C000032B04F00F0000F208810AEB4304B4F80A
:1092D0002CC04CFA00F414F0010400F03881012491
:1092E00004FA00F0013800EA0C00CDE9032350F045
:1092F000B3FE049BDFF844C2039A5344032193F85E
:10930000343018440CEBC00373619971DA715CF866
:10931000300099F8082000F13F4101F57E010AEB89
:10932000912191F8381001F01F0C4909032904FA22
:109330000CF400F0DC80042900F0D280022900F057
:10934000FF809B880893B3FA83F3C3F11F03C3F331
:10935000CC0100EB810103F007030C6A9B004FF086
:109360000F0C0CFA03FC24EA0C040C620C6A02FADF
:1093700003F323430B62022308A90993FEF76AFE55
:10938000059B002B00F08380B5F85437D5F8801A80
:1093900007EE903AF8EEE77AFCEEE77A17EE900ADD
:1093A000B1FBF0F202F57F42FF32120CB1FBF2F298
:1093B00095F85617B2FBF0F0042983B27ED007EE81
:1093C000902AF8EE676A66EE887A29EE677A95F851
:1093D000570706990091A6EEA87A019049463046B3
:1093E000C6ED027A86ED037A2EF070F9002F70DD5B
:1093F0007368D5F8D02793426DD0012F69D0D5F886
:10940000E827934267D0022F63D0D5F80028934213
:1094100061D0032F5DD0D5F8182893425BD0042F7C
:1094200057D0D5F83028934255D0052F51D0D5F8D4
:10943000482893424FD0062F4BD0D5F86028D31A36
:1094400018BF012301370122082F3374727406F10B
:1094500018067FF4F2AE33480BB0BDEC068BBDE8C6
:10946000F08F9FED318AF0EE488AC4E69FED2F8A97
:10947000F0EE488ABFE62E4A264BC5F8B4270020F6
:10948000C5F8BC370BB0BDEC068BBDE8F08FB0EE75
:10949000690A51F07BFCFCEEC07A4FF6FF7317EEC1
:1094A000902AD5F8801AB1FBF2F21A44120CB1FBE3
:1094B000F2F295F856170429184680D107EE900A63
:1094C00007EE102AF8EE677AF8EE476A67EE8A7AB6
:1094D0007BE70123B6E70023B4E7C6F814C04FE7E3
:1094E0001449D1F830C044EA0C040C6329E711494F
:1094F000D1F840C044EA0C040C6422E7B82A0020EA
:10950000ACC5A737ACC5A736996803088D11040808
:10951000A15C030881110408843200206F12833A91
:1095200000007A4450320020282930386F12033965
:10953000F15D03080038024054C50508B03300202F
:109540000E49D1F844C044EA0C044C64F9E6746155
:1095500016E7894699E69FED0A8A0A4A0A4BC5F83A
:10956000B427C5F8B03700220123CDE90532F0EE6B
:10957000488A064B4BE69FED068AEEE7003802402C
:109580006F12833A996803088D1104088111040849
:1095900000000000F8B50546262026F015F9144C09
:1095A000014600BBD4F8840A90F838301E3B012BEA
:1095B00002D894F8913A0BB13BF072F80D4F0026A7
:1095C000AE4208DBB4F8B23A0133A4F8B23A236BE6
:1095D000C4F8C43AF8BD17F8011BD4F8840A3BF06C
:1095E0005FF80136ECE7002384F8C03AEFE700BFEC
:1095F000B82A00204A35002038B5144C94F8C13000
:1096000094F8C0209A421AD004EBC303D3E9312066
:1096100004F692210023984212DC9378C4F8C80A19
:109620005B0884F8C03AFFF7B5FF94F8C130062113
:109630000133B3FBF1F201FB123384F8C13038BDC2
:10964000D55C01F8015B0133E5E700BFB82A0020D3
:1096500013B504462620019126F0B6F8019920B9E9
:10966000204602B0BDE8104064E502B010BD2DE90F
:10967000F04F244C87B094F8892A01924FF00009EA
:1096800005461E20CDF80C90ADF8149026F09CF8FD
:1096900094F888BA94F88A6AB4F88CAAB4F88E8AD6
:1096A00094F8907A019A28B1B8F1000F02D0C2461E
:1096B0000126CB4694F8CC3AD9070AD494F8D31AA9
:1096C00039B9012F1BD0022F03D113F0020F08BFAD
:1096D00001268DF814708DF80CB08DF80D208DF8E2
:1096E0000E60ADF810A0ADF8128003AB03CB1B8861
:1096F0002860284669602B8107B0BDE8F08F3E46A0
:10970000E7E700BFB82A002007B50DF1060214F004
:10971000C3FB70B1084BBDF80620B3F8F81AA3F8E4
:10972000A420914205D00549A3F8F82A142081F815
:10973000D80003B05DF804FBB82A0020980100208F
:1097400013B50446FFF7ECFA08B300230DF1060247
:109750002046ADF8063014F09FFBC0B10D4C9DF8CB
:10976000062094F9DA1084F8EF20032908BF62F08C
:109770007F024FF00501084808BF84F8EF20FFF78B
:1097800037FB062184F8F0000348FFF719FB02B00D
:1097900010BD00BF98010020830200202DE9F7438F
:1097A000C54CD4F87C370D464BB14FF0020800276A
:1097B0004FF00109D4F87C073AF06EFF60B900263B
:1097C00094F89E30042B00F27281DFE813F09700CA
:1097D000F6000A0157016001D4F87C073AF054FF03
:1097E000D4F894375A1C2344C4F8942783F8FA0A0F
:1097F00094F89037012B0AD0022B11D0002B78D18E
:109800000F280CBF84F89097C4F89437D2E7A0F1E2
:109810007203012B01D976286BD184F89087C9E7B0
:10982000102AC7D1A5490023012211F8010F0132E6
:1098300003440E2ADBB2F8D194F8082B84F8907711
:109840009A42C4F89477B5D194F8093B002BB1D172
:1098500094F8FB6A732E3FD0762E0FD0722EA9D1CA
:1098600094F8FD2A94F8FC3A53EA0223A2D0C4F8F3
:109870008C30B4F8FE3AC4F89030A1E794F8FD2A91
:1098800094F8FC3A53EA022394D094F8FF1A94F81F
:10989000FE2A94F8030BC4F8A03042EA012294F89F
:1098A000001B84F89F1094F8011B84F80C1B94F89B
:1098B000021BA4F80A2B41EA0021A4F80E1BD4F8DD
:1098C000941009B9C4F89430B4F8A430002B7FF494
:1098D00077AFA4F8A42073E794F8012B94F8003B29
:1098E00043EA02231AB2002B3FF464AFA4F8102B12
:1098F00066E784F89077C4F894775BE7722E4ED1D0
:10990000012384F89E30002294F8C836402B36D1CB
:10991000B4F8A400A4F8CE6694F80C6B94F89E30CA
:10992000B4F80ACBA4F8CC360502330394F89C10A3
:10993000D4F8A07005F4706503F440532B434FEA4C
:109940000C1543EA8133EDB22B43D4F894501BB28B
:10995000BD4214BF082500251343604514BF0420F1
:1099600000202B430343B14214BF022100211943BD
:10997000534BA4F8D01693F8D830A4F8D236D4F8C4
:10998000F43023B1D4F8A830002B40F0A3804D4927
:109990004D481F2203B0BDE8F04352F0C8BDD4F8D3
:1099A000143B4A4AEB1A934201DC0022ACE77220D6
:1099B000FFF7EEFBC4F8145BF7E7762E04D1022321
:1099C00084F89E3000229FE7D4F8143B3F4AEB1AFC
:1099D0009342EADD7620FFF7DBFBC4F8145B00223C
:1099E00092E7374FD4F8143B97F8D820EB1AB2B36C
:1099F000364A934236DD94F89F20D2071FD4D4F81C
:109A00009410D4F8A02091420FD089B24620FFF7DD
:109A10001FFE97F8D830C4F8145B013B87F8D830A4
:109A2000042384F89E3001226EE7B4F8A410B4F841
:109A30000A2B8A4203D05020FFF70AFEE9E794F888
:109A40009C1094F80C2B8A4206D0B1FA81F1490996
:109A50004920FFF7FDFDDCE7142287F8D8201C4AD7
:109A60009342B7DC762EA0D17320FFF791FB03233E
:109A700084F89E30C4F8145B002245E7732E94D01E
:109A8000D4F8141B114B691A994298DC8DE7D4F86D
:109A9000143B0E4AEB1A934287DD7620FFF778FBE2
:109AA000022384F89E30C4F8145B00222CE70023C4
:109AB00084F89E301A4627E7B82A0020B2350020E5
:109AC00098010020443A0608890200203F0D030057
:109AD0003F420F00334DD4F8186B2A2385F8F1303C
:109AE0000DF1020220230DF10101304685F8F2301C
:109AF00014F069FA30B19DF801109DF8027051EA36
:109B0000070339D1552385F8F330462385F8F4301F
:109B1000202301A9304685F8F53014F04EFA0346AB
:109B2000214813B1BDF804209ABB204947F07CFDC1
:109B3000B4F80E7B1E4D87B30DF10301304614F0CF
:109B40003FFA50B39DF803100DF10602304614F0B1
:109B5000A3F910B3BDF8062016493B46BA420CBF24
:109B600020222A22284647F05FFDB4F8103BA4F8D3
:109B70001C3B03B0BDE8F083304614F009FA3946C7
:109B800085F8F300304614F0EFF9037885F8F430E7
:109B9000BEE7094947F048FDCAE70849284647F0AB
:109BA00043FDE2E7980100208E020020663A060895
:109BB000920200205E3A0608FE8E0608653A060804
:109BC00038B50B680E4D5A1C0A6005221A700B68D6
:109BD00095F8DA200C46591C21601A70236895F814
:109BE000DD20591C21601A70B5F8E010204642F0C3
:109BF000FBFD236895F8E220591C21601A7038BDDE
:109C0000980100202DE9F0472DED028BFFF788F831
:109C1000C8B31E4B93F9DA00012834DD93F81041E4
:109C20001B4F9FED1C8A15468E1E02EB44084FF019
:109C30003209454504D1BDEC028B2046BDE8F087D2
:109C400037F802AB26F802AF07EE90AAF8EEE70A63
:109C5000B2EE040A60EE880A51F002FABCEEC00AC5
:109C6000BAF10E0F10EE103A9BB209D91933B3FBBB
:109C7000F9F39BB203EB830303EB83035B009BB21B
:109C800025F8023BD5E70024D5E700BF9801002066
:109C9000D6350020CDCCCC3D38B50D46FFF740F889
:109CA000044638B10C4890F8DD30DB0704D5B0F835
:109CB000DE002880204638BD084A90F9DB3092F853
:109CC000BC2093FBF2F102FB11320132013100F5AD
:109CD0008A7014F0F5F8ECE798010020B82A00200B
:109CE0002DE9F047A84D95F82E3B8AB08146002B10
:109CF00040F0B280D5F8186B002E00F0AD80A34A7A
:109D0000D2F8184104F0F021B1F1E02F6BD1C2F884
:109D10001831D5F8302B944265D004930593ADF8F3
:109D20001830B5F88C3A95F888EAADF8143095F803
:109D300089CA95F8903A95F88A8A8DF8183004AF58
:109D40008DF810E08DF811C08DF8128097E80700AB
:109D500007AB03C31A808E4AC5F8304BC4F3425395
:109D6000D15CC4F303428E4502F1010201D1944556
:109D700008D030468DF81C108DF81D2014F0A0F886
:109D8000ADF82000304614F0EEFA032804F0070A7C
:109D900034D0042836D00023984501A9304618BF96
:109DA0008DF81E3014F006F948B1019BC4F3001180
:109DB00003F001038B4202D0304614F0ABF90A22C3
:109DC00007A9384652F04DFB68B19DF81E30BDF82A
:109DD0001C2085F88A3ABDF82030A5F8882AA5F815
:109DE0008C3A43F07FFE95F834AB04AF95F8343BE2
:109DF000032B7BD8DFE803F00A3376A3654B13F817
:109E00000A30C9E7644B13F80A30C5E739463046D3
:109E100014F0D6F8044658B107A8FFF728FC9DF8BF
:109E20001E109DF810308B4260D0304614F0FEF9C1
:109E300095F8343B013303F0030385F8343B0CB948
:109E40009A45D3D195F8CC3ADB0700D524B13368D5
:109E500049461B68304698470AB0BDE8F08701A81C
:109E6000FFF705FC95F8CC8A9DF8044008F001083E
:109E7000ECB1B8F1000F39D13A460DF1030130468B
:109E800014F0A1F8044688B307A8FFF7F0FB9DF88B
:109E90001C109DF803309DF81D208B4203D19DF8C6
:109EA0001030934222D0304614F0CAF9C0E7B8F11E
:109EB000000FBDD13946304614F07FF80446A8B1F2
:109EC00007A8FFF7D4FBBDF82010BDF810308B4277
:109ED0000CD085F8358B85F8368B336830469B6916
:109EE0009847A5E795F8CC3AD80701D500249FE715
:109EF00007A9304614F05EF804460028F6D01E206C
:109F000025F062FC95F8373B83428046EED085F819
:109F1000370B60B1B5F88E3A002BE7D1079BD90714
:109F2000E4D40121304614F0F5F8444680E7079B5D
:109F3000DA07DBD50146304614F0ECF878E738460E
:109F4000FFF795FB97E8070007AB03C31A809DF85E
:109F500010309BB10DF11D0207A9304614F033F803
:109F60000DF11E01304614F02BF80A2207A93846DD
:109F700052F077FA041E18BF012459E708A93046A9
:109F800014F01BF8ECE700BFB82A0020980100206D
:109F90001C3A0608103A0608043A06082DE9F04172
:109FA000FD2984B0044669D0F02949D0EF2900F09A
:109FB000BF804AB10346861803AD002003F8010BA9
:109FC0009E4205F8010BF9D1BA4B0B2003F10905AC
:109FD00001E013F8010F814255D0AB42F9D14B1E7D
:109FE000152B21D8DFE813F0C500D000DA00E70018
:109FF000EE00F400160004010001200020002301FF
:10A000002301230110011001100100012000200094
:10A010001B01AD00A84D95F8CC3ADE0700F16D812B
:10A02000B5F8A43BADF80C303AB1224403AB13F8B9
:10A03000011B04F8011BA242F9D104B0BDE8F08174
:10A040009E4F03214FF00508B844002501370CE06E
:10A05000FFF73CF8064660193246FFF79FFF70197C
:10A060004745C5B2E9D017F8011B412981F08003AB
:10A07000084601D0042BEBD80426ECE7904F0B21C7
:10A080004FF00408E0E78C4BD3F8280C80060CD482
:10A09000002AD2D0224403AB13F8011B04F8011BA1
:10A0A0009442F9D104B0BDE8F08193F8380B10F078
:10A0B000020F93F8500B40D0052834BF022503252A
:10A0C000142917D97C39C8B20628E1D80629DFD867
:10A0D00001A050F821F000BFA9A20008A9A2000821
:10A0E00091A2000891A0000889A2000881A200089E
:10A0F00079A200080929CBD90A390A29C8D801A6AA
:10A1000056F821F065A20008DDA2000891A0000821
:10A1100091A0000891A0000891A0000891A000085B
:10A1200091A0000891A000085BA20008A9A2000865
:10A13000644F0C214FF0060886E70B29A8D10125B2
:10A14000CDE05D4BB3F8C41BCD055ABFCB4303F044
:10A150000103032311F0440F18BF042311F0020F71
:10A1600018BF072311F4806F18BF0923ADF80C3016
:10A170005AE7514BB3F8843B03EB83035B0003F5D1
:10A18000C873ADF80C304FE74F4BD3ED037AFDEEBB
:10A19000E77A17EE903AADF80C3045E7464B93F866
:10A1A000631B002900F0A08001922DF0EFFC019AC2
:10A1B000ADF80C0038E701922DF0E8FC019AADF8FB
:10A1C0000C0031E73C4BD3F8B43BADF80C302BE737
:10A1D000394BB3F8A41B002900F0898001922DF0BF
:10A1E000E1FC019A80B2E3E7334BB3F8263C19E770
:10A1F000314B3649B3F9243C81FB0301DB17C3EB38
:10A20000A103ADF80C300FE72B4B03EB4101B1F884
:10A21000023C03EB83035B00ADF80C3004E7264BF4
:10A2200093F8CC3A03F00103ADF80C30FCE6284B70
:10A23000DFED286AD3ED007A0C39C9B203EB810354
:10A2400093ED127A67EEA67A67EE877AFDEEE77AEB
:10A2500017EE903AADF80C30E6E6B3F84A3BADF8AD
:10A260000C3015E7B3F84C3B03EB830303EB83039C
:10A270009B00ADF80C300BE7D3F8443B039307E7A2
:10A28000D3F8403B039303E7D3F83C3B0393FFE64B
:10A29000B3F84A3B104903EBC3039B00A1FB031334
:10A2A0005B09ADF80C30F3E6B3F8543BADF80C3075
:10A2B000EEE600BFE0390608B82A0020F4390608A7
:10A2C000FC390608EC3906084036002067666666E9
:10A2D0008036002000007A441F85EB51EDB28DF8E6
:10A2E0000C508DF80D00D3E6B3F87C0B60E7D3F883
:10A2F000BC0B80F3100080B25AE7019227F038FCC3
:10A3000005F68833D3ED037A019AFCEEE77A17EE6F
:10A31000903A9BB200287FF485AED5F8C01B11F0AF
:10A32000100F18BF00237DE600F01F024009012333
:10A33000032803FA02F304D004280CD0022805D025
:10A340007047074A116C0B4313647047044A516C01
:10A350000B4353647047024A116B0B4313637047FE
:10A360000038024000487047103400200E4B30B4D3
:10A37000DB68427801780D4CDB43C3F30223C3F161
:10A380000403DBB202FA03F360181B0101F01F059E
:10A390000122490903F0F003AA4080F8003344F891
:10A3A000212030BC704700BF00ED00E000E100E07C
:10A3B000002877D02DE9F04104468088B0FA80F07B
:10A3C00020281F4684B0C0F11F0354D0DFF8E4807A
:10A3D000354D08EB03064FF0004C05EB83033CFAC8
:10A3E00000F096F84060C3F82C1C05D02F4B19687C
:10A3F00021EA0001196058611146204638F0C8FF73
:10A40000A3882168B3FA83F3C3F11F0202F0FC00B2
:10A4100000F1804000F59C3002F0030294004FF000
:10A420000F0C01F13F4281680CFA04FC21EA0C0197
:10A43000816002F57E0208EB8707D0F808C0396D0D
:10A440008DF80D10C2F38722A24042EA0C024FF0B1
:10A450000041354421FA03F382600021012202A861
:10A4600002938DF80C108DF80E20FDF7C9FD95F8BC
:10A470006C3CF02B02D804B0BDE8F0810C4B9B5D26
:10A480008DF80430F02103224FF4807301A885F881
:10A490006C1C8DF80520ADF80630FFF767FF04B09F
:10A4A000BDE8F081704700BFB82A0020003C0140A1
:10A4B0003C3A060854C5050800286BD0F0B58388DF
:10A4C000B3FA83F3202B85B00446C3F11F024CD0AE
:10A4D000314D32484FF00041104405EB820205F641
:10A4E000744731FA03F390F84060C2F82C7C05D031
:10A4F0002B4A116821EA03011160536120460021B3
:10A5000038F046FFA3882268B3FA83F4C4F11F032E
:10A5100003F0FC0101F1804101F59C3103F00303DC
:10A5200098000F2702F13F438A68874022EA07021A
:10A5300003F57E038A60C3F38723834088684FF066
:10A5400000420343354422FA04F48B604FF4406226
:10A55000012302A88DF80E300294ADF80C20FDF70F
:10A560004FFD95F86C3CF02B01D805B0F0BD0D4BBC
:10A570009B5D8DF80430F02103224FF4807301A815
:10A5800085F86C1C8DF80520ADF80630FFF7EEFE5F
:10A5900005B0F0BD704700BFB82A002054C50508BB
:10A5A000003C01403C3A0608454B5B68C3F3080396
:10A5B0002DE9F041002B61D1EFF31183002B5DD128
:10A5C000404A414C116BA068136B9942FAD1D2F802
:10A5D000803C9842F6D8D2F87C5C4FF47A7404FB45
:10A5E00005F3181AB0FBF5F004FB0101344D3648B1
:10A5F00010264FF47A7401276B68C3F30803E3B99C
:10A60000EFF31183CBB9136BD0F808E0D2F830C068
:10A610006345F8D1D2F880CCE645F4D8D2F87C8CEA
:10A6200004FB08FCACEB0E0CBCFBF8FC04FB03C306
:10A630005B1A772BE0D9BDE8F081EFF3118E86F33A
:10A640001288D0F808800368DB0344BFC2F8787C26
:10A65000D0F80880D2F830C0D2F8783C5FFA8EFE8D
:10A660008EF31188D2F87CEC634404FB0EFCACEB57
:10A67000080CBCFBFEFC04FB03C3D9E7EFF311801D
:10A68000102383F3128810490E4A8D680B68DC038F
:10A6900042BF0123C2F8783C8D68136BD2F8781C56
:10A6A000C0B280F31188D2F87C4C4FF47A70194410
:10A6B00000FB04F35B1BB3FBF4F300FB013195E7F4
:10A6C00000ED00E0B82A002010E000E0464B5B6897
:10A6D000C3F308032DE9F041002B62D1EFF311839E
:10A6E000002B5ED1414A424C116BA068136B99421A
:10A6F000FAD1D2F8803C9842F6D8D2F87C5C4FF47C
:10A700007A7404FB05F3181AB0FBF5F004FB0101A1
:10A71000354D374810264FF47A7401276B68C3F320
:10A720000803EBB9EFF31183D3B9136BD0F808E04A
:10A73000D2F830C06345F8D1D2F880CCE645F4D8E1
:10A74000D2F87C8C04FB08FCACEB0E0CBCFBF8FCD8
:10A7500004FB03C35B1AB3F57A7FDFD3BDE8F08156
:10A76000EFF3118E86F31288D0F808800368DB03BC
:10A7700044BFC2F8787CD0F80880D2F830C0D2F854
:10A78000783C5FFA8EFE8EF31188D2F87CEC63443D
:10A7900004FB0EFCACEB080CBCFBFEFC04FB03C38F
:10A7A000D8E7EFF31180102383F3128810490F4A82
:10A7B0008D680B68DC0342BF0123C2F8783C8D68CA
:10A7C000136BD2F8781CC0B280F31188D2F87C4C9D
:10A7D0004FF47A70194400FB04F35B1BB3FBF4F3F2
:10A7E00000FB013194E700BF00ED00E0B82A002033
:10A7F00010E000E02DE9F84FB34C94F8841C0546B6
:10A80000C1F34001D4F88C0C3DF0FAF994F8841CA3
:10A81000D4F8880CC94301F001013DF0F1F9002D95
:10A8200000F0C3806E1EA94FA94D5FFA86FB4FF062
:10A830001008D4F88C0C3DF0C7F9D4F8880C3DF022
:10A84000C3F9B4F8943C002B40F0358194F8961C81
:10A85000D4F8980C3DF0D4F94FF0FA094FF47A701F
:10A860004FF0010C7B68C3F30803002B40F0FB8022
:10A87000EFF31183002B40F0F680226BA968236B65
:10A880009A42FAD1D4F8803C9942F6D8D4F87C6C3C
:10A8900000FB06F35B1AB3FBF6F300FB02327B68A6
:10A8A000C3F30803002B40F09F80EFF31183002BCC
:10A8B00040F09A80236BD5F808A0216B8B42F9D128
:10A8C000D4F8801C8A45F5D8D4F87C6C00FB06F1DE
:10A8D000A1EB0A01B1FBF6F100FB03139B1AB3F5E0
:10A8E0007A7FDCD3B9F10109BCD1D4F88C0C3DF0EE
:10A8F0006BF9D4F8880C3DF067F9B4F8943C002B60
:10A9000040F0CD8094F8961CD4F8980C81F00101A9
:10A910003DF076F94FF0FA0C4FF47A704FF0010EDB
:10A920007B68C3F30803002B7ED1EFF31183002B68
:10A930007AD1226BA968236B9A42FAD1D4F8803C71
:10A940009942F6D8D4F87C9C00FB09F35B1AB3FB60
:10A95000F9F300FB02327B68C3F308033BBBEFF360
:10A96000118323BB236BD5F808A0216B8B42F9D14F
:10A97000D4F8801C8A45F5D8D4F87C9C00FB09F1FA
:10A98000A1EB0A01B1FBF9F100FB03139B1AB3F52C
:10A990007A7FE0D3BCF1010CC2D10BF1FF365FFA34
:10A9A00086FBBBF1FF0F7FF444AFBDE8F88FEFF3F8
:10A9B000118988F31288AE682B68DB0344BFC4F8A2
:10A9C00078ECAE68236BD4F8781C5FFA89F989F3C8
:10A9D0001188D4F87C9C0B4400FB09F1891BB1FB66
:10A9E000F9F100FB0313D1E7EFF3118E88F312881E
:10A9F000D5F808A02B68D90344BFC4F878CCD5F8A3
:10AA000008A0236BD4F8781C5FFA8EFE8EF31188B1
:10AA1000D4F87C6C0B4400FB06F1A1EB0A01B1FBFE
:10AA2000F6F100FB031359E7EFF3118188F3128865
:10AA3000D5F808902B68DA0344BFC4F878ECD5F851
:10AA40000890236BD4F8782CC9B281F31188D4F81C
:10AA50007C1C1A4400FB01F3A3EB0903B3FBF1F3E5
:10AA600000FB023277E7EFF3118188F31288AE68BA
:10AA70002B68DB0344BFC4F878CCAE68236BD4F8F2
:10AA8000782CC9B281F31188D4F87C1C1A4400FBDD
:10AA900001F39B1BB3FBF1F300FB0232FFE6D4F89A
:10AAA000B03C002B3FF436AFD4F89C3CC3F8009088
:10AAB00084F8AD9C2EE7D4F8B03C002B3FF4CCAE2C
:10AAC00039F096FAC8E600BFB82A002000ED00E091
:10AAD00010E000E02DE9F84FB04CB14F94F8841C21
:10AAE000D4F88C0CAF4DC1F340013DF089F894F8D7
:10AAF000841CD4F8880CC94301F001013DF080F8B2
:10AB00004FF0050B4FF01008D4F88C0C3DF05CF8BA
:10AB1000D4F8880C3DF058F8B4F8943C002B40F081
:10AB2000358194F8961CD4F8980C3DF069F83226DB
:10AB30004FF47A704FF0010C7B68C3F30803002BCD
:10AB400040F0FA80EFF31183002B40F0F580226B88
:10AB5000A968236B9A42FAD1D4F8803C9942F6D87E
:10AB6000D4F87CEC00FB0EF35B1AB3FBFEF300FBA6
:10AB700002327B68C3F30803002B40F09E80EFF3A2
:10AB80001183002B40F09980236BD5F808A0216B2E
:10AB90008B42F9D1D4F8801C8A45F5D8D4F87CECE6
:10ABA00000FB0EF1A1EB0A01B1FBFEF100FB031368
:10ABB0009B1AB3F57A7FDCD3013EBDD1D4F88C0C5F
:10ABC0003DF002F8D4F8880C3CF0FEFFB4F8943C59
:10ABD000002B40F0D08094F8961CD4F8980C81F0AB
:10ABE00001013DF00DF84FF0320C4FF47A70012660
:10ABF0007B68C3F30803002B7FD1EFF31183002B95
:10AC00007BD1226BA968236B9A42FAD1D4F8803C9D
:10AC10009942F6D8D4F87C9C00FB09F35B1AB3FB8D
:10AC2000F9F300FB02327B68C3F308032BBBEFF39D
:10AC3000118313BB236BD5F808A0216B8B42F9D18C
:10AC4000D4F8801C8A45F5D8D4F87C9C00FB09F127
:10AC5000A1EB0A01B1FBF9F100FB03139B1AB3F559
:10AC60007A7FE0D3BCF1010CC2D10BF1FF3616F0B4
:10AC7000FF0B7FF449AFBDE8F88FEFF3118988F33C
:10AC80001288D5F808A02B68DB0344BFC4F8786CA1
:10AC9000D5F808A0236BD4F8781C5FFA89F989F3FA
:10ACA0001188D4F87C9C0B4400FB09F1A1EB0A014C
:10ACB000B1FBF9F100FB0313D0E7EFF3118E88F33A
:10ACC0001288D5F808A02B68D90344BFC4F878CC03
:10ACD000D5F808A0236BD4F8781C5FFA8EFE8EF3AB
:10ACE0001188D4F87CEC0B4400FB0EF1A1EB0A01B7
:10ACF000B1FBFEF100FB03135AE7EFF3118188F378
:10AD00001288D5F808902B68DA0344BFC4F8786C31
:10AD1000D5F80890236BD4F8782CC9B281F3118848
:10AD2000D4F87C1C1A4400FB01F3A3EB0903B3FB2A
:10AD3000F1F300FB023276E7EFF3118188F312881A
:10AD4000D5F808E02B68DB0344BFC4F878CCD5F80D
:10AD500008E0236BD4F8782CC9B281F31188D4F8B9
:10AD60007C1C1A4400FB01F3A3EB0E03B3FBF1F3CD
:10AD700000FB0232FDE6D4F8B03C002B3FF433AFC9
:10AD8000D4F89C3C1E6084F8AD6C2CE7D4F8B03C41
:10AD9000002B3FF4CCAE39F02BF9C8E6B82A0020DE
:10ADA00000ED00E010E000E010B4B8B10D4CD4F8B4
:10ADB000B43C102B05D15DF8044B0521002038F080
:10ADC000CFBD03EB4302224482F8B91C01210B449E
:10ADD00082F8B80C82F8BA1CC4F8B43C5DF8044B95
:10ADE000704700BFB82A002000285FD00368374AA8
:10ADF0002DE9F04103F13F4404F57E0402EB942277
:10AE0000012492F8382002F01F055209032A04FA9F
:10AE100005F456D0042A4FD0022A48D08588B5FAC6
:10AE200085F0C0F11F00C0F3CC0603EB860600F0EE
:10AE3000070082000F24306A944020EA0400306248
:10AE4000306A01FA02F20243002132624FF0010E31
:10AE50000A464FF0030C02270EFA02F838EA050002
:10AE600002F101021CD118680CFA01F420EA040076
:10AE70001860186807FA01F606431E609E6826EA05
:10AE800004069E6098689860586820EA0800586038
:10AE900058685860D86820EA0400D860D868D8603C
:10AEA000102A01F10201D7D1BDE8F0817047084AAC
:10AEB000556C2C435464B1E7054A156B2C4314635D
:10AEC000ACE7034A156C2C431464A7E754C5050886
:10AED0000038024070B5464E96F8E84C04EB440347
:10AEE00006EBC303650093F8EC3C032B6ED8DFE858
:10AEF00003F059291E02254406EBC505D5F8F00CD0
:10AF0000002870D196F84C3D9C425FD0013404F08B
:10AF10000302934286F8E82C58D002EB420406EB79
:10AF2000C4040223C4F8F00C84F8EC3C70BD2B1967
:10AF300006EBC303D3F8F02C72B1013AC3F8F02C3E
:10AF4000002070BD2B1906EBC303D3F8F02C002AA8
:10AF5000F3D1022283F8EC2C254406EBC50595F8C5
:10AF6000F83C013BDBB285F8F83C8BBB214B96F8F3
:10AF70004C6DD3F81C11D5F8F40C621C02F00302DE
:10AF80004B1E0324B242034485F8EC4CB3FBF1F0B2
:10AF9000C5F8F00C1AD0994218D80138C5F8F00C51
:10AFA000012070BD3EF00EFF80B1124B2C44D3F84F
:10AFB0001C2106EBC404012102F51C5384F8EC1C8F
:10AFC0000F33B3FBF2F3C4F8F03C70BD012070BD49
:10AFD000084BD3F81C21012002F2E733B3FBF2F354
:10AFE000C5F8F03C70BD0138C5F8F00C002070BD0C
:10AFF000B82A0020980100202DE9F04FAF4EB04D47
:10B0000095B0002304460F464FF4F072202106F558
:10B010005560019486F84D3D86F84E3D51F049FA51
:10B02000202106F573604FF4F07251F042FAA54901
:10B03000BB4632244FF0100C4FF47A7001276B6836
:10B04000C3F30803002B40F0B780EFF31183002B0C
:10B0500040F0B280326BD1F80880336B9A42F9D15C
:10B06000D6F8803C9845F5D8D6F87C9C00FB09F3CF
:10B07000A3EB0803B3FBF9F300FB02326B68C3F3E5
:10B080000803002B78D1EFF31183002B74D1336BBD
:10B09000D1F808A0D6F830804345F8D1D6F8808C96
:10B0A000C245F4D8D6F87C9C00FB09F8A8EB0A0846
:10B0B000B8FBF9F800FB03839B1AB3F57A7FDDD365
:10B0C000013CBCD1804C627E002A50D0A37E013B63
:10B0D000022B4CD803EB830504EBC50104F1B4004B
:10B0E00091F8B4C000EBC500BCF1020F4FF00105B0
:10B0F000E06184F8A45000F0A882DBB204EB0313F3
:10B10000D3F82C31C1F8B8308BB302204FF48073E0
:10B1100081F8B400A1F8C03004F12C0004F16803F8
:10B12000C1E933031509013D032D02F00F0200F2BE
:10B130007082DFF8A08108EB4503988D40FA02F396
:10B14000DB0740F16682012303FA02F2013A104064
:10B1500045444EF081FF95F834205C4B104403EBDE
:10B16000C00060628379002B46D0412B44D06FF041
:10B17000010015B0BDE8F08FEFF311898CF3128850
:10B18000D1F808A00B68DB0344BFC6F8787CD1F87F
:10B1900008A0336BD6F8788C5FFA89F989F31188A7
:10B1A000D6F87C9C434400FB09F8A8EB0A08B8FBDE
:10B1B000F9F800FB03837FE7EFF311888CF3128823
:10B1C000D1F808900B68DA0344BFC6F8787CD1F850
:10B1D0000890336BD6F8782C5FFA88F888F31188DA
:10B1E000D6F87C8C1A4400FB08F3A3EB0903B3FBED
:10B1F000F8F300FB023241E72323C380092138F032
:10B20000C7F8636A13B11A689B881383D6F8802A3B
:10B210002F4BB3EB920F80F01E82B3EBD20F80F076
:10B220001C82B3EB121F80F01D82B3EB521F80F023
:10B230001E82B3EB921F80F01F82B3EBD21F80F00F
:10B240002082B3EB122F80F01E824FF48072002315
:10B250000DF10D01FF2022840122CDE90413CDE977
:10B260000833CDE90A33E1698DF80D000D9306929C
:10B270008DF81C208DF83020EFF31180102383F31C
:10B280001288E3691B6A002B00F0C681069B04AD9F
:10B290002A461BB1D3691432002BFBD10B6A002B59
:10B2A00000F00882996839B99A4218D0196899B1A2
:10B2B0005B6899680029F7D01433F3E7B82A0020B7
:10B2C00000ED00E010E000E0B03B0020B0330020D3
:10B2D000404B4C0054C50508AF4AC3E90025C0B235
:10B2E00080F31188E1690B6A002BFCD18C220120CC
:10B2F000CDE908330DF10E080DF10F0A05938DF815
:10B300001C300D93109312938DF80E200023002211
:10B31000CDE90E23CDF8108006900B908DF830000B
:10B320008DF84400CDF828A0EFF31180102383F3AB
:10B330001288E3691B6A002B00F07781069B2A467E
:10B340001BB1D3691432002BFBD10B6A002B00F028
:10B35000B181996839B993420AD0196829B15B68FB
:10B3600099680029F7D01433F3E78B4AC3E9002525
:10B37000C0B280F31188E269136A002BFCD19DF8FA
:10B380000F301B2B40F08781636A012286F84D2D18
:10B390000BB12322DA80DFF80092402248460A21CE
:10B3A0003EF03AFC8A21002301228DF80E10002085
:10B3B0000021CDE90E01CDE90833E169CDF8108017
:10B3C000CDF828A005938DF81C300D93109312939F
:10B3D00006920B928DF830208DF84420EFF3118007
:10B3E000102383F31288E3691B6A002B00F0258188
:10B3F000069B2A461BB1D3691432002BFBD10B6A82
:10B40000002B00F05481996839B9934209D019682A
:10B4100029B15B6899680029F7D01433F3E7C3E9D1
:10B420000095C0B280F31188E269136A002BFCD149
:10B430009DF80F20217EC2F3801284F85C21002940
:10B4400000F0CA80022900F0AD80D6F8803A534956
:10B45000B1EB930F80F01981B1EBD30F80F0FF8037
:10B46000B1EB131F80F00081B1EB531F80F001811D
:10B47000B1EB931F80F00281B1EBD31F80F0088104
:10B48000B1EB132F34BF4FF4807C4FF0800C96F853
:10B49000C816A4F85EC118290ED14149A6F8CCB649
:10B4A0005B08B3FBFCF3A1FB03135B0BA6F8CE26F2
:10B4B000A6F8D0C6A6F8D2363748A4F820C0022293
:10B4C00000213EF0A9FBC82038F092FBE0694FF064
:10B4D000800B0026002700230122CDE90E67CDE96D
:10B4E00008338DF80EB0CDF81080CDF828A0059364
:10B4F0008DF81C300D931093129306920B928DF8D9
:10B5000030208DF84420EFF31181102383F312884B
:10B51000E3691B6A002B36D0069B2A461BB1D36910
:10B520001432002BFBD1006A002800F0BD80836834
:10B530003BB9824209D003682BB140688368002B75
:10B54000F7D01430F3E7C0E90095C9B281F3118850
:10B55000E069036A002BFCD19DF80F3013F0020361
:10B56000B9D1019841788278007884F86001C1F1FE
:10B570002001C2F11002184684F8611184F862219A
:10B5800015B0BDE8F08F0562C9B281F31188024899
:10B590004DF0FEFADCE700BFCC3B0020809698001F
:10B5A0005917B7D1D6F8803A4448B0EB930F79D207
:10B5B000B0EBD30F53D2B0EB131F55D2B0EB531FE8
:10B5C00057D2B0EB931F59D2B0EBD31F34BF4FF01B
:10B5D000800C4FF0400C5AE7D6F8803A3849B1EB6E
:10B5E000930F52D2B1EBD30F39D2B1EB131F3BD231
:10B5F000B1EB531F3DD2B1EB931F3FD2B1EBD31F41
:10B6000046D2B1EB132F34BF4FF4807C4FF0800C47
:10B610003DE700206062F1E504ADC0B20D6280F349
:10B62000118828484DF0B4FA5CE60D62C0B280F390
:10B63000118824484DF0ACFA9DE60D62C0B280F34B
:10B64000118848464DF0A4FAEEE691F8C1302B443B
:10B6500081F8C13066E50222F9E50422F7E54FF0F2
:10B66000040C14E70822F2E54FF0080C0FE7102253
:10B67000EDE54FF0100C0AE72022E8E54FF0200C32
:10B6800005E74022E3E58022E1E54FF0020CFEE60B
:10B690004FF0400CFBE6606A202137F079FE4FF056
:10B6A000FF3066E58C46F2E6C0F80090FFDEC3F896
:10B6B0000090FFDE034A1A60FFDE00BF002D31015B
:10B6C000404B4C00CC3B002038B50C4C0546A11C2F
:10B6D000D52242F08FF82B68A342C5E90043A3EBC3
:10B6E00004000AD004F14002611C2960237802F8AA
:10B6F000013BD5E90041A142F6D138BD143D0020FF
:10B70000F0B40D6800240CE0BCF1050F18D8A0F1CE
:10B7100037030A2B14D104EB840415F8010B03EB57
:10B720004404A0F13003DEB2092EA0F16107A0F1BC
:10B73000410CF0D9052FE7D8A0F157030A2BEAD026
:10B740000D601460F0BC704710B5204B84B0C82465
:10B7500003F5D27103F265122128CDE9022183F8A5
:10B76000644118D00CD802281ED0082825D102A880
:10B77000019009F06BFF0198FFF7A6FF04B010BD20
:10B7800029281AD102A8019009F016FE0198FFF7A6
:10B790009BFF04B010BD02A8019009F057FE01986C
:10B7A000FFF792FF04B010BD02A8019009F09EFFC0
:10B7B0000198FFF789FF04B010BD02A8019009F0BD
:10B7C000BBFE0198FFF780FF04B010BDB03B002026
:10B7D000014488420ED010B40346074C074813F8C2
:10B7E000012B04FB00F0994280EA0200F7D15DF8DA
:10B7F000044B70470148704793010001C59D1C81AF
:10B80000094B93F85637042B08D9053B032B08D86E
:10B8100001231A4600B1037010467047002301222D
:10B82000F8E700231A46F5E7B82A00209FED727A60
:10B8300007EE901A20EE070AF8EE677A27EE800AE4
:10B84000FDEEC07A17EE903A2033402B00F2C48010
:10B85000DFED6A7AB4EEE70AF1EE10FAF0EE407A24
:10B860000CDD9FED676ADFED676AB0EE677AB4EED4
:10B87000E67AF1EE10FA77EEC67AF6DC9FED627AA0
:10B88000F4EEC77AF1EE10FA0CD59FED5D6ADFEDAC
:10B890005F6AB0EE677AB4EEE67AF1EE10FA77EE10
:10B8A000867AF6D49FED5A7AF4EEC77AF1EE10FA62
:10B8B00000F38A809FED577AF4EEC77AF1EE10FA22
:10B8C00044BF9FED517A77EE677A27EEA76ADFEDE6
:10B8D000525A9FED527ADFED526AA6EE257A67EE54
:10B8E000865AE6EE076AB6EE007AE5EEA67A27EE0D
:10B8F000877ADFED476A70EE267ABDEEE76A16EECC
:10B90000103A2033402B64D8B4EEE60AF1EE10FA78
:10B910000CDDDFED3B5A9FED3B6AF0EE676AF4EE1B
:10B92000C66AF1EE10FA77EEE57AF6DCDFED366AFC
:10B93000F4EEE67AF1EE10FA0CD5DFED315A9FED18
:10B94000336AF0EE676AF4EEC66AF1EE10FA77EE4B
:10B95000A57AF6D4DFED2E6AF4EEE67AF1EE10FA6F
:10B960003DDDDFED266A76EEE77A67EEA75A9FEDBA
:10B970002A5A9FED2A6ADFED2A6AA5EE856A27EE2C
:10B98000A55AE5EE866AB8EE006AE5EE267A67EE1D
:10B99000867AC7EE206AB7EE006A76EE865A76EEB1
:10B9A000666A86EE257A80ED091A67EE277A66EEDA
:10B9B000876AC0ED017AC0ED037A80ED007A80EDF0
:10B9C000027AC0ED046A70479FED0C7A77EE677AD1
:10B9D0007BE7DFED147ADCE79FED127A89E7DFED94
:10B9E0000D6AF4EEE67AF1EE10FA44BFDFED066A76
:10B9F00076EEE77AB9E700BF27D4D236DB0F4940AD
:10BA0000DB0FC940E4CB1641DB0F49C0E4CB16C1C4
:10BA1000DB0FC93FDB0FC9BF92E741B99730083C44
:10BA200015A82ABE000000002DE9F843E14FD7ED2C
:10BA30007A7A97F86047F8EE670A07F25C732DEDA3
:10BA4000028BC3ED000A002C70D1DFF8C4E3DFF8ED
:10BA5000C4C39EF8FC60C7F86C479CF80040002EF9
:10BA600039D0B7F866379FEDD46A9FEDD47A07EEE8
:10BA7000903AF8EE677A20EE877AC6EE276AD04BC6
:10BA80000022012E1A6076EE876AC7EE267AC3ED91
:10BA9000017A20D0022E9A60C3ED037A1BD0032EC8
:10BAA0001A61C3ED057A16D0042E9A61C3ED077AA8
:10BAB00011D0052E1A62C3ED097A0CD0062E9A62B7
:10BAC000C3ED0B7A07D0072E1A63C3ED0D7A02D0AF
:10BAD0009A63C3ED0F7A9EF876379FEDBA6A9FEDB1
:10BAE000BA7A9FEDBA0ABA4A07EE903AF8EEE77AC8
:10BAF0009CF8583BC6EE276A1C4414FB06F6F6B2C7
:10BB000007EE906A60EE870AF8EEE77AC2ED006A07
:10BB1000A7EEA00A4FF046FABDEC028BFCEEC07A0D
:10BB200017EE903A87F87437BDE8F88397F86137D5
:10BB3000DFEDA84A9FEDA82ADFEDA86ADFF8D0E282
:10BB4000DFF8D0C29EF8FC60C7F86CC707EE903AE9
:10BB5000B7F864378CF8004007EE103AFCEEE05A74
:10BB6000B7F8623706EE103A15EE903AF8EE655ADD
:10BB7000F8EE677A84EEA55ACCF81430012387F8E2
:10BB80006837B8EEC77A27EE822AB8EE466A67EEC3
:10BB9000266A22EE252A8CED025ACCED017A8CED34
:10BBA000036ACCED046A002E95D0DFED8D7A9FED0F
:10BBB0008D4ADFED8D5AC7EE871AC6EB0615A6EB48
:10BBC00006190CEBC5054FEAC9094FF00008B1EEA4
:10BBD000611A9FED866A09EB05009FED853ADFED5E
:10BBE000853ADFED856A0346002207EE902AB8EE1B
:10BBF000E77A27EE027AFDEEC77A17EE901A203127
:10BC0000402900F2D080B4EEC47AF1EE10FAF0EEE2
:10BC1000477A0CDDDFED794A9FED795AF0EE672A1D
:10BC2000F4EEC52AF1EE10FA77EEE47AF6DCF4EEE3
:10BC3000E57AF1EE10FA0CD5DFED704A9FED715AFE
:10BC4000F0EE672AF4EEC52AF1EE10FA77EEA47A48
:10BC5000F6D4F4EEC67AF1EE10FA40F39A8074EE60
:10BC6000677A27EEA75AB0EE630AA5EE030ADFED66
:10BC7000664AE5EE004A65EE272AB7EE005AE2EE84
:10BC8000A47AB0EE458AF0EE454AA1EEA78AE1EE2D
:10BC9000274AC5EE088A84EE880A77EE067ABDEE5A
:10BCA000E75A15EE101A203140296FD8B4EEC67A43
:10BCB000F1EE10FA0CDD9FED515A9FED517AF0EE46
:10BCC000674AF4EEC74AF1EE10FA77EEC57AF6DC71
:10BCD000F4EEE57AF1EE10FA0CD59FED485A9FED9F
:10BCE000497AF0EE674AF4EEC74AF1EE10FA77EEC1
:10BCF000857AF6D4F4EEC67AF1EE10FA3CDD74EEF5
:10BD0000677A27EEA75AF0EE632AE5EE032A9FED45
:10BD10003E7AA5EE227A65EE274AB8EE005AE4EEA6
:10BD2000877A67EE857A87EE887A0132A24203F13C
:10BD3000280343ED048A03ED037A03ED017A43ED12
:10BD4000028A83ED000AC3ED056AC3ED026AC3ED02
:10BD5000016AC3ED046AC3ED036AFFF646AF7830AB
:10BD600085427FF43AAF08F57078B8F5346F05F581
:10BD700070757FF42EAF74E69FED247AF4EEC77AE7
:10BD8000F1EE10FA48BF75EEE77ABAE7F0EE667AA0
:10BD9000C9E79FED1E5AF4EEC57AF1EE10FA48BFDE
:10BDA00075EEE77A5DE7B7EE000AF0EE408AB0EE96
:10BDB000408A72E7B03B002083F9223EBD378635CA
:10BDC00028430020555555406E12833A48E1FA3E0B
:10BDD000204300200060EA4827D4D2360AD7233C0B
:10BDE00000004842DB0F4940DB0F49C0DB0FC93F71
:10BDF00092E741B99730083C00000000DB0FC940D2
:10BE0000E4CB1641E4CB16C115A82ABEDB0FC9BF8F
:10BE1000B82A0020047300202DE9F04F07EE900AA5
:10BE20002DED068B9FEDF07AF049DFEDF16AB1F868
:10BE3000B83791F8BE57C1F81008B8EE679A0AEE05
:10BE4000103A87EE095AB1F8BA37C1F8CC57002238
:10BE500083B0C1F8D02708EE103AB1F8BC37DFED57
:10BE6000E57AB8EE4AAA08EE903AB8EEC88A3AEEF9
:10BE70000A7AF8EEE88AB4EEC78AF1EE10FA68EEB4
:10BE8000A77AB4EEE65A01F5F863B8BFB0EE478A78
:10BE9000F1EE10FA83ED028A83ED01AAC3ED007A78
:10BEA00000F1008307EE905AF8EEE77AB7EE007AD9
:10BEB000C7EE279AD04BDFF87CA3184614309C4677
:10BEC00001909AF88C2003F12C04F6EE005A65EEEE
:10BED000256AF7EE007A86EE887ADFEDC83ADFED64
:10BEE000C84A9FEDC86AD3ED05AAB4EEE77AF1EE31
:10BEF00010FAB8BFB0EE677ABDEEC77AB0EE004A6E
:10BF000017EE106AB8EEC77AC1F86C6AC5EE076A18
:10BF100087EE875A66EEA36AACEC015A8AEE267A5F
:10BF2000C8EE267A37EE257A77EEA57AB4EEC47A93
:10BF3000F1EE10FAB8BFB0EE447AF4EEE47AF1EE26
:10BF400010FABDEEC77A88BFF0EE647A17EE107A69
:10BF5000FDEEE77A07F1FF3B17EE900ABBF1230FE6
:10BF6000A8BF4FF0230BCCED006A012E00F1010CAD
:10BF7000B8BF0126BCF1230F2BEAEB7BE04629EE8C
:10BF8000066AA8BF4FF02308E345C8BFD846C1F8EA
:10BF9000787A83ED046AA8EB0B07C1F87C0A97FB5B
:10BFA000F6F70137002A40F0E380DFED970ADFED76
:10BFB000975A9FEDA12A9FED965ADFEDA32A9FED98
:10BFC000A33ADFEDA33A9FED934ADFEDA21A0AF1FF
:10BFD000900107EE902AB8EEE76A66EE207A37EE17
:10BFE000A57AFDEEC76A16EE903A2033402B00F298
:10BFF0001282F3EE026AB4EEE66AF1EE10FA0CDD9C
:10C00000DFED8F4ADFED8D6AB0EE471AB4EEE61A27
:10C01000F1EE10FA37EE647AF6DCB4EEC57AF1EEA2
:10C0200010FA0CD5DFED864ADFED866AB0EE471ACE
:10C03000B4EEE61AF1EE10FA37EE247AF6D4B4EE46
:10C04000E57AF1EE10FA40F3FB81DFED736A36EE2C
:10C05000C77A67EE076AB0EE431AA6EEA21AB0EEF0
:10C06000630AA1EE260A67EE264AFDEEE76AA4EE11
:10C07000807A16EE903A2033402B27EE047A00F2B5
:10C08000D481DFED666AB4EEE66AF1EE10FA40F3B1
:10C09000FD819FED6B0A9FED691AF0EE676AF0EE85
:10C0A000664AF4EEC14AF1EE10FA76EEC06AF6DCAA
:10C0B0009FED591AF4EEC14AF1EE10FA13D59FED37
:10C0C000601ADFED604AB0EE660AB4EEE40AF1EE03
:10C0D00010FA76EE816AF6D4DFED506AB4EEE66AC5
:10C0E000F1EE10FA0CDD9FED566ADFED546AF0EECA
:10C0F000674AF4EEE64AF1EE10FA77EEC67AF6DC1D
:10C10000F4EEC57AF1EE10FA0CD59FED4D6ADFED35
:10C110004D6AF0EE674AF4EEE64AF1EE10FA77EE79
:10C12000867AF6D4F4EEE57AF1EE10FA40F38081E7
:10C13000DFED396A76EEE77A67EEA76AF0EE434AFA
:10C14000E6EEA24AB0EE631AA4EEA61A27EEA66A9D
:10C15000E6EE017A67EE847A0132242A81ED007AD4
:10C16000C1ED017A01F108017FF433AFDFED2CAAB4
:10C170004FF0000944E9059B44E902764FF49072C0
:10C180000021204644F80C8C50F093F94FF4907243
:10C19000A018002150F08DF9224B04F51574A3422C
:10C1A000E8D1019BDFED207AC3ED00AA012329EE3F
:10C1B000279A8AF88C30002D00F02881DFED1B7A59
:10C1C0001B4E9FED152ADFED122AC7EEA81AA6F125
:10C1D000140406F5117738EE4A8AB1EE611A69EE59
:10C1E000889ADFED0A5A3BE000247449B03B0020F6
:10C1F0000000FA440AD7233C20460020398E633CD5
:10C2000000000C429C534937C3B8B23DDB0FC93F15
:10C21000DB0F49C072F97F3FDB0F4940000010423D
:10C22000BC297E3F484D002027D4D236000048422A
:10C2300084430020A84C002000000000E4CB1641FD
:10C24000DB0FC940E4CB16C192E741B99730083CF7
:10C2500015A82ABEDB0FC9BF000010C20000807FF6
:10C260005FED0B6A234630460022B7EE005A07EE18
:10C27000902AF8EEE77AB6EE007A77EE877AB0EE9B
:10C280004A7AA7EEA97AF0EE477A29EE077AE0EC2F
:10C29000017AFDEEC77A17EE901A2031402900F29C
:10C2A000D780B4EEC27AF1EE10FAF0EE477A0CDDE8
:10C2B0001FED1D4A5FED1F4AB0EE676AB4EEE46AF7
:10C2C000F1EE10FA77EEC47AF6DCF4EEE27AF1EEF3
:10C2D00010FA0CD51FED264A5FED264AB0EE676ACC
:10C2E000B4EEE46AF1EE10FA77EE847AF6D4F4EE66
:10C2F000E57AF1EE10FA40F3B58072EE677A67EEF8
:10C30000A74A5FED2F3A1FED2F4A1FED2F6AA4EECB
:10C31000A34A67EEA43AA4EE246AF0EE454AE3EE9F
:10C32000867AB0EE456AE1EE274AA1EEA76A84EE6E
:10C33000864AC5EE064A77EE257AFDEEE73A13EE19
:10C34000901A2031402900F28A80B4EEE57AF1EEAD
:10C3500010FA0CDD1FED463A5FED483AB0EE677A11
:10C36000B4EEE37AF1EE10FA77EEC37AF6DCF4EE8F
:10C37000E27AF1EE10FA0CD51FED4F3A5FED4F3A2D
:10C38000B0EE677AB4EEE37AF1EE10FA77EE837AE4
:10C39000F6D4F4EEE57AF1EE10FA6DDD72EE677A1E
:10C3A00027EEA73A5FED580A5FED583A1FED587A2D
:10C3B000E3EE203A63EE270AA3EE237AF8EE003A82
:10C3C000E0EE877A67EEA37A87EE867A0132AA4298
:10C3D00003F12803C3ED0B4A83ED0C7A83ED0E7A4B
:10C3E000C3ED0D4A83ED0F4A83ED145AC3ED116A74
:10C3F000C3ED106AC3ED136AC3ED126A7FF437AF61
:10C40000C834A74206F114067FF4EBAE03B0BDECCE
:10C41000068BBDE8F08FFDEEE76AB0EE427A16EECD
:10C42000903A2033402B7FF62CAEF0EE427A93E622
:10C43000F4EEE17AF1EE10FA48BF75EE677A7BE62A
:10C44000B4EEE17AF1EE10FA48BF35EE477A00E635
:10C45000B7EE004AF0EE444AB0EE446A6BE7F0EE05
:10C46000667AB1E71FED856AF4EEC67AF1EE10FA4E
:10C4700048BF72EEE77A42E71FED8A7AF4EEC77A98
:10C48000F1EE10FA48BF72EEE77A89E75FED8E6A47
:10C49000B4EEE66AF1EE10FA48BFF0EE676A3FF5D7
:10C4A0000EAE2DE65FED939AC1F8CC27154601E557
:10C4B00010B582B00A788DF80720040A18238DF889
:10C4C00004308DF806008DF805404AF023FC01AADF
:10C4D0000348114604233DF0F5FB02B010BD00BF38
:10C4E000584E002010B582B0040A192200238DF89E
:10C4F00001408DF800200C468DF803308DF80200C5
:10C500004AF008FC6A460548114605233DF0DAFB6F
:10C510009DF80430237002B010BD00BF584E0020BB
:10C5200070B4447941BB03684FF400524FF4007675
:10C53000202502213CBB1A8C22F001021204120CAD
:10C540001A841A8B188C22F0F30280B2120420F0A5
:10C550000A00120C014342F0010241F001011A836A
:10C5600019841A8B22F00C021204120C1A831A8BF3
:10C5700092B270BC1A8370470022036816461546B3
:10C580001146002CD7D0042C21D0082C38D0198C7F
:10C5900021F480510904090C19849C8B1D8C45F6EB
:10C5A000FF7040F6FF4128402140024342F4805290
:10C5B00041F4807199831A849A8B22F440621204A8
:10C5C000120C9A839A8B92B270BC9A8370471A8C21
:10C5D00022F010021204120C1A84188B198C89B2E2
:10C5E00040F6FF4221F0A00102400D4342F4807268
:10C5F00045F010051A831D841A8B22F44062B3E7BC
:10C600001A8C22F480721204120C1A84998B1A8CE0
:10C6100021F0F30192B2090422F42062090C3243A2
:10C6200042F4807241F0010199831A849A8B22F0BE
:10C630000C02C4E70B88F0B433BB028C4C880E8923
:10C640008B88C98822F001021204120C0284058B27
:10C65000028CADB225F0F30592B22B4322F00A0210
:10C6600043EA061322439BB242F001020383028491
:10C67000038B23F00C031B041B0C0383038B9BB263
:10C680001943F0BC01837047042B048C2CD0082B79
:10C690004E888A880D89C98851D024F48054240496
:10C6A000240C0484838B078C2C0344EA022440F678
:10C6B000FF421A4045F6FF733B4043EA06332243EC
:10C6C0009BB292B243F4805382830384828B22F420
:10C6D00040621204120C8283838B9BB243EA0123D3
:10C6E0009BB2F0BC8383704724F010042404240C14
:10C6F0004D880F898A88C9880484068B038C1202AE
:10C700009BB242EA073423F0A00340F6FF423240D6
:10C7100043EA051322439BB292B243F01003028313
:10C720000384028B22F440621204120C0283038BF6
:10C730009BB243EA01239BB2F0BC0383704724F40D
:10C7400080742404240C0484848B038CA4B29BB2D4
:10C7500024F0F30423F42063224343EA062342EA4D
:10C7600005129BB243F4807392B282830384838B5D
:10C7700023F00C031B041B0C8383838B9BB2194394
:10C78000F0BC8183704700BF2DE9F04F7D4C94F8D9
:10C79000BE8494F8C9A487B016460B220546894684
:10C7A0004046114602959DF840701D4636F012FC39
:10C7B000C245834640F0A680039040463AF030FFE1
:10C7C00017F008030246019300F09080BBF1000FC0
:10C7D00000F088809BF80710890700F18380C4E986
:10C7E000A20BC4F8840210B140F60B31C18005F0F1
:10C7F000020ADFF8A881029B634A84F84C5208F5CC
:10C8000080710025C4E997815846C4F874323146D6
:10C810004FF48073C4E99533C4F84822C4E99955AC
:10C82000C4E99B55C4F8506284F84D72C4F87892FC
:10C83000C4F8A05484F8A454A4F898542AF090FDA5
:10C84000D4F88C0207F00101FFF76AFE4F4A504B03
:10C85000D4F88C02C4F8AC54C4F8B024C4F8A8349A
:10C86000BAF1000F25D0D4F8907217B33A68036874
:10C870009A421ED001233146384684F8A5342AF066
:10C880006FFDD4F8900208F50572294635F004FFD3
:10C89000D4F88C022A4608F5077135F0FDFE019B9D
:10C8A00093B93C482AF074FD3A4801212AF0A8FDCA
:10C8B0000AE0394A002302F1080184F8A53435F072
:10C8C000EBFE019B002BECD032482AF06DFD314885
:10C8D00007B0BDE8F08FCDE90403039B13B1D9790C
:10C8E0008B0716D5002007B0BDE8F08F15F00103C7
:10C8F000F1D105F002018A46BAF1000F22D1D4F835
:10C900008CB276E70B220C21504636F063FB039085
:10C9100053E750463AF084FE039AC4F88C2215F08F
:10C92000020ADDE90423C4F8840205F0020123D0E1
:10C93000904219D0C0B140F60C3CA0F806C0BAF144
:10C94000000FDCD0B8F1000FCCD0C4F8882283B936
:10C95000BBF1000FC6D0C4F88CB212B140F60B3355
:10C96000D3805FFA81FACAE7B8F1000FBAD0C4F8F1
:10C970008822C4F890B2F0E70028DCD1DDF80CB0D2
:10C9800037E700BFA84C0020B0C50508B56703080D
:10C9900019740308F04E0020505100203C4F002035
:10C9A000F0B5C54BC54EC64DC64C0822C3F888200D
:10C9B000336B83B043F00103336307464FF4C05237
:10C9C000284640F202336946CDE90023FBF742FBDB
:10C9D0006A6AC4F8BC7A22F470426A626A6ABA4B24
:10C9E000C4F8C03A42F420426A626A6AB748C4F89E
:10C9F000D80422F470226A626A6AB548C4F8DC047A
:10CA000042F420226A62726CB24DC4F8E85442F4D7
:10CA100080427264726BB048C4F8F00442F0800245
:10CA20007263022284F8E024AC4FAD4AAD49C4F8E9
:10CA3000F4741C334FF0A046C4F8C43AC4F8E4645C
:10CA4000A94BC4F8F82405F5487506F51666C4F830
:10CA50003055C4F83435C4F8FC640123DFF8B4C29F
:10CA6000C4F82CC507F51077A5F5E465A2F5A0621A
:10CA7000A6F58C66C4F83875C4F8EC54C4F8A4253F
:10CA800084F8E33405F5A0754B61C4F86865194670
:10CA9000A03684F8EA35954BC4F8705502F59072CB
:10CAA000A7F5BC67A035C4F87C65914EC4F8742521
:10CAB000C4F8787502F52A6207F5D457C4F88035B2
:10CAC000C4F8845503F569534FF050250020ACF5A8
:10CAD000BC6CC4F8A825C4F8AC7502F5A04207F5F3
:10CAE000A047C4F8B065C4F8B43506F5A046A3F570
:10CAF0004853C4F8B85504F59B65C4F8BC25C4F880
:10CB0000C465C4F8E435C4F86CC50246C4F8C07501
:10CB10002B4684F8EC05402683F81C21A3F822213B
:10CB20000132042AC3E9496083F81D1183F81F010B
:10CB3000C3F8300103F12803EED1002211462B4641
:10CB4000402083F87423A3F87A230132042AC3E92E
:10CB5000DF0183F8751383F87713C3F8881303F1A3
:10CB60002803EED14FF0A04362489A6822F00102F8
:10CB70009A60DA6842F04002DA60FBF723FD94F82D
:10CB8000E1340022212161F317420BB142F48012FB
:10CB900094F8DB14D4F8E43401299A6300F0DF80C0
:10CBA000DA68D4F8E465D4F8E804C2F3076121F048
:10CBB000600141F0400161F31F620021DA603160E1
:10CBC000026861F3CC22026094F8E324012A00F0A9
:10CBD000B38010214848FBF7D1FF4748FBF7B4FF6B
:10CBE000D4F8E80494F8D93400224FF0FF31026100
:10CBF00042618161C26153B305F114073F4E114692
:10CC000007EB83074FEA830C4FF0FF0E56F8042F13
:10CC10001368002BACBF00234FF09043B742136062
:10CC20001161C2F808E0F1D105F1500334496344C1
:10CC30000027FF2651F8042F1568002DACBF0025F2
:10CC40004FF090459942156017619660F2D10369E3
:10CC500094F8DB1443F48073012903615CD0D4F8A9
:10CC6000E42428480023936100294FF0FF336FF03C
:10CC7000804151615360516114BF002310239061C2
:10CC800043F470139069D4F8C01A43F4605343F02E
:10CC90000803034393619368096843F001039360B9
:10CCA0008847194B194ADA606846194B0093FDF71B
:10CCB0005DFB03B0F0BD00BF00E100E000380240C2
:10CCC00000000240A84C0020B80200200804010027
:10CCD00040004001000800500009005020090050A9
:10CCE00040090050003C0140400B0050C00500507E
:10CCF000003000508C5100208051002094510020C1
:10CD0000D05100200008008000ED00E00005FA0589
:10CD100043020001000B0050D4F8E424144B0363D9
:10CD20006FF08041134D00234FF0FF30936151614C
:10CD3000506051619561A3E701680F4A0F4E41F0C1
:10CD400003010160802159629E62C3F80421E02240
:10CD5000C3F80821C0F24002C3F80C2139E79A68F1
:10CD600022F03E0141F02A0161F307029A6017E7C1
:10CD70000301810000080080A00040008000200026
:10CD8000036870B55E6A26B133460522BDE870407F
:10CD9000184704460D464E1D00E023689B68204658
:10CDA00098470028F9D0236815F8011B1B68204616
:10CDB0009847B542F1D170BD0A44914217D010B4E2
:10CDC0000139541E11F8013F08225840430010F069
:10CDD000800F08BF400083F0D50314BFD8B2C0B2A3
:10CDE000013AF3D1A142EDD15DF8044B7047704791
:10CDF0002DE9F047164D0746002095F9D19A05F622
:10CE0000D82684B007EB010805F6785504464FF0A4
:10CE1000B60A3368ABB193F83830142B11D019F13E
:10CE2000020F01D04B450CD1002269463046CDE9B6
:10CE30000244CDE90078ADF808A08DF80D402BF044
:10CE4000E7FEE036B542E4D104B0BDE8F08700BFAC
:10CE5000A84C00202DE9F0479AB0DDE9226ADDF800
:10CE6000909004460D461746984602E0206837F039
:10CE70000BFC206837F010FC0028F7D10146642233
:10CE800001A84FF016FB264B8DF80450CDF85CA09E
:10CE90000293002D3FD0AB1E012B3ED9042D14BFB1
:10CEA000002203221F4B03961B6B8DF805201E44A6
:10CEB0000123CDE9059404968DF85B3037B14246E5
:10CEC000394607A84FF094FA8DF85A80164E96F816
:10CED000BA9D00231893B9F1000F19D196F8B90D36
:10CEE000642202FB006001A900F6BC504FF080FAFA
:10CEF000012386F8B99D86F8BA3D236843B14346BD
:10CF00003A46294620461AB0BDE8F04710F046BA26
:10CF10001AB0BDE8F0870522C4E70222C2E700BFCD
:10CF2000205A0020B82A0020A84C00200C480D4BA5
:10CF3000D0F83C1E10B40C4CC0F82C3E8A1E223196
:10CF4000B0F85A3E1B01A4FB03C3DB08A3F5B06392
:10CF500022F8023F9142F3D15DF8044B704700BFC5
:10CF6000A84C0020B11C0208CDCCCCCC70B5084C2C
:10CF7000251D2E4614F8010B2EF0D6FA28B10378A1
:10CF800005F8013BB442F5D170BDFF23F8E700BFBF
:10CF9000285B00202DE9F0471D4F012607F1080509
:10CFA000B2464FF03C094FF0000817F8010B3AF079
:10CFB00037FB044690B180F80690C671FB7803F009
:10CFC0007F02012A18D013F0800F20460DD185F87A
:10CFD00004803AF009FE85F805802C600136052EA4
:10CFE00005F10805E1D1BDE8F08785F804A03AF025
:10CFF00001FE85F805A0F0E71B0605D401212046B7
:10D0000036F0C6F9FB78DEE73AF0F4FDF6E700BF4C
:10D01000305B00202DE9F04FDFF8FC91DFF8FCA138
:10D0200083B009F10C06012419F8018BB8F1000F47
:10D0300000F0C5804FEA1815013D032D08F00F02DE
:10D0400000F2C0800AEB4503988D40FA02F717F012
:10D05000010700F0D28001239340013B1840554462
:10D060004CF0FAFF95F83430664F184407EBC007D0
:10D0700004237761FC71BB71002302E0152B00F0E3
:10D080009E8003EB43026049895C41454FEA430BB4
:10D0900003F10103F2D15D4B1A4492F88D18002977
:10D0A00000F0AD80404635F019FE0546284635F0C3
:10D0B0005BFF0378002B40F08280544B5B440422DA
:10D0C00083F8CD4883F8CC28002D78D0002F5DD090
:10D0D0003B68287A03F13F4202F57E020AEB922276
:10D0E0004FF0010C92F8382002F01F015209032A78
:10D0F0000CFA01F171D0042A67D0022A75D0B7F872
:10D1000004E0BEFA8EF2C2F11F02C2F3CC0103EBBF
:10D11000810102F007020F6A92004FF00F0C0CFA27
:10D1200002FC27EA0C070F620F6A90403843002286
:10D1300008624FF0010B11460BFA01FC3CEA0E00AD
:10D1400001F101011ED118680327974020EA07006A
:10D150001860D3F800800220904040EA0800186070
:10D16000986820EA0700986098689860586820EAF4
:10D170000C00586058685860D86820EA0700D860EA
:10D18000D868D860102902F10202D5D1204B214A7B
:10D19000B3F8B01EB3F8B23E009100200134019004
:10D1A000B2FBF3F330469BB22946E4B22AF08EFA82
:10D1B0000123092C737406F118067FF435AF03B010
:10D1C000BDE8F08F0027776156E7DFF854C0DCF840
:10D1D00030200A43CCF8302091E7DFF844C0DCF877
:10D1E00040201143CCF8401089E7DFF834C0DCF868
:10D1F00044201143CCF8441081E777613CE70D46A9
:10D2000054E700BFB033002044330020B82A002088
:10D21000A84C002040420F005C5B002054C505086C
:10D22000003802402DE9F0412A4C2B4DB4F8846FB0
:10D23000A5F8946C82B0EEB994F8800F3AF0F0F94A
:10D2400094F8812FC5F8980C003A18BF012285F890
:10D25000962C48B194F8821F2B22002914BF11216B
:10D260000121C28036F094F8002002B0BDE8F04100
:10D270003BF0FABE94F8808F002240462B2135F017
:10D28000A9FE074640463AF0CBF9F8B1F7B12B2298
:10D29000C5F8B00CC280397AFDF7A6FD4FF0000842
:10D2A0000E4AB2FBF6F3C3F34F0000909BB239462F
:10D2B000CDF8048005F69C40A4F8866F2AF006FAA3
:10D2C000D5F89C3CC3F8008085F8AD8C02B0BDE871
:10D2D000F08100BFA84C0020B82A002040420F0077
:10D2E0002DE9F84F254C94F8943F84F8883F04F6D4
:10D2F0008B77002604F6A8745FFA86FB0BF1010811
:10D300005FFA88F8012117F8010F42460E448A4659
:10D3100035F060FE4FF00009054640B3387804F858
:10D320000E9C04F80D9C04F80FBC04F810AC44F8F3
:10D33000045C3AF075F918B180F806A080F807800F
:10D34000297AFDF751FD0E4A0021284635F0D0FA22
:10D350000C4B23600C4B221D21462846C4E90139A1
:10D3600035F09AF9697928684A462AF043F9082E77
:10D3700004F11C04C0D1BDE8F88F00BFA84C002008
:10D3800040420F002D760308715A030870B52C4DEA
:10D390002C4B15F8380C45F8403C0022022125F8AA
:10D3A0003C2C45E9202245F8782C45F8442C35F0F2
:10D3B00011FE002842D0244B0268044603F1C0004D
:10D3C000597C11B159688A422CD018338342F7D165
:10D3D0001E4E15F8380CC6F8A44F002386F8983F67
:10D3E0003AF01EF908B10223C380217AFDF7FCFC54
:10D3F0002046174A002135F07BFA164A1649C6F82E
:10D40000A81F0025111F2046144BC6F8AC3FC6F8D4
:10D41000B05F35F041F9617920682A46BDE8704077
:10D420002AF0E8B8138D0E490E4A9BB2D2F8802A32
:10D430000133B2FBF3F381F85831C9E770BD00BF87
:10D44000A05D002000FFFF0084320020A84C0020D7
:10D4500040420F00545C0020995A0308355C0308D1
:10D4600098010020B82A00202DE9F04FCD4DCE4C78
:10D4700085B007460E4605F2CC70C02200214FF061
:10D4800018F894F83430002B00F0E48094F835302C
:10D49000002B00F0FD8095F86437012B70D0022B33
:10D4A00000F00281DFF824C3BF4C95F85AE7BCE8CE
:10D4B0000F0027460FC7BCE80F000FC79CE8070006
:10D4C00095F85637DFF808C3C4F818C0BEF1000C51
:10D4D00018BF4FF0010C072B87E8070084F837C00E
:10D4E00000F23381042B00F23F81DFF8E8B20394AD
:10D4F000ABF166034FF000081C4646454FF00301B0
:10D500003CDD14F801AB05EB0A030AF1010993F8BD
:10D510005B775FFA89F938464A4635F05BFD03468A
:10D5200038461F46002B00F018813AF079F8CBF806
:10D53000140020B14FF00303837180F8079095F831
:10D54000572795F856375FFA88F1002A00F00381D3
:10D55000FA7982F0010200923846524608F1010839
:10D560004AF0C6F8002800F0F8804FF00103B8F147
:10D57000080F8BF811300BF1180BBED18A4B67E006
:10D58000DFF854C2894FDFF84C82E663BCE80F0035
:10D590000FC7BCE80F000FC79CE8070095F8563787
:10D5A00095F85AC784F87C300023BCEB030C87E85D
:10D5B000070018BF4FF0010C9B4607F19400194675
:10D5C0004FF44C7284F837C084F8383007F5717A1C
:10D5D0004EF06FFFA8F1660903965E46E36BB34217
:10D5E00040F3AA8019F8013B2B4493F85B77384647
:10D5F00035F076FD834638463AF012F895F85737FD
:10D600000746002B00F09B809BF8073083F0010B4E
:10D610000BF0010194F83700013184F8361008B19D
:10D620008BF0010B002F00F0AE80B87900285AD0A3
:10D63000412858D05E4B5F495F4A44F8183C039E2E
:10D6400044F81C1C012384F8383044F8102C0023C3
:10D65000C5F84C32D5F84C325BB10022012183F879
:10D660002C6083F82D101A6383F82E2005B0BDE8D6
:10D67000F08F524E524C0FCE0FC40FCE0FC496E80F
:10D680000700A4F1200384E80700C5F84C32EDE759
:10D6900095F85827003A384618BF01223146FBF763
:10D6A00081FDC5F84C02D5E795F85A37002B3FF4B9
:10D6B000F9AE95F85637082B7FF462AFDFF80CC14E
:10D6C000DFF80CE1BCE80F0027460FC7BCE80F00ED
:10D6D0000FC79CE80700012387E8070084F837306C
:10D6E000C4F818E034E0B888CAF80C704901B0FA00
:10D6F00080F041F009010136C0F11F004FF0030333
:10D70000CAF80400CAF814108AF810B0FE71BB7190
:10D71000384635F03DFE1BF0010F384612D03AF086
:10D7200063FADAF80C30C8F81430082E0AF1200A2F
:10D7300008F118087FF452AF039E1C4B88E79BF852
:10D7400007B065E73AF056FAEBE7082B7FF4CDAE69
:10D750001C4B2364C9E6FA79FDE6039C164B144A78
:10D760006362E261002373E795F85937164A226431
:10D77000012B05D0022B06BFBEFA8EF35B090023F6
:10D7800084F84430B1E6490141F009014FF0FF331C
:10D79000CAF81410CAF80430CAF80C708AF810B02D
:10D7A0000136B5E7B82A0020A05D00206C5D00209E
:10D7B000891104088D11040881110408E0C50508C9
:10D7C000E85D0020FD1104082D1204080CC60508B0
:10D7D0006D5705088432002038C605082DE9F84F3A
:10D7E000D34F97F8540E97F8555E39F019FF60B192
:10D7F0002D23C3802021044635F0CAFD0A2036F0CF
:10D80000F7F920463BF064FC20B9CA4BD3F8B0349A
:10D81000DE0001D5BDE8F88F013D092DFAD897F853
:10D82000535ED5B940202FF009FD0028F2D090F9C1
:10D83000043097F8251E092BC8BF143B3B440A2926
:10D8400093F8B45400F0B18193F8BF3497F8522E96
:10D85000002A08BF1D46002DDCD0284639F0E0FE26
:10D860008046002800F099812D23C380012135F0E6
:10D870008FFD012108463AF0CBF9D8F80030B8F80E
:10D8800004201A833C2036F0EFFA002101203AF000
:10D89000BFF997F8553E002B00F0CC80A64CDFF87E
:10D8A000A092A64D002694F8841CD4F8880CC94395
:10D8B00001F001013AF0A4F994F8841CD4F8900C1A
:10D8C00081F00401C1F380013AF09AF9B8F1000F38
:10D8D00004D0D8F80030B8F804205A83D9F80430BE
:10D8E000C3F30803002B40F0FF80EFF31183002BFC
:10D8F00040F0FA80226BA968236B9A42FAD1D4F8DF
:10D90000803C9942F6D8D4F87CCC4FF47A7000FB76
:10D910000CF35B1AB3FBFCF300FB02324FF0100C6C
:10D920004FF47A710120D9F80430C3F30803002BB7
:10D9300040F0BA80EFF31183002B40F0B580236BE9
:10D94000D5F808B0D4F830E07345F8D1D4F880ECBD
:10D95000F345F4D8D4F87CAC01FB0AFEAEEB0B0E19
:10D96000BEFBFAFE01FB03E39B1A772BDBD994F88D
:10D97000841CD4F8880C01F001013AF041F994F8C4
:10D98000841CD4F8900CC1F380013AF039F9B8F155
:10D99000000F04D0D8F80030B8F804201A83D9F862
:10D9A0000430C3F30803002B40F0CC80EFF3118365
:10D9B000002B40F0C780226BA968236B9A42FAD1F2
:10D9C000D4F8803C9942F6D8D4F87CCC4FF47A70E5
:10D9D00000FB0CF35B1AB3FBFCF300FB02324FF0CD
:10D9E000100C4FF47A710120D9F80430C3F3080306
:10D9F000D3BBEFF31183BBBB236BD5F808B0D4F8CE
:10DA000030E07345F8D1D4F880ECF345F4D8D4F87D
:10DA10007CAC01FB0AFEAEEB0B0EBEFBFAFE01FB7B
:10DA200003E39B1A772BDFD997F8553E01369E42C8
:10DA3000FFF639AF97F8533E002B40F0A680D7F899
:10DA4000543E03F0FF13B3F5803F7FF4E3AE394B50
:10DA5000D3F8B03413F080537FF4DCAE87F8553E32
:10DA6000BDE8F84F40F03EB8EFF3118A8CF312880E
:10DA7000D5F808B02B68DB0344BFC4F8780CD5F8A0
:10DA800008B0236BD4F878EC5FFA8AFA8AF311882D
:10DA9000D4F87CAC734401FB0AFEAEEB0B0EBEFB6C
:10DAA000FAFE01FB03E3BCE7EFF3118A8CF3128863
:10DAB000D5F808B02B68DB0344BFC4F8780CD5F860
:10DAC00008B0236BD4F878EC5FFA8AFA8AF31188ED
:10DAD000D4F87CAC734401FB0AFEAEEB0B0EBEFB2C
:10DAE000FAFE01FB03E33FE7EFF31181102383F319
:10DAF0001288D5F808C02B68DA0304D50123C4F8CE
:10DB0000783CD5F808C0236BD4F8782CC9B281F3DF
:10DB10001188D4F87C0C4FF47A711A4401FB00F39D
:10DB2000A3EB0C03B3FBF0F301FB0232F6E600BFFC
:10DB3000A84C0020A05D0020B82A002010E000E0E2
:10DB400000ED00E0EFF31181102383F31288D5F884
:10DB500008C02B68DA0304D50123C4F8783CD5F853
:10DB600008C0236BD4F8782CC9B281F31188D4F89B
:10DB70007C0C4FF47A711A4401FB00F3A3EB0C0305
:10DB8000B3FBF0F301FB023229E7322036F06CF9E7
:10DB90004046002135F0FCFB51E7012135F0F8FB50
:10DBA000012108463AF034F86CE6074CD4F8C03B43
:10DBB0005C057FF52FAE08F0B1F800287FF42AAE9F
:10DBC000002D7FF44AAE25E6B82A00202DE9F04169
:10DBD000214E224F96F8B73487F8843C06F2B446BB
:10DBE00007F6884500244FF0050816F8010B20BB06
:10DBF00028600134032C05F10405F6D197F8841C44
:10DC0000D7F8880CC94301F0010139F0F9FF97F802
:10DC1000841CD7F88C0C81F00201C1F3400139F06B
:10DC2000EFFF97F8841CD7F8900C81F00401BDE851
:10DC3000F041C1F3800139F0E3BF39F0F1FC013468
:10DC400001212860E3B210B180F80680C371286812
:10DC500035F09EFBCEE700BFA05D0020B82A002073
:10DC60000B6810B414681B1B036054684B681B1BC3
:10DC700043608B6892685DF8044B9B1A8360704721
:10DC80002DE9F047041E0D4612DB092C26DC824AE2
:10DC90000B468248A0FB0410C00800EB8000A4EBF8
:10DCA00040000021125C1A7059702846BDE8F087C8
:10DCB00064422D23092C01F8013B24D8764A774B86
:10DCC000A3FB0403DB0803EB8303A4EB4303002063
:10DCD000D35C48700B702846BDE8F0876F4B632C0F
:10DCE000A3FB04264FEAD60621DC6B4A0B466B49A0
:10DCF000A1FB0601C90801EB8101A6EB4101515CC2
:10DD000003F8011BC5E7654A632CA2FB04364FEA02
:10DD1000D60637D8604A614BA3FB0603DB0803EB4A
:10DD20008303A6EB4303D35C01F8013BC7E7A3FBE6
:10DD30000627B4F57A7F4FEAD7070DD2564A0B462D
:10DD40005649A1FB0701C90801EB8101A7EB41017D
:10DD5000515C03F8011BCAE7A3FB072842F20F72CC
:10DD600094424FEAD80836D84B4A0B464B49A1FBA0
:10DD70000801C90801EB8101A8EB4101515C03F8DE
:10DD8000011BDDE7A2FB0637B4F57A7F4FEAD70720
:10DD90000CD2414A414BA3FB0703DB0803EB83038F
:10DDA000A7EB4303D35C01F8013BB4E7A2FB0738C0
:10DDB00042F20F739C424FEAD80821D8364A374BBB
:10DDC000A3FB0803DB0803EB8303A8EB4303D35C4B
:10DDD00001F8013BDEE7324AA3FB080994424FEA0F
:10DDE000D90921D82C4A0B462C49A1FB0901C908A5
:10DDF00001EB8101A9EB4101515C03F8011BB5E77F
:10DE0000274BA2FB08099C424FEAD90921D8224A94
:10DE1000224BA3FB0903DB0803EB8303A9EB4303BA
:10DE2000D35C01F8013BCAE71E4AA3FB09039442F5
:10DE30004FEAD30A21D80B461849174AA1FB0A0119
:10DE4000C90801EB8101AAEB4101515C03F8011BF8
:10DE5000CAE7144BA2FB09029C424FEAD20A13D82C
:10DE60000E4B0D4AA3FB0A03DB0803EB8303AAEB6B
:10DE70004303D35C01F8013BCAE70A22BAFBF2F084
:10DE80003FF048FC0346D7E70A22BAFBF2F03FF026
:10DE900041FC0146E4E700BFA8390608CDCCCCCC54
:10DEA0009F8601003F420F0070B4344890F8B834A8
:10DEB000A3F13001092957D800F59764224600F2F2
:10DEC000C74012F8015FA5F13001092904D8824248
:10DED000F7D1002070BC7047141B022C4ADD284883
:10DEE000002101E010F8013B01EB810103EB41034C
:10DEF000161A303B022E044603F0FF01F2DC214BE0
:10DF000003FB01F1A2424FF000030DD903EB8303A1
:10DF100014F8016B5B00303B3344A24203F0FF0373
:10DF2000F4D1194800FB03F32E2D06D01748A0FBAF
:10DF3000032301EB930070BC7047013204200024DE
:10DF4000157804EB8404303D6400092D00F1FF30A6
:10DF5000A4B202D82C44A4B2013210F0FF00EFD1D9
:10DF6000642202FB0433E1E700211D4600F59762BD
:10DF70000B46D9E7064C0021C4E700BFA05D002096
:10DF8000596200208096980040420F00ABAAAAAACE
:10DF90005862002038B504460D460A460068FF2145
:10DFA0004EF087FA21682944216038BD83B50C46BC
:10DFB000164605462DF070FC20462DF06DFC002124
:10DFC000204B0846002E08BF1E4639F021FE0021D6
:10DFD000012039F01DFE284636F05EFBB0B101216C
:10DFE000002039F015FE284636F04EFB0746204645
:10DFF00036F04EFB0028FAD03946204636F050FB6A
:10E000003846B0470021084639F002FE204636F077
:10E0100043FB0028DFD00121002039F0F9FD204624
:10E0200036F032FB01462846019136F031FB01996A
:10E030000028F8D0284636F033FB0021084639F096
:10E04000E7FDC8E7BDB50308F0B50023C1E900331B
:10E05000C1E902330B610268DFF888C089B004AD02
:10E06000C2F385572E4647FA03F0C007344604D55D
:10E0700013F80C0004F8010B26460133062BF2D1ED
:10E08000164CDFF864C0C2F303200023205C337019
:10E090008DF81800C2F305370DF1190647FA03F0A1
:10E0A000C007344604D513F80C0004F8010B2646CB
:10E0B0000133062BF2D100233370C2F3834406AB45
:10E0C000CDE90134084602F00F0305490095C2F37B
:10E0D000031243F0A9FA09B0F0BD00BF2C3A0608BC
:10E0E000D0390608343A0608243A060870B5094CB7
:10E0F000D4F8C824054662B10026D4F8C8042D21FE
:10E1000001363BF033FEAE42F7DBBDE870403EF037
:10E1100023B870BDA05D002030B583B04D1C0093C6
:10E1200003688572C2729C690023A04703B030BDAA
:10E1300003685B6C0BB102211847704770B51D4C2A
:10E140000968D4F8405B1C4ED4F83C4BD6ED577AA6
:10E15000DFED1A6A491B00EE901A0168F8EEE00A3A
:10E16000091B60EEA70A00EE101A20EEA07AB8EEA6
:10E17000C00A1C46A0EE007AB1EE400AF1EEC77A62
:10E1800067EEA67AFCEEE77AC2ED007A48F094FCDE
:10E190009FED0B7ADFED0B7AE0EE077AFDEEE77A82
:10E1A00017EE902A002ABCBF02F50C42A032226072
:10E1B00070BD00BFB82A0020980100202C7D8E3F42
:10E1C000A00CB34500A00C4638B50F4C94F8D314FE
:10E1D00001F03F018B1C024601F10A0584F8D1349D
:10E1E00084F8CE5404F2CC4084F8CF24083119F0DE
:10E1F000BFF8254485F8CA0494F8CE341C44000ABC
:10E2000084F8CB0438BD00BFA05D002038B50B4CAE
:10E2100000250122802120462EF0FCFF30B194F928
:10E2200004002FF029F808B1006838BD0135042D2D
:10E2300004F10C04EDD10020F7E700BF9462002048
:10E2400038B5041F00F1080554F8043FD81780EAD8
:10E25000430011F0A3FFA542F6D138BDF8B5C44C78
:10E26000DFEDC47AD4F8282594F89035B4F8927587
:10E2700007EE102A2DED028BB8EE478A28EE278A8A
:10E28000002B60D1D4F89C3594F8AD25002B40F3D9
:10E29000FC8007EE902A9FEDB86ADFEDB86AF8EED1
:10E2A000E77AB7EE007AA7EE867AF0EE477A07EEC5
:10E2B000103AF8EEC78AB7EE087A87EE270AC6EE5C
:10E2C000A87A20EE270A4CF0EFFD0F28B8BF0F20E8
:10E2D00094F8913585B2A4F89255002B00F03C815A
:10E2E000AF4234D0B4F894359FEDA56A94F82C650C
:10E2F00007EE103A07EE905AB8EE477AF8EE677AD2
:10E30000C6EE076A86EE277A76EE887A37EE087AC6
:10E31000C8EE276AC8EE077AB6B39A4B94F89625EA
:10E32000B4F89855C3ED047AC3ED087AC3ED0C7ABE
:10E33000C3ED106AC3ED147AC3ED187A002A49D0F0
:10E34000BDEC028BF8BD94F89135002B72D094F897
:10E350002C65002E40F0F880B4F89435DFED886A23
:10E3600007EE907A07EE103AB8EE676AB8EE477A91
:10E37000C6EE877A86EE867A77EE887A37EE087A66
:10E38000C8EE276AC8EE077A7E4B94F89665B4F813
:10E39000985500225A609A60DA605A619A61DA618F
:10E3A0005A629A62C3ED047AC3ED087AC3ED0C7A1F
:10E3B000C3ED106AC3ED147AC3ED187ADA625A63BA
:10E3C0009A63DA635A649A64DA645A659A65DA651C
:10E3D000002E65D1D4F89C3594F8AD25002B40F380
:10E3E000948007EE902A9FED646ADFED646AF8EE90
:10E3F000E77AB7EE007AA7EE867A07EE903AF8EE63
:10E40000E77AB7EE086A86EE070A86EEA77A20EE6C
:10E41000070A4CF049FD0F28B8BF0F2080B2A4F8BE
:10E420009805002E3BD0A8428AD0002874D1BDECBC
:10E43000028BF8BDD4F89C3594F8AE25002B40F340
:10E440008E8007EE903AF8EEE78A3D4607EE902A76
:10E450009FED496ADFED496AF8EEE77AB7EE007A98
:10E46000A7EE867AF0EE477AB7EE087A87EE270AAB
:10E47000C6EEA87A20EE270A4CF016FD0F28B8BF8A
:10E480000F2080B2A4F894052AE794F891350F255F
:10E49000A4F89255002B7FF423AF2846F2E70546F7
:10E4A00094F8AC3584F8E938002D3FF449AF07EE15
:10E4B000905A9FED336A344BF8EE677AD3ED006AD9
:10E4C00086EE277ABDEC028B00220121C3F80823D7
:10E4D00084F8E818C3F80C23C3F81023C3F81823F2
:10E4E000C3F81C23C3F8202337EE267AC3F8282369
:10E4F000C6EE877AC3F82C23C3F83023C3EDC57A60
:10E50000C3EDC97AC3EDCD7AF8BD0F20A4F8980504
:10E5100046B30F2D3FF414AF07EE900ADFED186AF3
:10E52000194BF8EE677ABDEC028B86EEA77AD3ED35
:10E53000006A37EE267AC6EE877AC3EDC57AC3ED58
:10E54000C97AC3EDCD7AF8BD94F89635B4F89855EC
:10E55000002B7FF4F5AE3DE794F8AE2576E73D4617
:10E560000F208FE794F8AC3584F8E93805469EE72C
:10E57000A05D0020BD378635CDCCCC3D002474494C
:10E580004E2DA63DCC620020506300201D4991F81D
:10E59000B824A2B3F0B400260546334630463746C9
:10E5A0001BB991F8B8442D2C23D02E2A19D0CA18A3
:10E5B00000EB800092F8B844A4F13002092A4FEA37
:10E5C00040009CBFA0F13002A0180E2B14D80133DC
:10E5D000CA1892F8B824002AE2D106B14042F0BC31
:10E5E00070470133002DF8D0CA182A4482F8B87455
:10E5F000DDE701231E46EBE70020F0BC704700205A
:10E60000704700BFA05D00202DE9F0410C4F0124B0
:10E61000A0231825E6B2FF2B0BDCC5F11B0103F18B
:10E620000108D7F83C09DBB23246C9B2FFF774FDE6
:10E630004346013DEFD10134052CEAD1BDE8F0811C
:10E64000A05D00201FB503AC8DF80C3000940023B2
:10E650008DF80D3008F030FA04B010BD10B5FBF79E
:10E6600081FE1121044634F093FE204639F0BCFAB5
:10E67000C82035F0F9FB2046BDE8104039F0BABAA1
:10E68000704700BF704700BF704700BF704700BFB2
:10E6900070B501F07F0505EB850400EBC40428216B
:10E6A00001FB05010126C4F830310023C4E94A22E8
:10E6B00084F81C5184F81D61C4F8343101F58E7161
:10E6C0001DB9F9F7C3FF002070BDFAF733F8002039
:10E6D00070BD00BF2549D1F840390F2B04D05A1C1A
:10E6E000C1F840290020704770B5214C94F820599A
:10E6F0000023C1F84039F5B9D4F80829D4F80C3909
:10E70000B2F5006F19D09A422CD01AD9C2F5006325
:10E71000402B18D9403B02F14005C1F84439012390
:10E7200084F82039C4F8085992B2402311490A44A8
:10E730008121FFF7ADFF002070BDC4F808598BB1EF
:10E740002A469B1AE4E74FF0000502EB0306C1F8E6
:10E7500044590CBF02210121C4F8086992B284F81F
:10E760002019E3E7002384F82039E4E7A05D0020C6
:10E77000C0190020E4220020ACE700BF70B51E4C99
:10E7800094F82039012B03D0022B0AD0002070BD51
:10E7900001461A48D0F8443953B984F8203900208A
:10E7A00070BD00231A468121FFF772FF0023F4E7B2
:10E7B000402BD4F8082910D9403B02F14005C0F89D
:10E7C0004439C4F8085992B240230D4C08462244FB
:10E7D0008121FFF75DFF002070BD4FF0000503EBC6
:10E7E0000206C0F8445908BF0220C4F8086992B272
:10E7F00008BF84F82009E8E7C0190020A05D0020C8
:10E80000E4220020012905D008B50321FAF7B6F962
:10E81000002008BDB2E700BF10B500230422044663
:10E82000194680F811211A46FFF732FF2046F9F702
:10E83000EFFE002010BD00BF10B5044629B990F8C6
:10E840001131032B0DD0002010BDD0F8E4359B69A9
:10E85000002BF8D090F81221032AF4D19847002019
:10E8600010BDD0F89013D0F87C33994214D9C078F9
:10E87000D4F880230128A1EB030104BFD218C4F807
:10E8800080238B4228BF0B46C4F890139BB22046CE
:10E890000021FAF707F8D6E7D0F8E4351B691BB179
:10E8A00090F81221032A03D02046FFF7B5FFCAE7EC
:10E8B0009847F9E738B5134602250A46C0E94E33B2
:10E8C00080F811510021FFF7E3FE002038BD00BFA2
:10E8D00010B50C7814F0600413D0202C0AD14B78BA
:10E8E000023B092B18D8DFE803F01B211717171775
:10E8F0001717272E22490122FFF7DCFF00242046AC
:10E9000010BD4B78062B24D00A2BF3D01D4B8A78F0
:10E91000C3F85029204610BDF9F78AFE0224EEE71D
:10E9200019490122FFF7C6FF0024E8E71749012231
:10E93000FFF7C0FF0024E2E74B88124A1B0AC2F827
:10E940004C390024DBE70F4B8A78C3F848290024B0
:10E95000D5E74B881B0A222B0CD0212B04D0214653
:10E960002246FFF7A7FFCAE7CA880949092A28BF34
:10E970000922F6E7CA880749362A28BF3622F0E777
:10E98000F0660020A05D0020EC660020E866002014
:10E9900042030020F8020020F8B50B7813F0600560
:10E9A0000C46064611D0202D16D1CD88D5B11B06B8
:10E9B0002AD52A461F496078F9F7BCFCE2881D4930
:10E9C0003046FFF777FF00250AE04B780A2B16D078
:10E9D0000B2B0ED0062B03D13046F9F729FE02256A
:10E9E0002846F8BD022260781144F9F7A3FC2846B6
:10E9F000F8BD8B78DBB9104BC3F85459F0E70F49D9
:10EA00000122FFF757FFEBE70D4B4A780D4FC3F894
:10EA1000D42003230021C0E9E45580F8113107F127
:10EA200044022B463D640D46F9F73CFFD8E7F9F761
:10EA3000FFFDD5E7FC2A0020A05D0020F466002041
:10EA400098010020B82A00200B7803F00303012B63
:10EA500003D0022B04D0002070478B881BB937E706
:10EA60008B88832BFBD097E7F0B5012190F8D17507
:10EA700090F8D36590F8CFC590F8CE5590F8D03582
:10EA800090F8D22580F8111190F8CC1585B005EBDF
:10EA90000C2503EB072302EB062201F01F06AFB2A1
:10EAA00092B290F8CD558DF808109BB2012E044615
:10EAB000ADF80A70ADF80C30ADF80E20C0F840216A
:10EAC0008DF8095017D0022E1FD036B101F0800109
:10EAD000F9F744FD002005B0F0BD092D0FD8DFE89F
:10EAE00015F0BF00AC000E00D5000E00EA00850056
:10EAF0000E007700540090F81221032A2FD02046F0
:10EB0000F9F796FD002005B0F0BD01F06001202965
:10EB1000DAB234D0012D00F02081032D00F00681FF
:10EB2000002DD7D190F81211022900F0DF800329BF
:10EB3000E5D11B0600F14B8102EB820200EBC20320
:10EB400093F87633002B00F04D81BF4B0122C3F8C0
:10EB50006829BE4920460222FFF7ACFEBAE7DAB2C6
:10EB6000012ACCD8D0F8E43502A99B689847BDF8B3
:10EB70000E30002BAED12046FFF74EFEAAE7D0F8AC
:10EB8000E43502A99B689847A4E7F9B2AE4D012984
:10EB900085F85819B3D890F81231022B00F027816C
:10EBA000032BACD1002900F0868190F810110129C7
:10EBB000E1D0D0F8E4355B68984795F8581984F8A7
:10EBC00010112046F9F79CFC2046FFF725FE81E74F
:10EBD000012A94D190F81231022B00F01781032BF7
:10EBE0008DD100F58871FFF765FE73E73D0A022DB0
:10EBF000ADF8062000F05081032D00F00B81012DAF
:10EC00007FF47DAFD0F8EC3580781B680DF10601FC
:10EC10009847BDF80620002A3FF45CAFBDF80E30DF
:10EC2000002B3FF457AF9A4228BF1A4601462046B0
:10EC3000ADF80620FFF73EFE4CE790F81231023B9C
:10EC4000012B3FF65CAF012F7FF444AFD0F8E435E1
:10EC500000229B68C0F8182102A9204698478AE73D
:10EC600090F81231023B012B3FF649AF764BD0F8BA
:10EC700018210021C3F8601912B10222C3F86029DB
:10EC8000734920460222FFF715FE23E7012F00F00B
:10EC90009880022F7FF41EAF13F0FF0F7FF41AAF9E
:10ECA00002691B0A023B5268032B00F21D81DFE858
:10ECB00003F0393531241A437FF421AF90F8123133
:10ECC000032B3FF41CAF036907F07F0580F8145154
:10ECD000196867F30A120A431A60FFF79DFD002DB9
:10ECE00000F0E580022384F81231F3E651063FF488
:10ECF000F1AE1146F9F732FCECE6052363F3061298
:10ED0000514B012184F816112046C3F86429FFF7FE
:10ED100083FDDFE6042363F30612F1E7032363F3C5
:10ED20000612EDE7022363F30612E9E790F81231C9
:10ED3000022BDBD0032B7FF4E2AE27B9550602D0BD
:10ED40001146F9F70BFCD4F8E43502A99B6820467C
:10ED500098472046FFF760FDBCE690F812110229A3
:10ED6000C4D003297FF4CBAE002F7FF4B3AE12F0F2
:10ED70007F013FF400AF180600F1A78002EB820389
:10ED800004EBC30304EB810083F8767383F87413F8
:10ED900083F87573282303FB0243416D03F55D730C
:10EDA000DA780B68023A6FF35553012AD4F8E42558
:10EDB00098BF43F080530B602046936802A99847A0
:10EDC000D9E6D0F8E435C0F818719B6844E702F042
:10EDD0007F0202EB820200EBC20393F81E31002B8C
:10EDE0007FF4B3AE184B0022C3F86829B1E60029BE
:10EDF0003FF4C1AE0121032380F8101180F81231D5
:10EE0000F9F77EFB2046FFF707FD63E61149FFF7A0
:10EE100051FD5FE6FDB2052D3FF671AEDFE805F06E
:10EE2000342C241C0B03D0F8EC3580789B690DF151
:10EE300006019847EDE6D0F8EC3580785B690DF176
:10EE400006019847E5E600BFA05D002008670020A6
:10EE500000670020FC660020D0F8EC3580781B6944
:10EE60000DF106019847D4E6D0F8EC358078DB68E0
:10EE70000DF106019847CCE6D0F8EC3580789B6818
:10EE80000DF106019847C4E6D0F8EC3580785B6850
:10EE90000DF106019847BCE6D0F8E43580789B6A0E
:10EEA0000DF1060198474570C4F8F005B1E601235D
:10EEB00084F812310EE60222D0F8E43580F8101101
:10EEC00080F812215B68984755E6282202FB01432F
:10EED00004EB810083F81E7183F81C1183F81D5127
:10EEE000816903F58E735BE7012363F3061207E77D
:10EEF00070B5044649B990F81131022B1BD094F833
:10EF00001631012B0DD0002070BDD0F8E4355B69BF
:10EF1000002BF8D090F81221032AF4D19847002052
:10EF200070BD2A4A2369D2F864295A60002384F804
:10EF30001631002070BDD0F83831D0F82451AB42E2
:10EF400017D9C278012AD0F82821A3EB050308BFFE
:10EF50005219C0F8383108BFC0F828219BB20021EF
:10EF6000FFF796FB00231A4619462046F9F79AFC4C
:10EF7000C5E7D0F83C31B3FBF5F605FB163666B9AC
:10EF80009D420AD8D0F84021934206D233463246F9
:10EF9000FFF77EFBC4F84061E4E7D4F8E435DB68B2
:10EFA0001BB194F81221032A0CD00023052284F807
:10EFB000112119461A462046F9F774FC2046F9F744
:10EFC00027FB9CE720469847EFE700BFA05D0020A5
:10EFD000214A038890429BB212D002F5806290428F
:10EFE0000ED0B0F1804F0BD0A2F58032904207D006
:10EFF00002F58062904203D002F58062904203D114
:10F000004A8823F070031343144A904218D002F543
:10F010008062904214D030B423F440730C894D6860
:10F0200002F56C429BB2234390420C880380C56278
:10F0300004850DD18B7A0386012330BC838270470F
:10F0400003800B884A68C26203850123838270476C
:10F05000034B9842EED0EFE7000001400010004063
:10F060000004014082B0064B002201920193019BF3
:10F0700003EB80000190019B186802B0704700BF4D
:10F080005028004082B0064B002201920193019B60
:10F0900003EB80000190019B196002B0704700BF34
:10F0A000502800400023C0E90033C0E90233C0E922
:10F0B0000433C0E90633C0E90833C0E90A33C0E9C4
:10F0C0000C338363704700BF0B6870B4D1E905242B
:10F0D000CD682B431343D1E9072523431343D1E9DB
:10F0E00009422B43D1E90D652343134304680B4ABE
:10F0F000334322402B4313430360D1E90B3442696D
:10F100000D6922F0070223431343D1E90142436111
:10F110004560846070BCC260704700BF3F801CF0D7
:10F1200002683649002310B422F0010221248842EB
:10F130000260036043608360C3600361446138D050
:10F140002F4B98422ED02F4B98423CD02E4B9842BA
:10F1500040D02E4B984232D02D4B984241D02D4B6F
:10F16000984246D02C4B984217D02C4B98423CD01A
:10F170002B4B984216D02B4B984224D02A4B9842C6
:10F1800028D02A4B98421AD0294B984229D0294B93
:10F1900098422ED0284B984208D14FF03D5243F868
:10F1A000AC2C03E04FF4746243F8202C5DF8044B60
:10F1B0007047224B5DF8044B3D229A607047204A0D
:10F1C00043F8642CF2E74FF474125DF8044B43F8F3
:10F1D000382C70474FF074625DF8044B43F8502CA4
:10F1E0007047184A43F87C2CE0E73D2243F8082C8E
:10F1F000DCE7154A43F8942CD8E700BF10600240C2
:10F200002860024040600240586002407060024046
:10F2100088600240A0600240B86002401064024072
:10F220002864024040640240586402407064024016
:10F2300088640240A0640240B8640240006002405A
:10F240003D000020400F002000003D202DE9F04F40
:10F25000DFF8ACA32DED028B9AF88019002297B04D
:10F26000CAF87029CAF87429CAF87829CAF87C291A
:10F27000CAF86C2919B19AF881298AF86C299AF888
:10F2800082291AB19AF883298AF87B299AF8862963
:10F290001AB19AF887298AF876299AF884291AB136
:10F2A0009AF885298AF871299AF8883905935A1E9F
:10F2B000D3B257B203937B1C00F0AA80C54AC64E56
:10F2C00052F83790029602EBC7020023127901939D
:10F2D00008EE102A1D4634469846267839463046B0
:10F2E0003AF06CFE83463046BBF1000F1ED038F07A
:10F2F00097F9EA1D1321D2B220B14FF0000E8271AE
:10F3000080F807E034F044F820783AF081FE4FF0BE
:10F31000070308F1010223714FF0010384F8028012
:10F320006070CDF804B05FFA82F8E3700135042D07
:10F3300004F10504D1D118EE100A029ECDF8108018
:10F34000FAF7F2FFA549A64A4868024042F4403263
:10F350004A600FB9019B5BB9A24C4820FAF7E4FF61
:10F36000204602214AF006FDA26842F00102A26096
:10F370009A489C4A4168BAF88A4941F400014160C0
:10F38000516821F480515160916B21F4401141F496
:10F3900080119163D16841F46001D160956B85F46F
:10F3A0004011C1F3015101EB81011F2000FA01FC62
:10F3B00025EA0C0C112505FA01F141EA0C019163D3
:10F3C000D16841F0E061D160956BC5F30151C1F1A5
:10F3D0000401C9B201EB810188404FF0120C25EA0B
:10F3E00000000CFA01F108439063E4B1BAF88C19FB
:10F3F000CAF89449A1B1BAF88E29CAF8981962B12D
:10F40000019B7948521A90FBF2F2CAF89C296BB919
:10F4100017B0BDEC028BBDE8F08F744A1288EFE79D
:10F42000734A1188E7E7734A1488DFE7484604996E
:10F430004AF0A0FC684B012003F114080723F2787E
:10F44000441CE4B252B375783279A5F10A0101EB9C
:10F45000410105EB450C092D03FA01FE03FA0CFBF3
:10F4600002FA01F140F2A080D9F80C2022EA0E0E37
:10F4700041EA0E01C9F80C10421E02EB82021F2164
:10F48000062801FA02FC05FA02F273D8D9F8341002
:10F4900021EA0C010A432046C9F834200536B0455C
:10F4A000CDD1D9F80820039942F40072C9F8082098
:10F4B000D9F8082042F48072C9F80820D9F8082049
:10F4C000574442F00102C9F8082097F99029022018
:10F4D00035F030F8044600289AD04668304635F0BA
:10F4E00017F8454A431E242101FB032393F8D85102
:10F4F000002D8DD1059983F8D911062283F8D821E2
:10F50000002885D0304635F003F848F039F86068B7
:10F51000FFF706FE07A8FFF7C5FD049EA26837485F
:10F520000792012E8CBF4FF4806300230D9309F1E5
:10F530004C034FF48072CDE90A56089309904FF4BA
:10F54000003360680C9507A94FF400674FF400562C
:10F55000CDE91023CDE90E76FFF7B6FD626813689A
:10F5600043F001031360D9F8083043F08043C9F831
:10F5700008304DE7C11FA0F10D0201EB81014FF0F2
:10F580001F0E02EB82020C280EFA01FC0EFA02F0AA
:10F5900005FA01F113D8D9F8302022EA0C02114300
:10F5A0002046C9F8301079E7D9F8101002FA0CF2A9
:10F5B00021EA0B0B42EA0B02C9F810205CE7D9F8EC
:10F5C0002C1005FA02F221EA00010A432046C9F88C
:10F5D0002C2063E764C605080C6700200023014067
:10F5E000E030FCFF00200140803801002E7AFF1F30
:10F5F0002C7AFF1F2A7AFF1F980100204067002005
:10F60000A05D002000B583B009238DF80730F9F71D
:10F61000D3FA8DF807009DF80730012BF7D09DF83D
:10F62000070003B05DF804FB024A536A23EA0000B6
:10F630005062704700380240024A136A23EA000011
:10F640001062704700380240484B98422ED0B0F10B
:10F65000804F32D0464B984236D0464B98421ED00F
:10F66000454B984237D0454B98423BD0444B98424B
:10F670003FD0444B98424BD0434B984240D0434BF1
:10F6800098424CD0424B984251D0424B984256D06F
:10F69000414B98425AD0414B98425ED07047404A05
:10F6A000136A43F0040313620420C5E73C4A536A1B
:10F6B00043F0010353620120B6E7394A136A43F06D
:10F6C000010313620120B7E7354A136A43F00203CE
:10F6D00013620220B0E7324A136A43F00803136250
:10F6E0000820A9E72E4A136A43F010031362102082
:10F6F000A2E72B4A136A43F02003136220209BE702
:10F70000274A536A43F4803353624FF480308BE7C7
:10F71000234A536A43F002035362022084E7204ADB
:10F72000536A43F4003353624FF400307CE71C4AC1
:10F73000536A43F4802353624FF4802074E7184ADD
:10F74000136A43F040031362402075E7144A136ABA
:10F7500043F08003136280206EE7114A136A43F47A
:10F76000807313624FF4807066E700BF00000140B1
:10F770000004004000080040000C00400010004061
:10F7800000140040000401400040014000440140DA
:10F790000048014000180040001C004000200040CC
:10F7A0000038024010B504460068FFF74DFF0D4BCE
:10F7B000D3F8802A204652084FF6FF7133F098F8AC
:10F7C00020460021FCF7ACFE0749084A41F210230D
:10F7D0002046CA5001F59051BDE81040002210317A
:10F7E00032F05ABFB82A0020A05D002091AD010878
:10F7F00038B5124BD3F8804A054600686408FFF715
:10F8000023FFB4FBF1F3B3F5803F03D3012CFAD906
:10F810006408F6E7224699B2284633F069F80849A9
:10F82000084A41F20C232846CA5001F59051BDE820
:10F83000384000220C3132F02FBF00BFB82A002020
:10F84000A05D00201DE501082DE9F04FCCB200219C
:10F8500085B007460846164638F0DAF9002101203F
:10F8600038F0D6F937F0BAFE022E09D0042E44F64D
:10F87000C01818BF4FF49648072C06D900200BE09B
:10F88000FF2C4FF41648F7D10326C74D95F81C31CD
:10F890002BB90020C5F8200105B0BDE8F08F032E7C
:10F8A0000FD0C2490C44002294F85B07032133F0C7
:10F8B00091FB0028EDD0BE4BC3F8EC09C3799A0741
:10F8C000E7D4BB4C95F81C0141F207230022E65413
:10F8D000032133F07FFBC4F8F00D0028D9D04FF49A
:10F8E0008062B44BC4F8A839C4F8B4290323C4F81F
:10F8F000B82941F2F812A4F8AC390023A35441F21C
:10F90000F4124FF0010A24F802A004F5905204F515
:10F910001F61136041F20422C4F8BC19A35241F2E2
:10F92000062204F6F451032EA354C4F8B089C4F897
:10F93000D439C4F8C839C4F8C439C4F8C019C4F8F3
:10F94000D039C4F8CC3904F6A8190ED0D4F8ECB9E3
:10F950009BF8040037F064FEC4F8E80958460EF03E
:10F9600083FD514648460EF093FD322034F07CFA78
:10F97000012E09D1D4F8F00D4146FFF739FFD4F834
:10F98000EC09FFF70FFF0AE0022E3CD1D4F8EC0996
:10F990000EF059FDD4F8F00D4146FFF729FFC5F8E8
:10F9A00020914FF0060A022E12D0D5F8200134F033
:10F9B00073FE68B10121002038F02AF9D5F8200142
:10F9C00034F06AFE0146002840F0878038F020F9C4
:10F9D000384634F061FE80B10121084638F018F94C
:10F9E0004FF0050B4FF00008384634F055FE014645
:10F9F00000287BD1012038F00BF9042ED5D005204A
:10FA000034F032FACFE7032E5FD141F208234FF0F2
:10FA1000000A04F803A051466748DFF890B140227D
:10FA20004CF047FD8DF80FA0DFF894A19DF80F3042
:10FA3000072B09D9614801210EF02AFDD4F8F00DF9
:10FA40004146FFF7D5FEAAE79DF80F3003EB4303CD
:10FA50000BEBC30393F8DD3783B39DF80F3003EB53
:10FA600043030BEBC303D3F8E0373BB39DF80F30F0
:10FA70005B4493F85B0708B30022032133F0AAFA32
:10FA80000190D8B10EF0DFFC9DF80F309AF800100D
:10FA9000019A03EB43030BEBC30305EBC100D3F85F
:10FAA000E037C0F82431D379DB0748BF012301F1E7
:10FAB000010148BF80F828318AF800109DF80F3006
:10FAC0000133DBB28DF80F30B0E7042E7FF467AF5F
:10FAD000D4F8EC090EF0B7FC4CE7D5F8200134F06F
:10FAE000D3FD0146384634F0DBFD67E7384634F095
:10FAF000CBFD95F8723101468BB9242803D14FF024
:10FB0000010385F87231012E04D13846019134F099
:10FB1000C7FD0199D5F8200134F0C2FD64E7012B3F
:10FB200006D14D280CBF0223002385F87231EAE785
:10FB3000022B06D13C280CBF0323002385F8723129
:10FB4000E1E7032B10D10A2802D985F87281DAE7A0
:10FB5000042385F8650185F8648185F8678185F857
:10FB6000660185F87231CEE7042B09D195F866312C
:10FB700085F87301434085F8663185F872B1C2E7B4
:10FB8000052BC0D195F8643195F8659195F866011B
:10FB90004B4517D25A1C2B44484085F8660185F81E
:10FBA000642183F86811AEE7986E0020B82A00201F
:10FBB000A05D00206CC60508BC6F002048670020CF
:10FBC000A86F00208842C0D195F8733185F872A1E2
:10FBD000F42B98D1B9F1000F95D12421384685F83E
:10FBE000729134F05DFD4D21384634F059FD3E21CF
:10FBF000384634F055FD4946384634F051FDF4217D
:10FC0000384634F04DFDF421384634F049FD032EDA
:10FC10001BD0D4F8EC09437901689D080223AB405E
:10FC2000DB439BB20B828D892B408B810079202195
:10FC30000EF0F8FBD4F8EC094A46494632F02CFDA8
:10FC4000D4F8EC391868FFF7FFFC0022D4F8F00D67
:10FC5000114632F021FDD4F8F03D1868FFF7F4FCAE
:10FC6000012019E6224A936803F00C03042B10B418
:10FC700021D0082B22D01F4B03601D4C1E4AA168C7
:10FC8000C1F30311114491F8FC13CB404360A16808
:10FC9000C1F38221114491F8FC1323FA01F1816030
:10FCA000A1685DF8044BC1F342310A4492F8FC2389
:10FCB000D340C3607047114B0360DEE7546851685E
:10FCC00052686302C2F388124CBF0C4B094B01F01F
:10FCD0003F01B3FBF1F303FB02F3054A5268C2F3A1
:10FCE000014201325200B3FBF2F30360C5E700BFEB
:10FCF000003802400024F4009801002000127A002D
:10FD00002DE9F04FB34CD4F8E4345A69D2078BB0E4
:10FD100002D50BB0BDE8F08F5A699B6912EA030A5D
:10FD2000F7D0CAF307431AF4002F009340F0028182
:10FD3000009B5D0743D41AF0020F5FFA8AF503D0E7
:10FD4000D4F8E43402225A61BAF1000FC0F21182F1
:10FD50001AF4006FCAF3072740F084812E0708D5F4
:10FD60009D4B9E48D3F818349847D4F8E4340822C1
:10FD70005A61ED0600F1E981F80600F1A981B906A2
:10FD800000F12E81009BDA0609D5934B9348D3F8F6
:10FD900028349847D4F8E4344FF480125A61009B19
:10FDA0009B06B6D58C4B8D48D3F82C349847D4F8A5
:10FDB000E4344FF400125A610BB0BDE8F08FD4F870
:10FDC000E8249369D26913401FFA83FBBBF1000F4B
:10FDD000B1D0DFF80882CDF80CA045464FF00009FD
:10FDE00009E05FEA5B0B09F1010908F1040805F17C
:10FDF000280500F0DA811BF0010FF2D0D4F8E814E6
:10FE00005FFA89F708694A6B04EB8703FA40D3F875
:10FE1000F034D2019B68D2B202431A40D007D3B269
:10FE200016D54B6BD8F81820012000FA09F023EA08
:10FE300000034B63684B6948D3F81034012191608B
:10FE40003946984794F8DB64012E00F0FC810123C9
:10FE50001A0703D5D8F8182008239360DE0603D5C7
:10FE6000D8F8182010239360580603D5D8F8182026
:10FE700040239360990703D5D8F818200223936094
:10FE80001A06AED5D5E94C60D5F82431D8F818C09B
:10FE9000311A8B42DCF8182028BF0B46033392B28C
:10FEA000B2EB930F9DD9D4F8E824323704EB8703E3
:10FEB000CDE9019890469946B04238D2BEB3D5F804
:10FEC000241194F8DB34D5F82821371AB94228BF19
:10FED000394601F1030E4FEA9E0E83B98FB2033704
:10FEE000BF10D9F8E0A40AD0013352F8040BCAF8C5
:10FEF00000009F42F8D1D5E94C60D5F82821DCF804
:10FF0000183008440A44B042C5F82821C5F8340125
:10FF10000AD195F81C11D8F83420012707FA01F10D
:10FF200022EA0102C8F834209BB29E45C4D3DDE921
:10FF3000019856E7D4F8E8349D69DB691D402D0C23
:10FF40003FF4F6AE04F59B66DFF88CB0B046B146E0
:10FF5000002708E06D0807F1010706F1040608F123
:10FF600028083FF4E5AEEB07F4D5F9B204EB8102C3
:10FF7000D4F8E834D2F82C2592685B691A40D0078F
:10FF8000D3B218D594F8DB04726D012398429360C4
:10FF900007D11269D8F87C33C2F312029B1AC8F851
:10FFA0008C33DBF80C344846984794F8DB34012B4B
:10FFB00000F0578101239A0702D5726D02239360E6
:10FFC0001B07C7D5DBF8143448469847736D0822E1
:10FFD0009A60BFE7A84C00209801002080510020C3
:10FFE000D4F8E834D4F8F0149A680868C2F34102EF
:10FFF000022A08BF03224FF0000514BF65F30A0070
:020000040801F1
:1000000062F30A0008605A6842F480725A6006A8D7
:10001000FFF728FED4F8E424D4F8E804D368BF49F5
:10002000079D6FF38D23D3608068C0F341000144C6
:1000300091F84811032900F0CF80B949B948012649
:10004000294484F8DA6481424FF04006A4F8DC6465
:1000500000F215810E2161F38D234FF40051D3601E
:1000600051618FE6B04B94F8EA25D3F82034AF48BD
:1000700000218DF817108DF817209847D4F8E81450
:10008000D4F8E42494F8E23488684FF400615161B4
:10009000002B3FF463AEC3077FF560AE94F8ED35F7
:1000A000012B7FF45BAE9DF81730032B7FF456AE27
:1000B000D4F8E4359E491A6842F001021A601A68C1
:1000C00042F003021A600B6943F006030B6145E638
:1000D000D4F8E824954853684FF0000823F0010352
:1000E00041465360F8F74AFD94F8D964414656B149
:1000F000904BFF2203EB860653F8045FD86BAA608F
:100100009E428260F8D1D4F8E83488484FF0FF323C
:100110009A614FF00112DA610B2262F3070162F378
:100120000708C3F8148019611A686FF30A121A607D
:10013000F8F76EFAD4F8E4247B4B7C48D3F81C34EF
:100140004FF480515161984719E6D4F8E4349A6924
:1001500022F010029A611A6AC2F34340022802F0A8
:100160000F0144D0062823D09A6942F010029A6108
:1001700002E694F8E2343BB1D4F8E425136823F0A6
:10018000030161F307031360D4F8E8246649536858
:10019000D1F82414654823F0010353608847D4F84C
:1001A000E4344FF000425A61D2E5DDF80CA0C2E51C
:1001B00001EB8101D4F8A85504EBC1012E68D1F8F8
:1001C0006408C4F8A46AC2F30A1202442868C4F896
:1001D000A80AC1F86428C7E700214FF4007084F82A
:1001E000DA140921A4F8DC0461F38D2335E747F61E
:1001F000F0701042B8D001EB8100C2F30A1204EB98
:10020000C00002F1030C5FEAAC0CD0F85858D4F8E7
:10021000A8E54FEA810818BF002006D00130DEF8BB
:10022000006045F8046B8445F8D1414404EBC101FA
:10023000D1F85858D1F8640815440244C1F8585808
:10024000C1F8642890E7B9F1000F7FF400AE94F88C
:10025000E935042B7FF4FBAD3448F8F7D9F9334680
:10026000F6E5002F7FF4A6AE94F8E925052A7FF481
:10027000A1AE48460193F8F7CBF9019B9BE62E48C7
:10028000A5F57401A1F51051814203D80D2161F348
:100290008D23E2E629492A482944814203D20C21D0
:1002A00061F38D23D9E62748A5F18C71A1F543416F
:1002B000814203D80B2161F38D23CEE622492348E6
:1002C0002944814203D20A2161F38D23C5E62049E6
:1002D00020482944814203D2092161F38D23BCE6E1
:1002E0001D48A5F1B771A1F55851814203D20821EB
:1002F00061F38D23B1E6194919482944814203D29B
:10030000072161F38D23A8E6164917482944814245
:1003100034BF0621052161F38D239EE654C50508EF
:10032000401E1BFF3F420F0098010020805100201B
:1003300000ED00E094510020DFC810002013FBFE08
:1003400020D61300FF69180000D3CEFE40771B00B3
:10035000C05BB3FEC091210040AC2700C01D6AFE07
:1003600040E13300803C36FEE09C41000D4B93F8A9
:10037000CC2A12F0010F0C4A03D0012382F8743109
:10038000704792F8742162B9D3F8182B4AB193F8E8
:10039000882A104493F8892A83F8880A114483F83C
:1003A000891A7047B82A0020986E002010B50E4CAC
:1003B00040F0080284F83C2494F9DA20022A06DD91
:1003C000420704D583071CBF012384F8E2300521CE
:1003D0000648F8F70DFD062184F83D04BDE81040FD
:1003E0000248F8F7EDBC00BF98010020D0050020BE
:1003F00010B5F8F795FCA8B31B4C94F9DA30012B33
:1004000030DD59B3022B2DD094F8E2309BB971B195
:1004100080230521154884F84234F8F7E9FC0621C9
:1004200084F84304BDE810401048F8F7C9BCBDE8A3
:1004300010400420BAE7002914BF0020042094F8DB
:10044000DD301A0748BF40F002005B0701D411B14C
:1004500008B940F00100BDE81040A7E7022BD3D156
:100460000420ECE710BD00BF98010020D605002055
:10047000F8B5224C04F24447030A84F849040546BF
:100480000621384684F84834F8F7B2FC94F8DD3099
:1004900084F84A04DB072AD4B4F8DE20AA4226D125
:1004A000174DD4F84434C5F87531C3B285F87B31A3
:1004B00041F26F714FF6FF738A4218BF0123134454
:1004C00005F27516C3F307220621304685F8792117
:1004D00085F87A31F8F78CFC072185F87B013046E6
:1004E000F8F76EFC052104F24B40F8F769FCBDE813
:1004F000F84004480721F8F763BC00BF98010020CA
:10050000986E0020DC05002008B5F8F709FC48B11A
:10051000A1F59C53083BB3F57A7F03D2BDE80840B0
:100520000846A5E708BD2DE9F047C44DD5F8843A43
:10053000002B3BD0C24EC34C06F1DA07D5F8840A33
:1005400034F0AAF8A0BBB5F8B22A092A0CD9B5F83C
:10055000B41A64234B43B3FBF2F3452B40F3AC8155
:10056000A5F8B20AA5F8B40A94F8B531012B00F049
:10057000D181022B00F0EC8133B9B3480521F8F7A3
:100580001FFC012384F8B53195F8C03A2E6B002B7F
:1005900000F0E881D5F8C43AF31A782B40F2E281F2
:1005A000D5F8C80AF8F7F6FFC4F8B861BDE8F087D7
:1005B000D5F8840A34F068F894F87C318046052B2D
:1005C000BCD8DFE803F00309181E3947AA28B5D1C3
:1005D000012384F87C31B1E7552803D1022384F844
:1005E0007C31ABE7B5F8B63A0133A5F8B63A00234B
:1005F00084F87C31A2E7032384F87D0184F87C3100
:100600009CE7132884F87E01C4F8980108DDB5F84A
:10061000B83A0133A5F8B83A002384F87C318DE765
:1006200018B9052384F87C3188E70023C4F89C318D
:10063000042384F87C3181E7D4F89C31E21801333B
:1006400082F87F01D4F89821C4F89C3193427FF45A
:1006500075AFE6E7D4F898317C4803F1020A4FFA07
:100660008AF1F8F7C5FB804594F87D9140F01A8136
:1006700026201FF0A9F858B1002385F8C03AB5F834
:10068000B43A0133A5F8B43A002384F87C3155E735
:1006900095F8C03A4B451AD1002385F8C03A09F1C4
:1006A000FF33102B00F2F880DFE813F01F007F000B
:1006B0007F00E0007F00F600F600F6001F00F60065
:1006C000F600F600F600F600F600F6001F00B9F19D
:1006D000090F02D0B9F1110F01D1012BDCD0B5F80F
:1006E000BC3A0133A5F8BC3AD9E7BAF1060F5CDD94
:1006F000B9F1010F06D0B9F1090F0CBF4FF0020993
:100700004FF0030994F8820194F8831194F8812141
:1007100094F97FE194F981C194F8803186F8DA90F8
:1007200041EA002109B2900786F8DBE086F8DDC0D7
:10073000A6F8DE1006D512F00C0F14BF012200221D
:1007400086F8E220B9F1030F13D1BAF1090F2CDDBD
:1007500094F98521082AA8BF082222EAE27286F8C5
:100760001021002043B29A4200F101005EDC94F8AF
:100770008431D5F8A8A0002002469BB2524590468D
:100780006ADB95F8C83686F8DC00232B0DD109EB1F
:10079000890303EB83030CEB8303A5F8CC36A5F8A0
:1007A000CEE6A5F8D016A5F8D206294929480A228E
:1007B0004BF057FE10B1002384F8AA31244B3A685D
:1007C0001A607A685A603A891A8194F8AA3143BB50
:1007D00096F8E23095F8882A84F8AC21002B14BFF3
:1007E0000223012384F8AA3196F8DD3095F88A0AAD
:1007F00084F8B00113F001031CBFB2FA82F35B0965
:1008000095F8892A84F8AD21D9B2B5F88C2A84F8F4
:10081000AB11A4F8AE2113B10AB1A4F8B22184F847
:10082000B4110EF015FA0EF013FA28E705EB4308A1
:10083000234493F88731A8F81E3B93E7B82A002099
:1008400098010020986E0020E3050020157000201C
:10085000387000207202002005EB48080132B8F819
:10086000AC8052B2984508BF104687E7BAF1040F32
:100870009BDD94F87F2194F8803143EA02235904E8
:100880001AB204D5C3F30D03A6F8E0308DE7002AB1
:10089000F8DBA6F8DE3088E7B5F8BE3A0133A5F8F4
:1008A000BE3AECE619F0010F7FF4EEAEB5F8BA3AB5
:1008B0000133A5F8BA3AE7E63A4BD3F85024B3F837
:1008C0005414012A1DD141F25632914203D14FF006
:1008D000FF32C3F85024D3F85024D5F8840A02EB31
:1008E000820202EB820201EB420189B2A3F85414A6
:1008F00003681B6998470023A5F8B23AA5F8B43AF3
:1009000032E60132E7D1B1F5965F04BF0122C3F8A8
:100910005024E0E7234E96F9DA70002F3FF434AE0E
:10092000022F11D14FF48040FFF7A2FD84F8B5717A
:1009300096F9DA30012B7FF727AE96F8DD30C3F356
:10094000400386F8E2301FE6032384F8B531EFE771
:10095000144BB3F8E030002B3FF416AE032384F8B9
:10096000B53111E695F8C02095F8C1309A4204D00F
:10097000F8F742FEC4F8B86118E6D4F8B831F31AB3
:10098000B3F57A7FBFF412AED5F8C43AF61A952EB5
:100990007FF60CAE04480521F8F712FABDE8F047DF
:1009A000F8F72ABE98010020E305002010B5134C8B
:1009B000D4F8180B00B394F8881A59B194F8892A1E
:1009C0000DF07EFAB4F88C3A83421ABFA4F88C0A70
:1009D00001210021B4F88E2A62B141F2883393429A
:1009E000B8BF13469A4205D0A4F88E3ABDE810402D
:1009F0003DF078B80029F9D110BD00BFB82A002019
:100A000010B401440446002014F8013B0822584069
:100A1000430010F0800F08BF400083F0070314BFAD
:100A2000D8B2C0B2013AF3D18C42EDD15DF8044B9B
:100A3000704700BF10B54FF4806084B02CF0FEFB0F
:100A400050B3164B90F9040093F8BC31144A002BB4
:100A500018BF08234FF4E1310124CDE9014300918F
:100A600000234FF480612CF046FC0E4BFF22C3F8AC
:100A70004802003818BF012083F8D42683F8E42602
:100A800083F8F42683F8042783F8142783F82427AF
:100A900083F8342783F8442704B010BD986E0020F3
:100AA00099900008B82A00202DE9F04F384CD4F86E
:100AB000C03B13F0006383B05CD094F8FCC0604589
:100AC0005CD3FF2856D1334B93F8EA30002B4DD03E
:100AD000DFF8C8B00022CBE97022CBF8C821BCF106
:100AE000000F52D004F2D46E0EEB0C139A4610464F
:100AF0001546114616461746CDF804C07346B3F89E
:100B000002E0B3F80CC093F8009093F901807144AF
:100B100062444F45D3E901EC38BF4F461033464598
:100B2000B8BF46469A4509B212B275446044E6D150
:100B3000CBE971508BF8C0718BF8C161DDF804C04E
:100B400091FBFCF192FBFCF294F8C836ABF8CC2197
:100B5000092B104A08BF9BF8C031ABF8C2114FF007
:100B6000000182F8EA1008BFA4F8D2360A4803B0A0
:100B7000BDE8F08F002003B0BDE8F08F04F2D4642C
:100B800004EB001003B0BDE8F08F62466146DBE77E
:100B9000B82A00209801002058700020986E00208C
:100BA0002DE9F8434B4C427894F8D03102F00F0510
:100BB000CBB9F5B92B46002184F8D411EB1AD9B280
:100BC0000E290CD844490B4493F8641B39B102F048
:100BD000F002802A4AD0902A5FD0A02A0DD00027A8
:100BE0003846BDE8F8830021AB4284F8D411F6D82A
:100BF000E4E784F8D0512B46DDE7412966D081F047
:100C00008003042B62D90846F8F760FA031D0246F8
:100C1000DBB2324884F8D43165F05F0584F8D551F1
:100C2000F9F7BCF994F8D471002FD8D0BE1E16F095
:100C3000FF0024D1FF25A946022756B1DFF8A08086
:100C4000464418F8011BD4F8F80133F029FD464555
:100C5000F7D1D4F8F801494633F022FDD4F8F80171
:100C6000294633F01DFD3846BDE8F88365F07F0561
:100C70000427022684F8D55184F8D4713046184AE6
:100C80004FF6FF71104412F8015B491B904289B284
:100C9000F9D15FFA81F90D0ACFE7412914D081F02B
:100CA0008003042B10D90846F8F710FA65F06F0599
:100CB0000627042684F8D70184F8D55184F8D61184
:100CC00084F8D4713046DAE70420EFE708230422E1
:100CD0009FE700BF986E0020B82A00206E700020A9
:100CE0006C7000202DE9F04782B0054602AF18462F
:100CF0001C460E46904649F057F9083020F0070090
:100D0000ADEB000D0DF1080A013CD14614F8013F8E
:100D10005BB989F800304246CDF800A0314628463C
:100D200038F0B4FCBD46BDE8F08718463CF0D0FB77
:100D3000C3B2A3F120023F2A88BF202309F8013B58
:100D4000E4E700BF10B5114C94F8E23423B9104B1E
:100D50004FF480225A6110BD0E4A136823F0060337
:100D6000136049F0EDF894F8E234002BEFD0D4F89A
:100D7000E8349B68DB07EAD5D4F8E425136823F050
:100D8000030161F307031360E1E700BFA84C0020F3
:100D9000003C014010ED00E008B501210320FEF702
:100DA00071F972B646F07CF92DE9F04F8DB0D04C58
:100DB000DFF85493CF4D00904FF0000854F80B0C1F
:100DC000002800F0FF8033F067FC0646002800F0A2
:100DD000DF81D9F8303044F8073CE0260023C64FC5
:100DE00004F8033CA4F10B0B06FB08F654F80B0CBB
:100DF00033F052FC002800F0E58054F80B0C33F07F
:100E000043FC14F8023C5A1E82460B2A0DD8DFE838
:100E100012F020003B004700540084009C00E400D6
:100E20001801380143017D01950124280DD0009A55
:100E300042B9B24A92F82625824240F085810122C9
:100E400004F8032C0D2BD1D186E0012304F8023CD9
:100E5000CCE700234D28C4F8C53084F8CD3084F8A1
:100E6000CE3004D0582808D004F8023CBEE7022255
:100E700004F8022C84F8C430B8E7032304F8023CD9
:100E8000022384F8C430B1E704233C2804F8023C70
:100E90000BD0BAF13E0F0CD0002304F8023CA5E7BA
:100EA0000A233C2804F8023CF3D1002304F8013C57
:100EB0009CE7012304F8013C98E7D4F8C500BB196E
:100EC0000344421CC4F8C52083F8E3AA94F8CD007B
:100ED000022A8AEA000184F8CD1087D12378C02B3A
:100EE000DAD86278FF2A08D1052BD5D9012384F8F6
:100EF000C430072304F8023C78E7A4F8C12000229C
:100F00009342C4F8C93014BF0523062384F8C320D4
:100F1000C4F8C52004F8023C68E7D4F8C500BB1942
:100F20000344421CC4F8C52083F8E3AA94F8CD001A
:100F3000D4F8C9308AEA00019A4284F8CD107FF4CF
:100F400055AF062304F8023C50E794F8CD308342B5
:100F5000A2D10D2304F8023C14F8017C002F40F0CC
:100F6000F980674B08940FCB04AE86E80F00D4F8E5
:100F7000C930D4F8D100ADF82A7023440993B4F8ED
:100F8000C130ADF8283094F8C3308DF82C300123EF
:100F90008DF82D30324603AB08A903972CF0F2FDF3
:100FA00048B1049B059394F8C420564B04933146F2
:100FB000584627F02DFE039E002304F8023C002E25
:100FC00040F0DE8008F10108B8F1030F04F1E004FD
:100FD0007FF4F4AE0DB0BDE8F08FD4F8C500BA19B7
:100FE0000244431CC4F8C53082F8E3AA94F8CD202B
:100FF00094F8CE0001938AEA020284F8CD2051468B
:10100000D5223CF019FC019B84F8CE00072B7FF41D
:10101000EDAEB4F80530C02B3FF63EAFB4F8032078
:10102000A4F8C120A27884F8C32000229342C4F817
:10103000C93014BF08230923C4F8C52004F8023CB2
:10104000D4E6D522014694F8CE003CF0F5FB94F8A6
:10105000CD3084F8CE008AEA0303D4F8C50084F8C2
:10106000CD30BB190344421CC4F8C52083F8E3AA61
:10107000D4F8C9309A427FF4B9AE092304F8023C8F
:10108000B4E694F8CD30434084F8CD3094F8CE30B7
:1010900083427FF401AF54E7D4F8C500BA19024483
:1010A000431CC4F8C53082F8E3AA94F8CE0001933B
:1010B000D52251463CF0C0FB019B84F8CE00052BA5
:1010C0007FF494AEB4F80120B4F80330A4F8C12042
:1010D000227884F8C32000229342C4F8C93014BF98
:1010E0000B230C23C4F8C52004F8023C7EE600BFA5
:1010F0008B570020986E0020A84C0020A05D002097
:10110000A0C60508C4180120B82A0020D52201462F
:1011100094F8CE003CF090FB84F8CE00D4F8C500E3
:10112000BB190344421CC4F8C52083F8E3AAD4F8D1
:10113000C9309A427FF45AAE0C2395E694F8CE302B
:1011400083427FF4A9AE04E7232804BF022204F8F7
:10115000032C77E6012F4FF0000602D004F8026C52
:1011600030E7D4F8C93008942344099308A8B4F8A8
:10117000C130CDE90A66ADF8283025F0D7FDEDE79E
:1011800054F80B0C2AF088FB54F80B0CB04719E705
:1011900014F8033C002B3FF415AFD9F8302054F875
:1011A000071C521A632A7FF60DAF012B28D0022BA1
:1011B0007FF408AF54F80B3CC5F80832C5E97F331B
:1011C0000122402389F82E2B85F80C320D4A0E4B54
:1011D000C5F8042285F80D020C4A0D48C3F8C8244E
:1011E000C5F850223AF0BCFF4FF400502CF01CFB25
:1011F00008483AF0ABFF85F8546285F85562E1E69D
:10120000FFF7CAFD25110408A05D00209C70002096
:101210006B3A0608A13A060800B5062983B00A46CB
:101220004FF03203014628BF06220DF101008DF870
:1012300000304BF0DDF8034B68461B68984703B05D
:101240005DF804FBB88900205E2810B50ED05D283B
:1012500004D00B4BBDE810405B681847084C63682E
:10126000984763683D20BDE810401847044C5D2056
:101270006368984763683E20BDE81040184700BF88
:10128000B8890020084B5A881B88801A9B1AC00016
:1012900090FBF3F00628A8BF062020EAE070C0F11A
:1012A0009600C0B2704700BF50360020094B03EBD8
:1012B00040021189084A127802EAD122520707D067
:1012C000D3F88420511CC3F88410134483F8880099
:1012D000704700BFB8890020F005002010B5164BFC
:1012E00042681B7803F00303032B21D1134B1B88A7
:1012F000DBB1134B1349B3F9C630B1F904100A241A
:1013000091FBF4F15B1A1B0103F5B95314334FF44D
:10131000B471B3FBF1F3C3F1080303F00F036033BF
:101320001370436800225A7010BD05231370F8E74C
:101330002D231370F5E700BFF03500200C36002098
:10134000B8890020D8360020436872221A7043689A
:1013500073225A70436874229A7043680022DA70CC
:1013600070470F4B4268B3F904300A2193FBF1F345
:101370001B0110B503F5B9530A4C4FF4B471143383
:10138000B3FBF1F303F00F031919E35813604B6833
:1013900053600B7A1372436800225A7210BD00BF6B
:1013A000D836002080400608044B93F8CD3013F067
:1013B000FD0F14BF9E209D20704700BFB8890020FC
:1013C000094B93F8CD3013F0FD0F06D142F21073A4
:1013D0005843064B90FBF3F07047242358434FF4D7
:1013E0007A7390FBF3F07047B889002040D2060072
:1013F000064B07EE900A93F8CD30B8EEE70A1BB91A
:10140000DFED037A20EE270A704700BFB88900207D
:1014100048F9514010B5104B93F83421012A10D1EE
:10142000D3F83821811A00290BDD0221B3F82E41AF
:1014300083F834110949B1FBF4F142B10A44C3F80D
:10144000382193F83401013818BF012010BD084439
:10145000C3F83801F5E700BFB889002040420F000B
:10146000831E00F17A02EA2123F8021F9342FBD186
:101470004E2243F64913C280CE2243850281CD23FA
:1014800023228380A0F87220A0F87830704700BF34
:1014900008BB1F48B0F83C3103F001036BBB30B40C
:1014A00090F84041ACB11B4A02F1F00502E0013373
:1014B000A3420ED052F8041B4904F8D590F82C1220
:1014C00000EB8101D1F8C41145F823100133A34288
:1014D000F0D130BC70470E48B0F83C21032A4FEAE7
:1014E00052030BD90A68A0F83C3102F5C332A0328E
:1014F00003F001030A60002BD1D070470B6803F59D
:10150000C333A03348F205020B60A0F83C217047BA
:10151000B8890020FC8A00202DE9F04100283AD14A
:101520002D4A92F8400180B32C4A2D4B92F804E0EA
:1015300092F905C092F90680CEF1FF07AEF17F0661
:10154000FFB2F6B203EB800003F1F002002403E0E7
:10155000834202F1040218D053F8041B8904F7D522
:10156000E1B2A1EB0C0181EAE175A5EBE175012D7A
:101570000DDC71B1414514BF394631468342D1700B
:1015800004F1010402F10402E6D1BDE8F081082172
:10159000F4E77146F2E7114B1A79F02A09D802F103
:1015A0000F000D4A18710B6803F582431A330B6064
:1015B000B7E7094A93F9054092F842017F25844232
:1015C0001D71987905DB4042C0B298712044587172
:1015D000E9E7002CFADAF6E7B8890020F0050020E8
:1015E000FC8A0020F0B5384E78B196F8B432002B62
:1015F00046D0364A013BDBB286F8B4321378DC07BA
:1016000041D4334B0A681A440A6096F840414CB3FF
:10161000304B2E4F03EB840403F1F001002503E06F
:101620009C4201F104011DD053F8042BC2F30320A6
:101630000628F5D13878C00715D596F8B40296F883
:1016400043E100EB050CBCFBFEF00EFB10C00128D3
:10165000CCBF0020012058B99C4205F1010501F1E1
:101660000401E1D1F0BDE84300F001000028F3D00F
:10167000C2F3834206EB8202D2F8C4210A60EBE790
:1016800096F84331B5E7D6EDB17A134B134CFDEE26
:10169000E77A642017EE902AA2F57A7200FB02F234
:1016A00083FB0230D317C3EBA01303EB4303C3EB5D
:1016B000031384FB0302DB17C3EB62130533084AF1
:1016C00092FBF3F39EE700BFB88900208435002029
:1016D000400D0300FC8A0020D34D62101F85EB51A2
:1016E00040420F00F0B4524C002868D194F8000337
:1016F000002856D04F4BD3ED007AB3EE097AF4EEC2
:10170000C77AF1EE10FA4EDCBBEE097AF4EEC77A36
:10171000F1EE10FA4CBF08270027D3ED017AB3EEA3
:10172000097AF4EEC77AF1EE10FA3EDD47F00107D0
:1017300094F84051ADB3404ADFF808C102EB85058B
:1017400002F1F00014E094F90363B142ACBF02214E
:10175000002194F90463B3421CDB41F004010F4201
:101760001CBFDCF80C300360954200F1040018D077
:1017700052F8043BD903F7D594F9026303F00F0143
:10178000B142C3F30313DEDC94F90463B3424FF0B8
:101790000101E2DA94F90563B342D8BF41F00801D0
:1017A000DDE7F0BC70470427B7E7BBEE097AF4EE3B
:1017B000C77AF1EE10FA48BF47F00207B8E794F88D
:1017C000013363B31B4B1D4DD3ED007A93ED017ACA
:1017D0000A6894F80003F0EEE77AB0EEC77AF4EE08
:1017E000C77AF1EE10FAB8BFF0EE477AFDEEE77A6D
:1017F00080F0010017EE903A193B03EB4303C3EB73
:10180000031385FB0365DB17C3EBE51305330C4DB1
:10181000B5FBF3F31A440A6084F8000368E70B6829
:1018200094F8000303F5433303F5A0730B605FE7FF
:10183000B889002040360020FC8A0020353AFC445C
:1018400040420F00ECC60508F0B40B4F97F840611A
:1018500086B107F5A272054607F50D77002352F809
:10186000044B35EA040004BF086847F8230001333D
:10187000B342F4D1F0BC7047B889002030B42A4B91
:1018800060B92A48027DCAB993F82D32284920331D
:1018900001EB830130BC4FF4A060D5E793F8062339
:1018A000F2B1013A214883F806230A6802F5C322FF
:1018B00002F520720A60027D002AE5D01D4A1268F6
:1018C0009106E1D51C4A93F80613127892071AD5AF
:1018D00011BB93F82F321649203301EB8301D9E76E
:1018E000124893F80743057DA54205D8042483F8E0
:1018F000072383F80643D8E70134012283F807431E
:1019000083F80623D1E70029BED193F82E32084987
:10191000203301EB8301BDE793F82B3204492033D8
:1019200001EB8301B6E700BFB8890020F435002041
:10193000FC8A0020E0360020F035002010B41E4A5A
:1019400048B91E4C92F808030B6823440B6098B109
:101950005DF8044B704792F8093303B3012B16D09E
:1019600092F808030B68164C80F00100234482F8BB
:1019700008030B600028EBD192F82B3211495DF877
:10198000044B203301EB83014FF440705CE792F885
:1019900008030D4C80F0010082F80803D4E70B68BF
:1019A0005DF8044B03F5742303F5107301200B60FD
:1019B00082F80803704700BFB889002040420F003A
:1019C00048E80100FC8A002020A107003C4AA0B999
:1019D00092F80A336BB192F80B138A081341DB07B4
:1019E0000AD501F00101032A06D8DFE802F05048C9
:1019F000403892F8113353BB704792F80B330133E0
:101A000003F00F0382F80B333BB192F80A330868F6
:101A100000F5C330A0300860DCE72A4882F80A33BA
:101A2000437A002B44D12848C07818B143F004030E
:101A300082F80A3325480078C00730D592F81003A1
:101A40000028E4D043F0080382F80A33DFE792F875
:101A50001E331F4901EB83014FF40030F4E61C4BA9
:101A600003F13002002914BF19461146F4E7194B5F
:101A700003F1180200290CBF19461146ECE7144B7C
:101A800003F10802002914BF19461146E4E7104B80
:101A900003F11802002914BF19461146DCE7D2F8F9
:101AA0000C030028CAD043F0010382F80A33C5E7CB
:101AB00092F80933002BB6D0022382F80A33B2E73A
:101AC000B889002050360020883500208435002059
:101AD000ECC60508FCC6050870B5214D95F8203305
:101AE000EA181C4692F824238AB11E4E09225C1C77
:101AF000A6FB04135B0803EBC303E31AE918DCB28B
:101B000091F8241309B1013AF1D185F82043026814
:101B10001549561C06600C2616700268561C066095
:101B2000002616700268561C066003EB430603EBA2
:101B30008603147019440D223AF00EFE95F8201316
:101B4000084B4A1CA3FB02035B08294403EBC303B5
:101B50000120D31A81F8240385F8203370BD00BF1B
:101B6000B8890020398EE338E88C00202DE9F04F49
:101B7000C31D85B0534C03F4FC7300AFADEB030DF4
:101B8000D4F8A83304F56E7B0DEB00025B450646E6
:101B90008A46FA60E9462FD094F8F81494F8F9C40C
:101BA000D4F8AC5301F00F0040EA4C1001310DF1B4
:101BB00001088DF8000084F8F814C7F8088007F1D0
:101BC0000800ED1AA2EB0808A845194644DD2A468C
:101BD0003AF0C2FDD4F8A823B968C4F8A8B32A44DF
:101BE000A1EB09014846C4F8AC23C9B2D047002094
:101BF0001437BD46BDE8F08F94F8F8C494F8F904A2
:101C0000B4F9B2530CF00F0141EA401141F0100158
:101C1000002DC9B2D4F8AC53B8BF41F080010CF12B
:101C2000010C012884F8F8C489F80010A5EB0B0812
:101C300022D1B8F1FE0F38DDFF2394F8B02389F8E4
:101C4000013007F1080009F103031FFA88F17860F9
:101C500089F80220BB6020E042463AF07DFDD4F8CE
:101C6000A823424448463146C4F8A823D04701205F
:101C70001437BD46BDE8F08F94F8B433B4F8B01310
:101C800089F8013007F1080009F102037860BB60B0
:101C90003AF0AAFD78681FFA88F13AF0A5FDD7E975
:101CA0000282D4E9EA3578688BE794F8B01389F8B2
:101CB000018009F1030889F80210C7F8088007F1CC
:101CC00008007EE7B8890020012979D9F0B50378AA
:101CD000614CC3F34115032D83B084F8F95403F02C
:101CE0000F077ED013F01003164606D0012D69D0E1
:101CF000052912D8002003B0F0BD94F8CC25002AA5
:101D0000F8D094F8CD25013202F00F02BA4250D03B
:101D1000184684F8CC3503B0F0BD437884F8C83554
:101D20004388A4F8C43585884318811DC02D77D811
:101D30004A4AC4F8BC2515444FF0000C0120C4F8F1
:101D4000C055A4F8C6C584F8CC05AA1A5B1A9342FC
:101D500084F8CD755FDB424D002A55D1B4F9C43506
:101D6000FA2B4CD03D4A3F49D4F8BC358868C4F8BA
:101D7000BC252946A2F5A276151FC4E9EA65C4F878
:101D8000C0350025A2F5AA7201AB84F8CC55C4F881
:101D9000B05301952BF0F6FE013054D0019B0BB1EE
:101DA00000209847D4F8A8330120C4E9EA6303B0BF
:101DB000F0BD4318D4F8C055D4F8BC25411CC4E785
:101DC00000207047022995D045788378A4F8C4355F
:101DD000FF2D1DD104298DD94318B0F80350411DA2
:101DE000A4E70023204984F8B83304F56E7204F2A6
:101DF000B933C4E9EA23C4F8B01301207BE7002E0D
:101E0000B0D005233370ADE728463AF0A5FCA5E72E
:101E10004318C11C8AE712481A463AF09DFC69E74C
:101E2000124BB4F8C405C4F8A833032101334FF6AC
:101E3000F672A4F8B003C4F8AC3384F8B813A4F86D
:101E4000B223012057E7D4F8A8330222591CC4F862
:101E5000A8131A70A2E700BFB8890020B48E002032
:101E6000748F0020F00500200000F6FF708D002028
:101E7000024B0146D3F8D00532F012BCB8890020DD
:101E8000044B93F831310BB125F080BE024B18881A
:101E9000704700BFB889002034360020084B93F803
:101EA000CD3007EE900A4BB9F8EEE77A9FED057A50
:101EB0009FED050AA7EE870A48F0F6BF704700BFFE
:101EC000B88900206766E63F0000004210B5194C53
:101ED000A379D3B194F82230DFED176A07EE903A78
:101EE000F8EEE77A154B86EEA77AC0B203EB8000D6
:101EF000B0F8E03507EE903AF8EEE77A67EE277A29
:101F0000FDEEE77A17EE900A10BD0D4B1B6813F03B
:101F100000630CD0C0B2FEF7C7FD8089642310FBBC
:101F200003F094F822305B0890FBF3F0ECE71846DE
:101F3000EAE700BF0C32002000004843B8890020C7
:101F40007836002008B5FFF7C1FF3C2390FBF3F083
:101F500008BD032811D8DFE800F00A0C0206084B80
:101F6000D3F85C067047074B1B78DB0701D431F0D0
:101F7000DFBE034BD3F8580670470020704700BF00
:101F8000B8890020843500202DE9F041294D2A4AE6
:101F90002B682A4C2E89B4F8847682FB0352DB1717
:101FA000C3EBA2031FFA83F8474582B00D4603D165
:101FB000B4F88636B34233D002680190511C342302
:101FC0000160137002680023511C016013704146C8
:101FD0003AF00AFC019831463AF006FC019847F6BF
:101FE000FF713AF001FC019847F6FF713AF0FCFBF3
:101FF000019847F6FF713AF0F7FB019847F6FF7139
:102000003AF0F2FB01980221FBF7C4FF0120A4F88B
:102010008486A4F88666C4F8885602B0BDE8F081CC
:10202000D4F88836064ACB1A9342C5D8002002B0AD
:10203000BDE8F0816C36002067666666B8890020CE
:1020400080841E00026810B57F21541C046011704A
:1020500002680024511C01600E211470FBF79AFFE6
:10206000012010BD2DE9F041694F6A4DD7F800807D
:1020700084B0044640460E460CF075F985F88C068F
:10208000B8F1000F0AD00DF1090202A940460BF089
:102090009AFF002840F08D8095F88C060023ADF85B
:1020A00008308DF80A301A46431EDBB20021FF20AB
:1020B000FD2B8DF80C20ADF80E108DF80B0003D918
:1020C000002004B0BDE8F0819DF80830042B00F03A
:1020D0009580052B00F09880032B00F09780022B51
:1020E00000F08B80012B08BF042100F087809DF851
:1020F000093038689DF80A10013B0DF10E028DF889
:1021000009300BF0C9FE95F88C36032B73D0042BE5
:102110000CD1414A9DF80A000121002301E012F888
:10212000011F81426DD20133082BF8D1D5F89026DA
:10213000029B3A4F9A420DF108084FD023680D22B6
:10214000591C21601A7023680022591C21601A70E2
:1021500023689DF80820591C21601A7023689DF897
:102160000920591C21601A7023689DF80C20591C05
:1021700021601A7023689DF80A20591C21601A708A
:10218000BDF80E1020463AF02FFB23689DF80B2077
:10219000591C216020461A700721FBF7FBFE98E8C6
:1021A000030087E803000120C5F8986604B0BDE885
:1021B000F08101A940460BF0FDFE00283FF46CAF12
:1021C00040460DF10A010BF0FBFE00283FF464AF1E
:1021D000019B95F88C0603F0010265E77A68D8F850
:1021E00004309A42AAD1D5F898360D4AF31A934290
:1021F0007FF666AFA2E70B4A8CE703218DF8081043
:1022000075E78DF80A3091E70121F7E70221F5E73C
:10221000D0350020B8890020043A060848900020F4
:1022200080841E00103A06082DE9F04FC14B1B6850
:10223000804613F0800083B000F07081BE4B1878A8
:1022400010F0020000F06A81DFF80CB39BF8143044
:10225000052B40F26881DBF80030B84D0093002B6D
:10226000B8BF5B42A5FB0342B548B649920D00FBDF
:102270000233C3EB03139B0085FB034502EB820291
:10228000DC1702EB8202C4EBA55400FB043304EB21
:102290008204A4B281FB0321DB17C3EBA111BCB103
:1022A0000025A94F2E46A7FB0432D20802EB820379
:1022B000A4EB4303E8B2A4469BB280008340BCF188
:1022C000090F94B246EA030605F10105EBD8340480
:1022D00089B2B9B100259C4F2E46A7FB0132D20826
:1022E00002EB8203A1EB4303E8B28C469BB2800071
:1022F0008340BCF1090F91B246EA030605F10105DE
:10230000EBD83443DBF804E08C4D8D4E8D498EEADA
:10231000EE70A0EBEE70A5FB0032920D06FB020002
:10232000C0EB0010830085FB035002EB8202DD1737
:1023300002EB8202C5EBA05506FB053305EB8205D7
:10234000ADB281FB0321DB17C3EBA111C5B10020A6
:10235000DFF8F4C10646ACFB0532D20802EB82037B
:10236000A5EB4303C7B2A9469BB2BF00BB40B9F17E
:10237000090F95B246EA030600F10100EBD83504D7
:1023800089B2C1B10020DFF8C0C10646ACFB013202
:10239000D20802EB8203A1EB4303C7B289469BB28A
:1023A000BF00BB40B9F1090F91B246EA030600F144
:1023B0000100EBD83543DBF80830634A0193002B6A
:1023C0001846B8BF5842A2FB0030604E6049030A6D
:1023D000A6FB0363DB0901FB03F1C1EBD00189B26A
:1023E000B9B1002691463746A9FB0132D20802EB6B
:1023F0008203A1EB4303F0B28C469BB28000834082
:10240000BCF1090F91B247EA030706F10106EBD8C8
:10241000B9B2BBF81070DFB10026DFF82CA1B446CA
:10242000AAFB0732D20802EB8203A7EB43035FFA51
:1024300086F938469BB24FEA890903FA09F309285D
:1024400097B24CEA030C06F10106E9D81FFA8CF7A3
:10245000BBF812303C4AA2FB0306F608632E28BFE5
:102460006326092B63D9002093468146ABFB0632D5
:10247000D20802EB8203A6EB43035FFA80FAB4466C
:102480009BB24FEA8A0A03FA0AF3BCF1090F96B22B
:1024900049EA030900F10100E8D85FFA89F9009BD5
:1024A000019A002BCCBF392338231616BEF1000F3A
:1024B00026F07F0635DD274A3343964543F0020672
:1024C000C8BF43F00606D8F800301622581CC8F8DA
:1024D00000001A70D8F800300022581CC8F800001C
:1024E0001A7040463AF080F9214640463AF064F9C5
:1024F000294640463AF060F9404639463AF074F9C8
:10250000D8F800305A1CC8F8002083F80090D8F89A
:1025100000305A1CC8F8002001201E7003B0BDE82E
:10252000F08F1E43CFE7002003B0BDE8F08F4FF0DF
:102530000009B4E778360020F03500206BCA5F6BE5
:10254000806967FFD34D6210CDCCCCCCC55A7C0AD4
:10255000A0860100FFC99A3BF43500202DE9F04721
:10256000AB4B1B68064613F0800084B000F09D80E2
:10257000A84B187810F0020000F09780A64F397D24
:10258000052940F29780632900F292800024DFF849
:102590009CC289B22546ACFB0132D20802EB820311
:1025A000A1EB4303E0B28E469BB280008340BEF1B4
:1025B000090F91B245EA030504F10104EBD8EDB22D
:1025C000BB68964A82FB0312D917C1EB623189B20C
:1025D000002900F018814FF0000CDFF850E264464B
:1025E000AEFB0132D20802EB8203A1EB43035FFA98
:1025F0008CF088469BB280008340B8F1090F91B2FD
:1026000044EA03040CF1010CEAD8E4B2FB898449E2
:102610004FF4F36707FB03F7A1FB0737C7F38F17E7
:1026200042F20F739F4249D8CFB10020DFF8FCE19E
:102630008446AEFB0732D20802EB8203A7EB4303CA
:10264000C1B2B8469BB289008B40B8F1090F97B26E
:102650004CEA030C00F10100EBD81FFA8CF7714B28
:10266000D3E9002313433ED14FF0FF3833681722DC
:10267000591C31601A7033680022581C306039468A
:102680001A7030463AF0B0F8414630463AF094F8C5
:1026900033685A1C32601D7033685A1C32603046F1
:1026A0001C700621FBF776FC012004B0BDE8F08722
:1026B000992585E7002004B0BDE8F0870021DFF808
:1026C0006CC10F46ACFB0302D20802EB8200A3EB05
:1026D00040039BB28B400431102947EA030793B2B1
:1026E000F0D1BFB2BBE701A83BF066F89DF8081037
:1026F000002900F08A804FF0000CDFF830E1E0465E
:10270000AEFB0132D20802EB8203A1EB43035FFA76
:102710008CF089469BB280008340B9F1090F91B2D9
:1027200048EA03080CF1010CEAD84FEA08289DF8A2
:102730000910E1B10020DFF8F4E08446AEFB01327D
:10274000D20802EB8203A1EB43035FFA80F98A46C9
:102750009BB24FEA890903FA09F3BAF1090F91B262
:102760004CEA030C00F10100E8D848EA0C089DF897
:102770000A104FEA0828E1B10020DFF8B0E08446F3
:10278000AEFB0132D20802EB8203A1EB43035FFAF6
:1027900080F98A469BB24FEA890903FA09F3BAF134
:1027A000090F91B24CEA030C00F10100E8D848EAA5
:1027B0000C08BDF80C301C49632BA1FB03214FEA28
:1027C00008184FEA51117FF651AF0020DFF85CE0A6
:1027D0008446AEFB0132D20802EB8203A1EB430335
:1027E0005FFA80F98A469BB24FEA890903FA09F336
:1027F000BAF1090F91B24CEA030C00F10100E8D8DC
:1028000048EA0C0832E70C4600E788468FE700BF2D
:1028100078360020F0350020F435002089B5F81412
:10282000D34D6210589000201F85EB51CDCCCCCCFD
:1028300002683B4B70B505467E21501CB3F9A836A3
:10284000286011702968374C03EBC30384FB030233
:10285000481CDC17002328600B70FF20C4EB6204C7
:10286000FEF722F92034304BA4B200284DD01B785B
:10287000B0F90C1023BB2D4BA1F57A729A4246D8C1
:102880002B48B0FBF1F189B2284639F087FF294B7C
:10289000DB7A7BB125F07AF90146284639F07EFFD4
:1028A0002146284639F07AFF28460821FBF772FBBB
:1028B000012070BD204B2846198839F06FFFEFE7E3
:1028C0001E4B1E78002ED6D01D48002300EB83023D
:1028D00001339289B3421144F8DB1A4B9FED1A6A17
:1028E00093F8223007EE103A07EE901AB8EEC77A46
:1028F000F8EE676AC6EE077A67EEA67AFCEEE77A2C
:1029000017EE901AB1FBF6F1B5E71B7813B94EF646
:102910009C21B9E7094B1E78002EF8D00146D3E779
:10292000B889002067666666D75D00201783930329
:10293000008793031036002034360020B42B00208B
:102940008C8F00200C32002000004843034B0449C8
:10295000B3F90C30406801223EF066BEF00500205D
:102960005F3A060837B504462A4800EB4303B3F83C
:10297000CE5005F00F0049B1022804F101011DD825
:10298000002814BF9C239B2323700C460AB3C5F375
:102990000315FFF7DEFA3C21012D1F4BB0FBF3F3CB
:1029A000B3FBF1F201FB123315D0022D23D01B49EA
:1029B000204603B0BDE830403EF036BE032806D1C5
:1029C000174B1B7803F00103653BDBB2DCE72023E8
:1029D000DAE71546DDE7642542F21071B0FBF1F14C
:1029E000B1FBF5F005FB101000900E4920463EF0BB
:1029F0001BFE03B030BD0A250B49B0FBF1F1B1FB62
:102A0000F5F005FB10100090084920463EF00CFE42
:102A1000EFE700BFB889002040420F00A63A060841
:102A200084350020B03A0608A0860100BF3A0608A7
:102A3000037840680122053B114693E7064B07499E
:102A40001A88074B40681B68534342F2107293FB8D
:102A5000F2F23EF0E9BD00BF34360020CE3A06085F
:102A60006C360020054A064992F8AD3692F8AC263D
:102A70004068013301323EF0D7BD00BFB889002065
:102A8000D33A06080B4B4068B3F904300A2293FB93
:102A9000F2F31A0102F5B9524FF4B4711432B2FBD9
:102AA000F1F2C2F1080202F00F02034960323EF077
:102AB000BBBD00BFD8360020D93A0608034A0449F6
:102AC0009268406807233EF0AFBD00BF6C3600201F
:102AD000E03A060807B5144A406892F8BC16B2F806
:102AE000BE36012909D1009392F8C0360F497B22E6
:102AF0003EF09AFD03B05DF804FB022906D10C49B3
:102B00007B2203B05DF804EB3EF08EBD0A225343F6
:102B100040F2FF32B3FBF2F39BB2092B054928BF09
:102B200009237B22EDE700BFB8890020E63A0608BA
:102B30009B3B0608F03A060813B54468FEF734FCE0
:102B40000F4B1B789B07024612D50E4B93F8CB1602
:102B50000D4B59B19889FEF733FC0C49009203469E
:102B6000702220463EF060FD02B010BDD889F2E729
:102B7000009007492D23702220463EF055FDF3E7D3
:102B8000F0350020B8890020F43500204E3B0608BF
:102B9000F63A06082DE9F0413F4F90F800C03C7826
:102BA000416890F803E0BCF1170F0CBF4FF0980894
:102BB0004FF0890814F0040486B0064605D0374B60
:102BC000BCF1170F0CBF5C681C68354D84EAE473D8
:102BD000A3EBE473BEF1010FB3FBF5F201F10100C9
:102BE00005FB123343D0BEF1020F44D181F80080BF
:102BF0003C214B43B3FBF5FE05FB1E334B43BCF1BD
:102C0000170FB3FBF5F105FB1135264BB5FBF3F5BB
:102C100028D1002CB4BF5723452305932223CDE9A7
:102C200003532723CDE900E3029108231E493EF018
:102C3000FBFC33781D495A0901EB820103F01F03A5
:102C4000012202FA03F33A78D1F8D00602F0060224
:102C5000042A0CBF034320EA0303C1F8D03606B0B0
:102C6000BDE8F081002CB4BF53234E23D5E74FF4C9
:102C70007A75B3FBF5F3002C81F8008002DA2D247D
:102C8000881C4C700A4C0B49BEF1000F08BF21464E
:102C90003EF0CAFCCDE700BFF0350020F43500203F
:102CA0008096980040420F000D3B0608B88900202E
:102CB000FD3A0608053B06080D4B1B681B0137B59E
:102CC00014D50C4C4568D4F8D83693F90100FFF7B9
:102CD000E5F894F8CD200849002A0CBF0D220E22F9
:102CE0000346009228467A223EF09EFC03B030BD97
:102CF00078360020B8890020233B0608034B04499E
:102D0000D3F8DC2640683EF08FBC00BFB8890020B5
:102D10002C3B0608044B1B78DB0703D403494068AF
:102D20003EF082BC704700BF84350020303B06086F
:102D300007B5094A0949B2F906300193B2F90430DE
:102D40000093B2F902304068B2F900203EF06CFC0A
:102D500003B05DF804FB00BF84310020393B060856
:102D600037B50A4C4568B4F9A806FFF797F894F808
:102D7000CD200749002A0CBF0D220E2203460092E7
:102D800028467A223EF050FC03B030BDB8890020BE
:102D90004D3B0608084BD3F8EC26002A0ADD074B0A
:102DA00003EB82035A6B2AB1054B06491B69406845
:102DB0003EF03ABC704700BFB8890020ECC6050859
:102DC000F0050020563B06081FB5938802939378C0
:102DD00001935378009313780A4603493EF024FC8C
:102DE00005B05DF804FB00BF5E3B0608034B0449D9
:102DF000D3F8F02640681432E6E700BFB889002017
:102E0000713B0608034B0449D3F8F02640680832AA
:102E1000DAE700BFB8890020753B0608034B044978
:102E2000D3F8F02640680E32CEE700BFB889002004
:102E3000793B06082DE9F0472DED028B82B09246D2
:102E40009DF834809DF8302007460C469946002BAB
:102E500052D0022B14BF0A25642507EE905AF8EED3
:102E6000E77A27EE808A002A48D0B0EE480A48F078
:102E70001BF807EE900AF8EEE77AF0EEE77AFDEE3F
:102E8000E77A17EE906AB6FBF5F205FB12660CB115
:102E90003C700124B5EEC08AF1EE10FA05D552EA75
:102EA000060302D02D233B5501349AF80010154B30
:102EB0003819002914BF514619463EF0B5FB2518B4
:102EC000B9F1000F0AD010494A4668463EF0ACFB03
:102ED0007819324669463EF0A7FB0544B8F1000F69
:102EE00002D007F805800135002328467B5502B043
:102EF000BDEC028BBDE8F0870125AEE7F0EE487A25
:102F0000BBE700BF7D3B0608823B0608194B1B68E8
:102F100013F0200F13B5446825D0174B1B789B077F
:102F200021D5164BB3F90000FEF762FADFED147AF3
:102F3000144B154A93F8CD3020EE270A2046B5EE03
:102F4000C00AF1EE10FA4CBF76217521002B0CBFA0
:102F500099239F23019301230093B0EEC00AFFF74A
:102F600069FF02B010BD2D232370436800225A7000
:102F7000F7E700BFE0360020F0350020DE36002005
:102F80000AD7233CB8890020218B06081FB5184BAF
:102F90009FED187A1B88184A9FED180A92F80923AA
:102FA000446807EE903AF8EEE77AF4EEC77AF1EE6D
:102FB00010FAACBF01230223022A27EE800A14D0A4
:102FC0008DED030A029324F0E1FDFEF75BF9029B0D
:102FD0009DED030A014601220620CDE90020084AA2
:102FE0002046FFF727FF04B010BD9721F3E700BF8D
:102FF0003436002000007A44B88900200AD7233CE8
:10300000218B0608114BB3F8F436B3F57A7F07B578
:10301000406806D20E49012203B05DF804EB3EF091
:1030200003BB07EE903A5722F8EEE77A00239FEDB4
:10303000090ACDE900320123074A27EE800A194622
:10304000FFF7F8FE03B05DF804FB00BFB88900206D
:103050008A3B06086F12833A218B060873B5194E16
:1030600096F81037052B0546406807D016491F23F0
:103070001E2202B0BDE870403EF0D6BA134C14498F
:10308000237D00931E221F233EF0CEFA96F82231B4
:10309000ABB16B68DFED0F7A20221A54638A0E4AB7
:1030A00000EE103A441CB8EEC00A68680123002103
:1030B000CDE9003120EE270A2044FFF7BBFE02B025
:1030C00070BD00BFB8890020923B0608F43500208F
:1030D000993B06080AD7233C218B060807B5012334
:1030E0004722CDE900320549054A91ED000A4068C2
:1030F0000021FFF79FFE03B05DF804FBD090002095
:10310000218B060807B50B4BDFED0B7A93ED000A18
:103110000A4A00219A23B8EEC00ACDE9001320EE36
:10312000270A0223B0EEC00A4068FFF783FE03B00F
:103130005DF804FB6C3600200AD7233CA13B06084F
:1031400013B5044624F022FD0E4B646893F809334E
:10315000022B00EE100A13D0FEF794F80146DFEDC3
:103160000A7AB8EEC00A00230622CDE9003220EE2A
:10317000270A064A02232046FFF75CFE02B010BD74
:103180009721ECE7B88900200AD7233C218B060859
:1031900013B50378134ADFED147A144C1A2B0CBFC5
:1031A000B2F90220B2F9002000EE102AB8EEC00AEF
:1031B0001A2B20EE270A4FF001034FF00002CDE951
:1031C0000032B5EEC00A0CBF15211421F1EE10FA41
:1031D000074A406848BF2246B0EEC00AFFF72AFE01
:1031E00002B010BDD8360020CDCCCC3DA53B0608A2
:1031F000AB3B0608174B1B6837B59A06446820D5C9
:10320000154B1B789B071CD5144AC17892F8CD301A
:10321000D2F81C07002B0CBF0F250C25FEF7E8F891
:103220000123DFED0F7A0093CB1A0E4A019520EEB1
:10323000270A18BF01237F212046FFF7FBFD03B0BB
:1032400030BD7F23237043682D225A7043680022CB
:103250009A70F4E7E0360020F0350020B8890020AD
:103260000AD7233C218B060813B5044608461146AD
:10327000FEF7BEF8174B93F8CD30002B0CBF4FF480
:10328000A5534FF47A7307EE903AF8EEE77A08BF49
:103290007E22F4EEC07A16BF7D220F230C23F1EEBE
:1032A00010FA13DC80EE270AF2EE047AB4EEE70A95
:1032B000F1EE10FAACBF012302230192002200922A
:1032C0002046054AFFF7B6FD02B010BD1A4600239E
:1032D000F3E700BFB8890020218B060810B40C4B1F
:1032E00044681B7803F00303032B06D1094B2046E7
:1032F00019885DF8044B1122B6E711232370436847
:103300002D225A70436800229A705DF8044B704772
:10331000F03500200C360020094B40681B7803F084
:103320000303032B07D1074B7122D3F82017642323
:10333000B1FBF3F198E704492D2371223EF074B9F3
:10334000F0350020B8890020F83A06081E4B1F49C6
:103350009A68B1F8C8309FED1E7A406807EE902A4F
:10336000F8EEE76A07EE903AF8EEE77A67EE877ACA
:10337000F4EEE76AF1EE10FA02D816493EF054B9BD
:10338000934202DA14493EF04FB99B1A07EE903A85
:1033900001F5CB63B8EEE77AD3ED007A0F4AF8EE89
:1033A000677A3C2167EE277A87EEA67AFDEEC77A28
:1033B00017EE903AB3FBF2F3B3FBF1F201FB1233D9
:1033C00007493EF031B900BF6C360020B8890020B3
:1033D000CDCCCC3DB13B0608B73B060840420F00C0
:1033E000A63A0608244A00234361D2F8DC1041F4CF
:1033F0005C5130B541F02C010124C2F8DC1044715D
:10340000D2F8D41004FA03F50133112B41EA050177
:10341000F8D121F4F0314FF42063C2F8D410C38006
:1034200040F601230381154B0360142303718023AD
:10343000037642F614035022114903824FF6FF73BC
:103440004383A0F8562003F58C036FF07E42C0E959
:103450001612C3610B4A40F2012303844FF0A064AB
:103460000023C0E9184280F8223080F8333080F819
:103470004430A0F8683030BDB88900209808640056
:10348000C4FF00FF180B0C0008B5A0F10103B3FA4C
:1034900083F302284FEA531301D0184608BD0F20CA
:1034A0001EF078FA28B9054B1B7803F00103184683
:1034B00008BDBDE808400F201CF086B98435002007
:1034C00010B5044613201CF07FF9A0B10A4B6068C8
:1034D00093F82527032A4FF0100202D1D3F8303792
:1034E00023B9BDE8104005493EF09EB8BDE8104044
:1034F00003493EF099B810BDB8890020BD3B0608CD
:10350000C28E060838B5802200F1800400210546ED
:1035100048F0CFFF00212046382248F0CAFF0C496E
:10352000002351F8232044F8232001330E2BF8D137
:1035300008491E2205F1C00048F05AFF06490B2237
:1035400005F1E40048F054FF032385F8EF3038BD5F
:10355000ECC60508A8C70508C8C70508224B1B8884
:103560005A0510B5446805D520462049BDE81040ED
:1035700048F0C3BF180505D520461D49BDE81040D9
:1035800048F0BBBF590605D520461A49BDE8104092
:1035900048F0B3BFDA0705D520461749BDE810400B
:1035A00048F0ABBF9B0705D520461449BDE8104045
:1035B00048F0A3BF25201CF007F928B12046104988
:1035C000BDE8104048F099BF0E4B93F834372BB14B
:1035D00020460D49BDE8104048F08FBF20460B49FA
:1035E000BDE8104048F089BF7C360020C13B06088A
:1035F000C63B0608CB3B0608D03B0608D53B060871
:10360000DA3B0608B8890020DF3B0608E43B0608E1
:10361000074B93ED6E7AD3ED6B7AB4EEE77AF1EE69
:1036200010FA03DD0349406848F067BF704700BFE8
:1036300050630020E93B060810B50C46A0B9184AB3
:10364000184892F8351723680344236001B110BD70
:1036500092F82B3214492033BDE8104001EB83016E
:103660004FF48060FEF7F0B812F0B8FE32280ADDA1
:1036700023680B4A03F5742303F5107301212360BB
:1036800082F8351710BD064A92F83517142881F0D4
:103690000101CCBF0548064882F83517D3E700BFC3
:1036A000B889002040420F00FC8A002020A10700BA
:1036B00048E8010010B5044623F04CFB03490346DB
:1036C00004226068BDE810403DF0AEBF5F3A0608D6
:1036D000F0B52B4B2B4E1C68317887B0074620463F
:1036E0000AF056FC7178054620460AF03DFC00229F
:1036F0000592B2788DF8132003466CB1039005A9AA
:1037000020460AF057FC327A039B2AB10DF11301CF
:1037100020460AF055FC039B9DF81310ECB1E1B173
:10372000194A1268914218DC184A02EB8102D2F859
:103730003847039326201CF047F80599039B70B97E
:1037400011F0010F14BF502200228907786808D5B4
:103750000F493DF069FF07B0F0BD0E4CE9E7442288
:10376000F3E732B1CDE900420B492A463DF05CFF58
:10377000F1E70A4900942A463DF056FFEBE700BF07
:10378000D035002040350020602B0020B889002073
:10379000EC3B060841420608F43B0608003C0608DC
:1037A000F8B50446417882782C48237890F8E9509F
:1037B000302B05F1FF352A4B4FEA85052B444FF49A
:1037C0007A770BBF93F8E75093F8E95093F8E860E5
:1037D00093F8EA6000EB8505D5EDAE7AFDEEE77A69
:1037E00000EB860017EE903AD0EDAE7A40F2CF753E
:1037F000FDEEE77AAB4217EE900AA8BF2B46B3F571
:103800007A7FB8BF4FF47A73A842A8BF2846A3F5C1
:103810007A73B842C3EB0313B3FBF7F3C3F10E03A0
:10382000B8BF3846DBB24FF0030CB3FBFCFC0CEB2B
:103830004C0EA3EB0E03A0F57A706244C0EBC000FF
:103840000833B0FBF7F73944DBB2D2B2C9B2204635
:10385000FAF7F8FE00232373F8BD00BFB8890020F3
:10386000ECC605082DE9F04790F8029090F8018029
:1038700009F1020704460026FFB2002508EB060AFC
:10388000032E1BD108F10301022DC9B20ED10B2367
:103890003A462046FAF7D6FE0135052DF0D101361D
:1038A000072EEAD100232373BDE8F08709EB050258
:1038B0001623D2B22046FAF7C5FEEDE7022DEBD172
:1038C00017233A465FFA8AF12046FAF7BBFEE3E790
:1038D00070B504466FF00205A278617852FA85F25D
:1038E00007391323D2B2C9B22046FAF7ABFEA27849
:1038F0006178EEB2324407311323D2B2C9B2204606
:103900000135FAF79FFE042DE6D16178A2780639D9
:103910000323C9B22046FAF795FE6178A2780631F2
:103920000223C9B22046FAF78DFE0023237370BD2F
:103930002DE9F8432B49054691F8D83091F8D92064
:10394000294891F8E710B0F90040002902EB820203
:1039500014BF4FF0FF31012152004C43C2F1000867
:1039600003EB830344454FEA430303DB9442A8BFC0
:103970001446A046B0F902205C424A43A24203DB4F
:103980009A42A8BF1A4614461BB11922544394FB0D
:10399000F3F4293C4FEA88066FF003074FF009095A
:1039A000002E3346B8BF06F13F03C4EBA313512BDF
:1039B0000FD893FBF9F101EBC1029B1AAA780A44D4
:1039C0006978803B3944DBB2D2B2C9B22846FAF7F3
:1039D00039FE0137052FA6EB0806E1D100232B7332
:1039E000BDE8F883B8890020D836002010B5044619
:1039F00012F030FD642202FB00F3C3F38F23632B2C
:103A000060680449BDE8104028BF632301223DF0EF
:103A10000BBE00BF9B3B06082DE9F843054617F097
:103A200087F81D4EDFF87490074600244FF0880891
:103A300033786968A342214403DC00230B70BDE89E
:103A4000F88337B3D6ED427AFDEEE77A09EB8403CB
:103A500017EE900AD3ED007AFDEEE77A17EE902A82
:103A6000D6ED437AFDEEE77A121A17EE903AD200BD
:103A70001B1A92FBF3F3C3F188030B702046FEF789
:103A800025FAB0F57A7F02DA6B6853221A550134B1
:103A9000CEE781F80080FAE7B42B002014910020D3
:103AA00013B5374BC1789A68364B02299B89044677
:103AB00041D0032945D0012905D19A1A9A42A8BFBD
:103AC0001A4622EAE272D3B19A1A9A42A8BF1A465B
:103AD00022EAE27207EE902A0B20B3FBF0F307EE26
:103AE000103AF8EEE77AB8EEC70A87EE800A47F098
:103AF0004DF9FCEEC07ACDED017A9DF80430626894
:103B00008A211170012261689342ACBF8B208D2005
:103B1000885401320C2AF6D162688F2111735A1E23
:103B2000092A03D8626813448E225A7063680022FF
:103B30005A7302B010BD9A1A9A42A8BF1A4622EAD6
:103B4000E272ABB107EE902AB8EEE70ADFED0E7A2B
:103B500020EE270A07EE903AF8EEE77A80EE270A81
:103B600047F0A2F964280346A8BF642323EAE3735D
:103B700006496068072202B0BDE810403DF054BD20
:103B80006C360020503600200000C842093C060870
:103B9000244B1A6812F0200213B5044624D0224B9D
:103BA0001A7812F001021FD0204B1A7812F002028C
:103BB0001AD01F4BD88963282AD9FDF701FC1D4B69
:103BC000D3ED007A07EE100AF8EEE77AB2EE040AB7
:103BD00067EE807AB8EEC70A174887EE800A37F09A
:103BE000F9FD47F061F90246144B606893F8CD3057
:103BF000541E002B42F20E710CBF7E237D238C429B
:103C000008D800930E4907233DF00EFD02B010BD09
:103C10000022E9E70B49072202B0BDE810403DF061
:103C200003BD00BFE036002084350020F0350020C1
:103C3000F43500206C36002034910020B889002033
:103C4000103C0608193C0608F8B52D4F0A24B7F9B0
:103C5000002092FBF4F484EAE473A3EBE4739BB2D8
:103C60005A2B054605D90A32CCBFB4236FF0B303F3
:103C70001C1B244E96F8102332B9234B1B78DB070C
:103C800029D41BF0E5FE30BB96F88837B32B02D859
:103C90001BF0DEFEF8B9B7F902100A2391FBF3F32B
:103CA00004B9C3B1002BB8BF5B4284EAE4709BB295
:103CB000A0EBE470B3EB400F6A6813DAB0EB430F8C
:103CC00010DA092908DD002CCCBF6E2362231370A3
:103CD0006B6800225A70F8BD002CCCBF6A236623A3
:103CE0001370F5E7834205DD0929CCBF6023682303
:103CF0001370EDE7002CCCBF6C2364231370E7E74F
:103D0000D8360020B88900208435002030B585B031
:103D1000054601A839F050FD044618B92870204620
:103D200005B030BD044A0123B2F98C2701A9284609
:103D30003EF03EF9F3E700BFB88900204068E5E7B0
:103D400073B50D4D0091044616460023024602212C
:103D5000286835F09BFC094B009322462868002315
:103D6000142135F093FC2868009600232246162182
:103D700035F08CFC02B070BDDC660020C670060811
:103D80002DE9F043C24C94F88E378BB0D3B1C14EBD
:103D9000C149DFF854C3C148C14A012794F88F379D
:103DA000D4F8DC80F518172B33D984F88F3794F8C2
:103DB0008E3794F89027002A40F0818284F890375B
:103DC000012023E094F89057002DE0D0B54A106808
:103DD000027A95422946A8BF1146954238BF013163
:103DE000A2EB010202EBD27238BF0123C2F34702F9
:103DF00013B984F88E27CAE7531C84F88E37AA4B70
:103E000000930221002335F041FC00200BB0BDE8F7
:103E1000F08315F801EB07FA0EF9013319EA080FE0
:103E2000DBB2C0D094F88E5784F88F37BEF1170FED
:103E3000B4D801A353F82EF0993E0108D73E0108EB
:103E4000093F01085D3F0108893F0108CF3F010894
:103E50000F4001084F400108ED4001080B410108E7
:103E60002D410108253F01084F4101089D3D0108F2
:103E700073410108A1410108CB410108E14101085A
:103E8000A93F010801420108474201085D420108BB
:103E9000834201082F42010802AE3046FFF736FF89
:103EA00018B9824930463DF0BFFB7E480096006855
:103EB00000232A46022135F0E9FB7A4A94F88E372E
:103EC00012680133127ADBB29A4284F88E377FF699
:103ED00070AF00209AE7B4F8CE20002312F00F0252
:103EE000194618BF012202A8FEF73CFDB4F8CE30F7
:103EF00003F00F026E4B03EB82032846D3F8F81051
:103F000002AAFFF71DFFD8E7B4F8D020012312F072
:103F10000F0218BF1A46002102A8FEF723FDB4F8CD
:103F2000D030E5E7D4F86C06FDF762FA94F8CD30AE
:103F3000DFED607A604A002B0CBF0F230C23019346
:103F4000012320EE270A0093002102A8FEF772FF4A
:103F50005A4902AA2846FFF7F3FEAEE713681B068C
:103F60007FF51CAFB4F96006FDF72AFA0246FDF7AB
:103F70001BFA5349034602A83DF056FB514902AAD9
:103F80002846FFF7DDFE98E713681B067FF506AFAE
:103F9000B4F9701602A80022FFF766F94A4902AA8E
:103FA0002846FFF7CDFE88E713681B067FF5F6AEBF
:103FB000D4F82017642302A8B1FBF3F10022FFF725
:103FC00053F9424902AA2846FFF7BAFE75E7B4F949
:103FD0006236DFED387A384A00EE103AB8EEC00AA1
:103FE00001230620CDE9003020EE270A022300211C
:103FF00002A8FEF71FFF94F83101354B354902AA9C
:10400000002808BF19462846FFF79AFE55E7B4F87E
:104010006436DFED287A284A00EE103AB8EEC00A7E
:1040200001230621CDE9003120EE270A02230021D9
:1040300002A8FEF7FFFE94F83101274B274902AA98
:10404000002808BF19462846FFF77AFE35E7FDF736
:1040500017FF07EE900AB8EEE70ADFED167A0123A4
:104060000622CDE9003220EE270A134A022300215E
:1040700002A8FEF7DFFE94F83101194B194902AA94
:10408000002808BF19462846FFF75AFE15E700BF6B
:10409000B8890020F4C7050870430020503600207E
:1040A00078360020DC660020633C0608733C060876
:1040B000ECC605080AD7233C218B06087A3C060883
:1040C000873C06088C3C0608963C0608A33C06087C
:1040D000303C0608233C0608493C06083C3C0608E0
:1040E0004D3C0608553C0608E036002002A994F82D
:1040F0006806F9F7C5FD734902A848F0E2F972496C
:1041000002AA2846FFF71CFED7E6837A002B3FF46D
:1041100045AEB4F966266D499A2302A83DF084FAAB
:104120006B4902AA2846FFF70BFEC6E6837A002BEE
:104130003FF434AE674A65499268072302A83DF010
:1041400073FA654902AA2846FFF7FAFDB5E694F826
:104150002537002B3FF422AE032B3FF41FAE5F49FF
:1041600002A83DF061FA5E4902AA2846FFF7E8FD81
:10417000A3E6DCF800309B077FF510AE0123472251
:10418000CDE900325749584A91ED060A02A80021AC
:10419000FEF750FE554902AA2846FFF7D1FD8CE6EE
:1041A000B4F97806FDF77AFE94F8CD304749002B34
:1041B00002460CBF0D230E2302A83DF035FA4C49F0
:1041C00002AA2846FFF7BCFD77E602A9D4F87C06D0
:1041D000F9F756FD474902AA2846FFF7B1FD6CE6FC
:1041E000B4F88026444902A83DF01EFA354902A8D9
:1041F00048F067F9414902AA2846FFF7A1FD5CE6AD
:10420000CB68002B7FF7CAAD0A69002A09DD3C495B
:1042100002A83DF009FA3B4902AA2846FFF790FDA3
:104220004BE6394A37492846FFF78AFD45E6B4F997
:104230008226364902A83DF0F7F9354902AA2846F8
:10424000FFF77EFD39E602A9D4F8DC06F9F718FD80
:10425000304902AA2846FFF773FD2EE63C21D4F828
:10426000E036B3FBF1F302A8B3FBF1F201FB12332A
:1042700029493DF0D9F9294902AA2846FFF760FDEE
:104280001BE694F8CD30D4F8E42673B940F24961C6
:104290007E23B2FBF1F202A80C493DF0C5F920499A
:1042A00002AA2846FFF74CFD07E64FF47A717D23FA
:1042B000B2FBF1F202A805493DF0B6F9EFE70120A3
:1042C000A4E500BF0E3C0608B33C0608873C060880
:1042D000BC3C06086C360020C83C0608D13C0608E9
:1042E000D73C060814900020218B0608E03C060805
:1042F000EC3C0608F93C06080F8C0608053D06084C
:104300000E3D0608133D06081C3D06085A3B0608EC
:10431000253D0608323D0608403D0608493D060891
:104320005B3D06082DE9F043744B1F6883B0002FF6
:1043300056D0FF238DF803308DF80230002877D156
:104340006F4B93F89127002A4DD093F84051002DE0
:1043500046D06C4A93F896176B48936992F814808C
:1043600000294FF0000103F0010C14BF4FF00F0EB5
:104370008E4600F1F0020B460F4612E0984554D3EA
:10438000BCF1000F51D174461E260133DBB21680FA
:104390009770D4700131A94222D0062B02F1040299
:1043A0001ED050F8044B2404F4D5002BE6D17446FB
:1043B0007826EAE7012203EB8202B169D2F8C42130
:1043C0000192CA077CD593F89637002B14BF0F23B0
:1043D000002301A94FF400408DF80730FDF734FAAF
:1043E00003B0BDE8F083474EB3F8922741F228614D
:1043F0008A42DFD941F24F618A4263D941F2766144
:104400008A4261D941F29D618A4262D941F2C56115
:104410008A426FD941F2EB618A426DD941F2127141
:104420008A4294BF0B220D22C5E700242646ACE742
:10443000344E0DF102020C4638460DF1030109F02D
:10444000C2FD06F11401384609F0BAFD06F1180163
:10445000384609F0AFFD9DF803909DF8028049466B
:104460004246384609F02CFDB569317D244B05F0F4
:10447000010505EB410505EB091593F89127A3F814
:10448000920705EB0825ADB202BBB3F89427AA4208
:1044900021D0A3F894570F22206893F8965700F57F
:1044A0004331013AD2B201F5A07185F0010083F8E1
:1044B0009127216083F89607002A7FF446AF92E7A0
:1044C000FF2386E7022276E7032274E7A3F89457D6
:1044D000E2E704226FE7216893F89607A3F8942790
:1044E00001F5433202F5A07280F00101226083F8E9
:1044F000961779E706225EE70A225CE7D0350020AE
:10450000B8890020F0050020FC8A00200B4B9B7A24
:1045100013B10B4B9B8B53B90A4B0B4AB3F90430C5
:1045200082FB0312D817C0EBA20000B27047074A03
:10453000906890FBF3F000B2704700BF5036002047
:1045400010360020D8360020676666666C3600207C
:10455000F8B5184CC6B205463146D4F8980730F085
:104560009FF894F89C17D4F89807C5F307274E4096
:10457000394684F89C6730F093F894F89C17D4F887
:104580009807C5F307464F40314684F89C7730F0D2
:1045900087F894F89C17D4F898072D0E4E402946BA
:1045A00084F89C6730F07CF894F89C174D4084F8B0
:1045B0009C57F8BDB889002070B50C4DC6B2314685
:1045C0000446D5F8980730F06BF895F89C17D5F8A5
:1045D0009807240A4E40214685F89C6730F060F821
:1045E00095F89C174C4085F89C4770BDB889002011
:1045F00038B50B4C002305462421D4F8980784F8DD
:104600009C3730F04DF8D4F89807542130F048F832
:10461000D4F898072946BDE8384030F041B800BFCB
:10462000B88900202DE9F043DFF898932DED028B37
:1046300099F89D4783B00E461546002C00F0418244
:10464000013C89F89D479FEDD48AD44FDFF87883E9
:104650003378002B60D099F89D47002C5CD135B1A0
:104660002FF066FB2B68C01A002880F2028499F8AC
:104670009E47002C40F0A68399F89F07062840F239
:10468000E081C74991F8213091F820209A4200F04A
:10469000088251F81C4F99F8A02734F813401444AD
:1046A00001300133A4B2C0B2DBB2B4F5E06F89F8D7
:1046B0009F074B7100F0DB8100F2AA80B4F5806F98
:1046C00000F0F08264D9B4F5A06F00F0C4823CD948
:1046D000B4F5A16F25D8601EC0B2FCF7E5F9C8B1EA
:1046E000B0F90C30AF4AADF8014092F82210D9F879
:1046F000002003EB830303EB830349089B0093FB38
:10470000F1F31021CDF803308DF800106846904782
:1047100000233370002D9BD103B0BDEC028BBDE8AC
:10472000F083B4F5C06FF5D19F4B9B89002B00F04F
:10473000568323F037FA10220024CDF80300062315
:104740008DF800208DF8014023E2B4F5826F00F06F
:104750004F82B4F5846F40F03981944B1B789A07EF
:10476000D8D5934AD9F800301288CDF8032010220A
:104770008DF80020202104228DF801108DF80220F0
:104780006846002498473470002D7FF461AFC3E77A
:10479000B4F5067FBED8B4F5007FC0F03381A4F530
:1047A0000073182BB6D801A252F823F0314B010840
:1047B0001F4B01081F4B01081F4B01081F4B01082D
:1047C0001F4B01081F4B01081F4B01081F4B01081D
:1047D0001547010815470108154701081547010845
:1047E000154701081547010815470108074B01083F
:1047F000F14A0108F14A0108F14A0108F14A0108A9
:10480000F14A0108F14A0108F14A0108F14A010898
:10481000B4F5116F00F0D9815CD8B4F5026F00F0E7
:10482000C38122D9B4F5036F00F06A82B4F5046F36
:104830007FF470AF5F4BD9F80020B3F9043003EB7D
:1048400083035B001020CDF80330402108238DF84E
:1048500000008DF801108DF8023068460024904762
:104860003470002D7FF4F4AE56E7B4F5E46F00F039
:104870007B81B4F5006F6ED14C4A127891077FF5B9
:1048800049AF13F0010F4C4B00F006835A6882EADF
:10489000E273A3EBE27303EB5303A7FB0313DB0801
:1048A000002AACBF43F0004343F0404310210024F2
:1048B0000822CDF803308DF800108DF80140D9F8AA
:1048C00000308DF80220684698473470002D7FF440
:1048D000BFAE21E745F230239C4200F0AF8115D9ED
:1048E00045F240239C4200F0208245F250239C4236
:1048F0007FF410AF314AD9F800309268CDF8032028
:1049000010228DF800205021522235E7B4F5376F80
:1049100000F03A826FF437616318072B3FF6FAAE66
:10492000A4F17100C0B2FCF7BFF800283FF4F2AE6A
:1049300090F90130CDF8033010238DF80030ADF838
:104940000140D9F800306846984700233370002DA5
:104950007FF47EAEE0E6B4F5E26F7FF4DBAE184B99
:1049600093ED130AD3ED007A20EE270A002420EEFF
:10497000080A46F099FA10230722CDF803008DF8B3
:1049800000308DF801308DF80220D9F800306846EB
:10499000984734709AE700BF0000C8421F85EB516A
:1049A000F00500200C32002050360020F0350020A9
:1049B0000C360020D8360020F43500206C3600205C
:1049C00080360020B8890020C5B3A29140F201438F
:1049D0009C427FF49FAEB9F9A836CDF80330102180
:1049E000012204238DF800108DF801208DF802308B
:1049F000D9F800306846002498473470002D7FF4C1
:104A000027AE89E6B4F5807F00F00C81B4F5887F8D
:104A10007FF480AECB4BD9F80020B3F90030CDF84D
:104A20000330012110238DF800308DF801308DF80E
:104A300002106846002490473470002D7FF408AEC1
:104A40006AE60130C049C0B291F8292091F82830B7
:104A5000934221D0531CDBB252004C6ABB49A45A8A
:104A600089F89F07B4F5E06F4B717FF425AEB84B22
:104A700093ED120AD3ED007A20EE270A002420EEEF
:104A8000080A46F011FA10220723CDF803008DF82A
:104A900000208DF801407CE0002281F829200123CC
:104AA000DBE7AC4A99F8A037127881F8214001334E
:104AB000DBB20132934289F8A03700F07F810120F8
:104AC000C2E700283FF4BFAD0378303B012B3FF62F
:104AD000BAAD013009F29D720621FDF7F5F899F89B
:104AE0009D3789F89E07002B3FF4ADAD3470AAE5E1
:104AF000A4F11100C0B2FBF7D7FF00283FF40AAEC3
:104B0000B0F9023016E7944BDB7A002B40F0A88115
:104B1000924B1888CDF80300102302225BE0601E40
:104B2000C0B2FBF7C1FF00283FF4F4AD436801E7D2
:104B30008B4B8C491B68D9F8002081FB0301DB17E4
:104B4000C3EBA10300241021CDF8033002238DF81C
:104B500000108DF801408DF802306846904734709F
:104B6000002D7FF475ADD7E5794B93ED140AD3EDA5
:104B7000007A20EE270A002420EE080A46F094F975
:104B8000102320228DF80030CDF8030007238DF884
:104B900001208DF802306846D9F80030984734700B
:104BA000002D7FF455ADB7E56F4B1B789B077FF564
:104BB000B1AD6E4AD9F800309268CDF803201022CA
:104BC0008DF8002020210822D6E522F0DFFF1023F7
:104BD0000922CDF803008DF800308DF801308DF8F2
:104BE0000220D9F80030684600249847347005E761
:104BF0005F4B1C6814F0200440F0F4805D4B1B6890
:104C00001B0640F13C81102304228DF803408DF8EF
:104C100004408DF805408DF806408DF800308DF881
:104C200001304CE6D9F81C37CDF8033010220024AF
:104C300001238DF800208DF80140AAE74E4AD9F8EB
:104C40000030B2F90220CDF8032010228DF80020A8
:104C50003021522290E5FF20FBF726FF00283FF489
:104C600059ADB0F90C304549D9F8002091F822101F
:104C700003EB830303EB83031020490800249B000C
:104C800093FBF1F305218DF80000CDF803308DF88A
:104C900001408DF80210684690473470002D7FF473
:104CA000D7AC39E599F8A1370133DAB2042A00F01C
:104CB000DA8042F2107389F8A12703FB02F3D9F8D6
:104CC0000C23002A00F0CA8002332D4A1278D20742
:104CD0002C4A128848BF0433D40748BF0A339007D0
:104CE00048BF1433D10548BF2833540748BF643345
:104CF000500648BF03F57A63102100240422D8E54A
:104D0000194B1B7898077FF505AD184BD9F8002093
:104D1000D9894FF4F36303FB01F3A7FB03135B098A
:104D20001020CDF80330302190E5134AD9F8003037
:104D3000B2F90020CDF8032010228DF80020402188
:104D4000522219E5DE360020F0050020140600206E
:104D500080360020B42B002010360020343600208E
:104D60006C36002067666666F0350020F43500205A
:104D7000E036002078360020D83600200C320020A3
:104D8000843500207C360020FF20FBF78DFE0028B4
:104D90003FF4C0AC90F90130CDF8033010217022FF
:104DA0000B238DF802308DF80010D9F800308DF803
:104DB000012068460024984734701FE689F8A04710
:104DC000012041E65C490620FCF7D0FE002389F86B
:104DD0009E07337003B0BDEC028BBDE8F083574BE8
:104DE0009868A8E4564A5749538A0978643BC3EB4C
:104DF0004370C3EBC00388FB03401844DB17C3EBCD
:104E000020230933092BA8BF092323EAE37303EB0B
:104E1000830311F0020F03EB830314BF4FF47A7086
:104E200000209B00C90748BF00F5FA60117DD9F842
:104E300000209BB203440B44042010218DF8020093
:104E4000CDF803308DF800108DF80110684600246D
:104E500090473470002D7FF4FBAB5DE4013334E701
:104E600022F094FE56E6012389F8A13742F210732E
:104E700025E7347003B0BDEC028BBDE8F083324B04
:104E80009B7A002B3FF446AC99F8A237032B4ED8FF
:104E9000DFE803F043392A111A6882EAE273A3EBD0
:104EA000E27303EB5303A7FB0313DB08002AB8BF2D
:104EB00043F08043FAE4D9F8A427537A907AD17A60
:104EC00003F1407303EB0023002203EB014389F855
:104ED000A22710220421CDF803308DF800208DF890
:104EE00001208DF8021083E5D9F8F0168A7D087C40
:104EF000897A120402EB00220A44591C89F8A2178D
:104F000002EB0363E5E7D9F8F0164A7DC87B497ADE
:104F1000120402EB00220A44EFE7D9F8F0160A7DEA
:104F2000887B097A120402EB00220A44E5E75A1C46
:104F300089F8A2271B06CCE7191201086C3600205D
:104F4000F4350020F03500201036002030B5A0F1F7
:104F50007D03012B044683B00D46104608D9214637
:104F60002FF09EFB15B1288804442C8003B030BD7F
:104F70007D2101922FF094FB019884F020012FF005
:104F80008FFBEFE730B50F4B85B0D3F8A827002390
:104F90000446C51DADF80E3014F8010B01920DF159
:104FA0000E01FFF7D3FFA542019AF5D10DF10E00D6
:104FB00012F06AF9019A9DF80E000021FFF7C6FF72
:104FC00005B030BDB8890020044AD2F8AC3743F4AC
:104FD000DF2343F48063C2F8AC377047B889002000
:104FE000013070B5094EC4B203E041F0B7FC0134A2
:104FF00048B9E5B2152D21463046F6D9162D04BF25
:10500000034B93F8B057284670BD00BF6491002051
:10501000B889002000B1D7E7044AD2F8AC3723F4AE
:10502000DF2323F48063C2F8AC377047B8890020CF
:1050300070B5104E84B00446D6F8B4070D4628F07B
:10504000BDF80D4B1A795B79003A18BF01220BB1FC
:1050500042F00802CDE9015200234FF4964194F941
:10506000000000911A46082128F045F9C6F8B40757
:1050700004B070BDB88900201036002010B5064C71
:1050800003E0D4F8B4072FF0FFFAD4F8B4072FF0F8
:1050900003FB0028F5D110BDB889002010B50D4CD8
:1050A000D4F8B8371B791E3B012B0DD9D4F8B407BF
:1050B00001213830FFF7BCFF0023C4F8BC3784F867
:1050C000C037BDE81040D9E7D4F8B40701212FF06C
:1050D000D3FAF1E7B889002070B5094E0546736828
:1050E0005E200C469847736828469847E0B2FCF764
:1050F000ABF8C4F30720BDE87040FCF7A5B800BFCB
:10510000B889002003682DE9F041002B3C4D3D4F4C
:105110003D4EB8BF5B42A5FB0321890D07FB01375C
:10512000C7EB0717BF00B37985FB0725FA170446BD
:10513000C2EBA555002B56D101EB810101EB81019A
:1051400005EB810109B2DFF8BC801320FFF7C4FF33
:105150002E4908FB057581FB0531ED17C5EBA11143
:1051600009B21B20FFF7B8FF2368254D002BB4BF01
:1051700053214E212320FFF7AFFF6368B27983EA02
:10518000E376A6EBE376A5FB0631890D08FB016803
:10519000C8EB08184FEA880885FB08354FEAE87322
:1051A000C3EBA5552ABB01EB810101EB810105EBA6
:1051B000810109B21220FFF78FFF124B134903FB45
:1051C000058581FB0531ED17C5EBA11109B21A2048
:1051D000FFF782FF6368002BBDE8F041B4BF5721A1
:1051E0004521222078E7C1EB011105EB810109B2CD
:1051F000A9E7C1EB011105EB810109B2DAE700BFB4
:105200006BCA5F6B806967FF10360020D34D621058
:105210000B2814D810B401EB4103094C01EB8303B4
:105220002344184490F83033934205D0214400239E
:1052300080F8302381F824335DF8044B70477047C1
:10524000B8890020F0B5464C94F8C137012B83B0E3
:10525000054650D994F8C2074249434E94F8C377A3
:10526000421CA1FB02C1184406EB800001F4FE764B
:1052700006EB9101521AD0F8206184F8C2272FB1B1
:10528000D4F8C41704F5F96291420DD06EB9374ACB
:105290000133A2FB031222F0010101EB52029B1A1F
:1052A00084F8C13703B0F0BD314E94F8DC3793B9C0
:1052B000304B019348F2A501123B15226F46A4F82A
:1052C000E017009384F8E22729463846B04758B9DA
:1052D00094F8C137DBE76F46384610F0DBFE29460D
:1052E0003846B0470028F3D094F8DC1759B1384657
:1052F00010F04AFEECE71C4A02EB8302D2F8206170
:10530000002EC4D0D1E7009E1B4A964214D9013A20
:10531000013E41F2210512F8013F81EA03210823F1
:1053200011F4004F85EA41000ABF490081B289B2F9
:10533000013BF5D19642EED1384637F055FA0F4988
:10534000009D6D1A152DA8BF15252A4601F11800DC
:1053500047F04EF894F8C13784F80D5897E700BF2E
:10536000B8890020CDCCCCCCECC60508ABAAAAAA43
:10537000D91A0108AD9100209B910020989100203E
:1053800070B50C4E054606F61201D52238F032FAF9
:105390002C686C6006F50161641A182CA8BF1824EB
:1053A0002960224606F6280047F022F886F8404891
:1053B00070BD00BFB8890020F0B58BB004461F4B0C
:1053C0001F4A2049009302A81F4B3CF02DF9266884
:1053D0000025731C2360357023682922591C216025
:1053E0001A702368EA22591C21601A702368C822A7
:1053F000591C216002A81A7044F0D6FD471C02A96E
:105400003A46206846F0F4FF236829461F440C23DF
:1054100000E027687A1C013B22603970F9D12268CC
:10542000511C2160137023680122991821601A70A1
:1054300023689B1B33700BB0F0BD00BF6B90002046
:105440008C390608943E06088C3E060870B505683F
:105450002B4E00236A1C02602B7003682122591C0A
:1054600001601A703378DB0704461DD5254B1B8875
:1054700059050FD52449204637F05CF93378DB070E
:105480001DD523680022591C21601A7023685B1BFC
:105490002B7070BD1A0524D4D80524D4D90724D480
:1054A0009A0724D51949E6E7194BD3F80C3363B1B1
:1054B0001849204637F03EF93378DB07E1D42368FA
:1054C0002A22591C21601A70DBE7134B1B6818064F
:1054D000CCD5124B1B7803F00303032BC6D0104925
:1054E000C9E71049C7E71049C5E71049C3E7084BAA
:1054F0000F4993F834270F4B002A18BF1946BAE713
:10550000843500207C360020C13B0608A03E0608FA
:10551000B8890020A43E060878360020F035002027
:10552000AC3E0608B43E0608B83E0608C03E060873
:10553000E43B0608C83E060838B50368394D591CD7
:10554000082201601A7003681E22591C01601A703B
:10555000B5F90230B3F5E16F044650DDA3F56163A0
:105560001BB2B3F5E16FF9DC07EE903A9FED2E7AAE
:10557000F8EEE77A204667EE877AFDEEE77A17EED7
:10558000903A99B237F00AF9B5F90030B3F5E16F06
:105590003CDDA3F561631BB2B3F5E16FF9DC07EE07
:1055A000903A9FED217AF8EEE77A204667EE877A07
:1055B000FDEEE77A17EE903A99B237F0EFF8B5F9C9
:1055C0000430B3F5E16F28DDA3F561631BB2B3F5D9
:1055D000E16FF9DC07EE903A9FED137AF8EEE77A87
:1055E000204667EE877AFDEEE77A17EE903A99B299
:1055F000BDE8384037F0D2B803F561631BB213F54C
:10560000E16FF9DBB0E703F561631BB213F5E16FFE
:10561000F9DBC4E703F561631BB213F5E16FF9DB56
:10562000D8E700BFD836002058A08B41026810B4DC
:105630000421541C0460117002680B24511C016089
:1056400014705DF8044BC82137F0A8B838B503686A
:10565000214A5D1C0A2105601970036808215D1C40
:1056600005601970D37A044663B322F08FFA1B49A0
:105670000530A1FB0031C1F3CF01204637F08EF891
:10568000174D18492B6881FB0321DB17C3EBA101E0
:1056900089B2204637F082F822F084FAAD68236898
:1056A0002A0C591C21601A7023682A0A591C21608F
:1056B0001A7023685A1C22601D7023685A1C2260CD
:1056C000187038BD084A054B11880531A3FB01311C
:1056D000C90837F063F8D3E710360020CDCCCCCC26
:1056E0006C36002067666666343600200368112237
:1056F000591C70B501601A7003681D4D1D4E5A1C6F
:10570000026002221A700446296837F02FF869688F
:10571000204637F02BF8E98901EBC10189003231CD
:10572000A6FB0131C1F34F11204637F037F8298A23
:1057300001EB8101490089B2204637F02FF80E4A6B
:105740000E4BD2F81C179942A8BF194621EAE17105
:10575000A6FB0131490901F57A7189B2204637F07B
:105760001DF823682A7D591C21601A7070BD00BF86
:10577000F43500201F85EB51B889002020A10700D7
:10578000F8B50B4D0B4F06462946D52238F032F8B6
:1057900034687460A91E641A402CA8BF402431608C
:1057A000224607F6440046F023FE87F88448F8BDF9
:1057B000163D0020B889002070B5104E104B0A46E7
:1057C000151D014696F8850803F83F5C82B003F882
:1057D0003D0C7B25C82003F83C0CA3F13B0403F8E7
:1057E000400C03F83E5C68460193009436F0B4FF29
:1057F0006846FFF7C5FF02B070BD00BFB889002042
:10580000543D0020F0B5434C94F88838D90785B052
:10581000054637D594F889380F2B57D900210F4604
:105820003D4B94F888283D4843F8400CA3F14006CE
:1058300040F6C82CC2F38202712003F8381CA6F887
:1058400004C0B11C0393B071373B02A8F271BA22B5
:10585000029337F0CFFF029A731CD21A727010F0C5
:105860003BFC02A8FFF78CFF10F036FC94F8883858
:10587000C4F88C5823F0030343EA470384F88838BC
:1058800005B0F0BD9A0729D5D4F88C082D1AB5F5C6
:105890007A6FF5DB94F88938D4F890080F2B97BF0E
:1058A0001F4A204902EB8303D3F83C11036801919E
:1058B0001B69984701990620F9F7E4FB94F88838AA
:1058C0006FF3410384F8883805B0F0BD164B93F8A8
:1058D00034301F1E18BF01273946A1E7134B1B6840
:1058E0005B05CDD4104B93F83430002BC8D00A4B55
:1058F0000393C821A3F13F0202A803F8401C0292BF
:10590000FFF794FE10F0E8FB02A8FFF739FF10F054
:10591000E3FBB5E7B8890020543D0020C80032EC15
:10592000ECC60508A0680600F05A00207836002072
:105930002DE9F843254E96F89448804634BBD6F8B6
:10594000F8386BB306F698074FF001090DE0013502
:105950002C44EFF31183502282F31288D6F8F828F2
:10596000944220DADBB283F311883319601C93F878
:105970009858384429460022FCF7A6F90028E6D0BA
:1059800096F88438D3B186F89498E0E796F884388E
:1059900033B901463A20FCF7E9F8044686F8940842
:1059A0002046BDE8F8830022DBB2C6F8F82896F856
:1059B000944883F311882046BDE8F88341463A2095
:1059C000FCF7D4F886F89408C1E700BFB889002036
:1059D000034B1B6A30EA030314BF01200020704709
:1059E00010360020AE4A38B50820002382F829304E
:1059F000FFF7EEFF48B1536A4FF4806402204FF482
:105A000082611C8082F8290059804FF40020FFF742
:105A1000DFFF48B192F82930516A5C1C40F2014026
:105A200082F8294021F813009E494B7A002B68D157
:105A30008B7A002B40F03C814FF40070FFF7C8FFD9
:105A400048B192F82930516A5C1C4FF4046082F826
:105A5000294021F81300944B1968880700F1D5807C
:105A6000490700F1B180914B1B681B0668D492F87E
:105A7000293082F828304FF48030002382F8293012
:105A800082F82130FFF7A4FF30B1D36901204FF431
:105A9000047182F8210019804FF40040FFF798FF4D
:105AA00048B192F82130D1695C1C4FF4007082F843
:105AB000214021F813004FF40030FFF789FF48B16F
:105AC00092F82130D1695C1C4FF4A06082F821402B
:105AD00021F813004FF48020FFF77AFF48B192F8C5
:105AE0002130D1695C1C4FF4376082F8214021F8E5
:105AF000130092F8213082F82030002382F8213000
:105B000038BD0120FFF764FF002891D04FF48030AA
:105B1000FFF75EFF48B992F82930506A5D1C4FF4D8
:105B2000047482F8295020F8134092F82930506A02
:105B30005D1C4FF4116482F8295020F8134077E778
:105B40004FF40050FFF744FF48B192F82930516AF2
:105B50005C1C4FF4036082F8294021F813004FF4D5
:105B60008050FFF735FF70B192F82930506A591C08
:105B70001D46C9B24FF40064023320F8154082F884
:105B8000293020F811404FF48040FFF721FF48B141
:105B900092F82930516A5C1C4FF4846082F82940E5
:105BA00021F813004FF48060FFF712FF00283FF444
:105BB0005EAF92F82930516A5C1C4FF4026082F8A3
:105BC000294021F8130052E74FF48060FFF700FFEF
:105BD00048B192F82930516A5C1C4FF4807082F809
:105BE000294021F813004FF40060FFF7F1FE002870
:105BF0003FF439AF92F82930516A5C1C4FF4887039
:105C000082F8294021F813002DE78020FFF7E0FEFD
:105C100048B192F82930506A5D1C45F2302482F870
:105C2000295020F813404FF48070FFF7D1FE48B19F
:105C300092F82930506A5D1C45F2402482F82950C0
:105C400020F813401020FFF7C3FE48B192F8293026
:105C5000506A5D1C4FF4E06482F8295020F813402C
:105C60002020FFF7B5FE48B192F82930506A5D1C3C
:105C70004FF4E26482F8295020F813404020FFF7E7
:105C8000A7FE00283FF4ECAE92F82930506A5D1C64
:105C90004FF4E46482F8295020F81340E0E600BF96
:105CA000F005002050360020E03600207836002035
:105CB0000220FFF78DFE00283FF4BEAE4FF40040F7
:105CC000FFF786FE48B992F82930516A5C1C4FF400
:105CD000007082F8294021F813000420FFF778FEB5
:105CE00048B192F82930516A5C1C4FF4C06082F8C8
:105CF000294021F813004FF48010FFF769FE0028B7
:105D00003FF49AAE92F82930516A5C1C45F250205B
:105D100082F8294021F813008EE600BF03685A0676
:105D200007D513F4057F04D007298CBF002001207C
:105D3000704703F48253B3F5825F03BFC81FB0FA04
:105D400080F040090020704770B5BC4C94F8FC38D6
:105D5000012B84B000F04D8194F80909FDF794FB04
:105D600094F80A39834205461FD0002800F0D780F6
:105D7000D4F8B837CBB1B24A93F904005279002A6B
:105D800018BF08224FF4964100230325CDE90152A4
:105D900000911A46082127F0AEFAC4F8B40720B1E2
:105DA000FFF77CF9012384F80A3994F80B39012BA9
:105DB00000F0C280D4F814693EB1A24B3046597845
:105DC000FFF7ACFF002840F0F28094F81909FDF7C6
:105DD0005BFB94F818398342054622D0002800F076
:105DE000F680F6B1337A002B00F01881964A02EB68
:105DF0008303D3F83C31924A96F904001279009358
:105E0000003A18BF012202210023CDE901121A46EF
:105E1000102127F070FAC4F8980710B1012384F814
:105E20001839D4F81C693EB1864B30465978FFF7D3
:105E300075FF002840F0AB8094F82809FDF724FB9B
:105E400094F820398342054623D0002800F0C8800A
:105E5000FEB1337A002B00F0E4807B4A02EB83032F
:105E6000D3F83C31764A96F9040012790093003A4F
:105E700018BF012202210023CDE901121A464FF476
:105E8000007127F038FAC4F8240910B1012384F80E
:105E9000203994F82909FDF7F7FA94F82A39834252
:105EA000054630D088B3D4F82C3DD4F8EC6F4FF4CD
:105EB0007A721A613EB34FF480524021304627F087
:105EC000A9F90546F8B95E4B96F904001B79002B39
:105ED00014BF0921082103224FF4E133CDE9012148
:105EE00000932A462B464FF4805127F004FAC4F859
:105EF000F00F40B15549564A84F8F45F0123086019
:105F0000157084F82A3904B070BDD4F8F00F27F06A
:105F100055F9C4F8F05F84F82A5904B070BDD4F87C
:105F2000B40727F04BF994F80B39C4F8B457012B98
:105F300084F80A597FF43EAF94F80C09FDF7A4FAEF
:105F40000546002870D0D4F8A837002B7FF432AF74
:105F5000D4F81029002A3FF42DAF394992F90400F2
:105F60004A790979002A14BF08220022002908BFB3
:105F700042F0010203254FF46141CDE90152009145
:105F80001A46202127F0B7F9C4F8A80712E794F8B9
:105F90002039002B7FF47DAFD4F80439002B3FF477
:105FA00078AF0122C4F8243984F8202971E794F8E5
:105FB0001839002B7FF435AFD4F80439002B3FF4A7
:105FC00030AF0122C4F8983784F8182929E7D4F8AB
:105FD000980727F0F3F8C4F8985784F8185920E781
:105FE000D4F8240927F0EAF8C4F8245984F8205991
:105FF0004FE7D4F80059134B28465978FFF78EFE27
:1060000040B3D4F8D035002B7FF4A6AED4F80439D1
:10601000002B3FF4A1AEC4F8D0359DE64FF4964373
:10602000E9E64FF461431DE7D4F8A80700283FF4E0
:10603000C1AE27F0C3F8C4F8A857BBE6B889002062
:1060400010360020CC5A0020ECC6050890700020C5
:106050006870002094F80809FDF716FA0646D8B1D2
:10606000D4F8D035002B7FF477AE002D3FF474AE1A
:106070000E4A95F904001279B2FA82F252094FF4ED
:1060800016510225CDE9015200911A46042127F04C
:1060900032F9C4F8D0055FE6D4F8D00500283FF403
:1060A0005BAE27F08BF8C4F8D06555E610360020BB
:1060B0002DE9F041C84C94F8FC38002B00F0C18168
:1060C000082027F0BBF8C4F8B807002800F0828148
:1060D000082127F0A9F800270346C049C04884F8E2
:1060E00009390522C4F8FC7F33F09EFABD48BE4D45
:1060F00041F2040341F2085220F808290122E25437
:1061000009F06CFE39462B22A5F1EC0046F0D1F9DE
:1061100048F67C627D26E023394625F8EC2CA5F173
:10612000C0002B2205F8E93C05F8C16C46F0C1F926
:1061300048F67C21A0224EF27B0305F8956C05F809
:10614000927CEE7525F8C01C05F8BD2C25F8943C12
:1061500094F80B39002B00F05F81102027F06EF8C7
:106160001021C4F8140927F05FF8A04EA04B84F862
:10617000190940F23B113A201980727A18719F2157
:106180004AF21E409971002198601973002A40F06C
:106190001281B37A002B71D1DFF87882D8F8003001
:1061A0005A0700F101819F0700F1F580180700F1FF
:1061B000EB80904F3868C0F3C010FEF72BFF002033
:1061C000FEF70EFF03464FF4007084F8B03727F057
:1061D00035F84FF40071C4F81C0927F025F8AB69B5
:1061E00084F82809002B14BF012300232B7740F0EB
:1061F0008F80D4F89038002B14BF0123002385F83A
:10620000253042D1D5F868210023C4F8F838002A97
:1062100000F0B080012284F8DC3785F86C2100237F
:1062200075487649C4F8CC37062233F0FDF940F6BC
:1062300009437148A4F8D03709F0D0FD4FF48050DD
:1062400026F0FCFF4FF48051C4F8EC0F26F0ECFF71
:10625000D5F874316A4A6B4E84F82909C4F8A8232A
:1062600002F5A070591C0022C4F8AC03B360C5F855
:10627000741184F82A29BDE8F04165E5D4F8AC37FB
:1062800043F00403C4F8AC3786E7D8F800000023D5
:1062900010F0020085F8263085F8273040F0E980BC
:1062A0000246737A2BB10120FFF792FB002840F0E1
:1062B000F280B37A002B40F0E8800820FFF788FBDB
:1062C00020B1AB18042183F8281001323B681B066B
:1062D00000F102814C4B10219818053300F8011B86
:1062E0008342FBD105220921202042F2090385F8CF
:1062F0002D2085F8511185F8520144494448A5F8EC
:106300005C31042233F090F9414809F067FD79E7E8
:10631000737A2BB10120FFF75BFB002840F0C180AE
:10632000B27A002A40F0E5803B68190600F1BD8092
:10633000D8F800104B070CD54FF48060FFF748FBEE
:1063400038B1AB18082183F82010013285F82420D9
:106350004FE7080705D54FF40070FFF739FB002819
:10636000EFD10905F2D54FF40060FFF731FB0028AB
:10637000ECD0E6E7D5F87031002B75D0012385F815
:106380006C3184F8DC374AE7D4F8AC3743F48073D7
:10639000C4F8AC370DE7D4F8AC2742F4601242F0F1
:1063A000C002C4F8AC2701E7D4F8AC2742F402726B
:1063B000C4F8AC27F7E6D4F8AC37B27A43F0020160
:1063C000C4F8AC17002A3FF4E7AE43F03603C4F834
:1063D000AC37E1E6044DBBE6B889002068C8050883
:1063E000B0990020B8990020B09A002050360020C3
:1063F0006C620020783600208091002010C90508CA
:10640000708D0020F0050020D89A0020BCC8050837
:10641000049C0020E0360020202026F00FFFC4F866
:10642000100900283FF499AE202126F0FDFE344BE0
:10643000236084F80C09FFF7D5FA012384F80B399F
:106440008BE6042026F0FAFEC4F8000900283FF489
:1064500037AE042126F0E8FE2A4A84F80809012311
:10646000626084F8FC382BE685F86C3184F8DC3700
:10647000E4E64FF46070FFF7ABFA00283FF410AF8A
:10648000012085F8280002460BE70620FFF7A0FA56
:1064900000283FF412AFAB18022183F82810013214
:1064A0000BE7012285F820203EE74FF4A050FFF7CC
:1064B0008FFA20B1AB18022183F8201001324FF47B
:1064C0000850FFF785FA00283FF432AFAB180421DB
:1064D00083F8201001322BE74FF45850FFF778FA79
:1064E00000283FF4F7AEAB18082183F828100132DA
:1064F000F0E60620FFF76CFA0028D2D1024613E737
:10650000854F0108711E01082DE9F04F1546AB4A71
:10651000AB4F92F809A389B004460E462DF008FC53
:10652000A64A8346002020702870D2F8D49030709C
:1065300019F0010F904649D019F046F9002842D0D1
:10654000D8F80C23002A3ED0910104D5B2F1007F87
:1065500018BF02F17E42D7F878119FED9A7AABEB23
:10656000010307EE903AF8EE677AF4EEC77AF1EE9F
:1065700010FA05DCD7F87C0101238340134212D1C5
:1065800011B91923C7F87C31D7F87C31C7F878B135
:10659000012001331A2B28BF002300FA03F1114216
:1065A000F7D0C7F87C31D7F87C21874B874903EBBC
:1065B00082032046D3F878223BF036F802232B7072
:1065C00009B0BDE8F08F0023C7F87831D7F88031E3
:1065D0008BB37F4B1B78DB072DD4D7F884319FED2D
:1065E0007D7A03F5921303F57863A3EB0B0307EEB3
:1065F000903AF8EE677A67EE877AFDEEE77AB8EEC2
:10660000E77A17EE903AF1EE0C7AB4EEE77AF1EE13
:1066100010FA06DB704920463BF006F801232B7088
:10662000CEE70A212046B3FBF1F201FB12336B499E
:106630003AF0FAFFF2E719F4007F0BD0684BDB78F1
:1066400043B1684920463AF0EFFF03232B70012342
:106650003370B5E719F0200F16D01B2019F0B4F8ED
:1066600090B198F8103323B15F4920463AF0DCFF2F
:10667000D4E7574B1B78D80706D45C4920463AF03C
:10668000D3FF01232B709BE719F4806F34D097F868
:106690008831012B30D1564B1B68990727D5554BB4
:1066A000B3F90220B7F99831D21A6FF463739A42A2
:1066B00018DB40F28D339A4217DC0A2392FBF3F287
:1066C0004D4920463AF0B0FF20F044FBD8F8F036B0
:1066D00093F863300A3B23EAE37398429EDB01237D
:1066E00033709BE76FF05902EAE75A22E8E7434923
:1066F00020463AF099FFE7E719F4005F0ED00FF05B
:106700006DFE98F8CC30834208D93D4920463AF0D6
:106710008BFF02232B700123337051E719F4004FD4
:1067200008D0384BB8F92021B3F90C309A4201DD7A
:106730003549EBE719F4804F07D00FF037FEB8F872
:106740001E31834201D93149E0E719F0080F04D026
:10675000BAF1020F01D12E4974E719F4006F0FD07E
:106760001B4B1B78DA070BD51BF03AF940B1294BCC
:106770001B78DB0704D597F8D5310BB92649C5E757
:1067800019F4805F14D0124B1B78D80710D51BF07A
:1067900027F968B11F4B1B78D90709D4D8F85C36A4
:1067A000A3F53713A3F5D863002B01DA1B49ADE736
:1067B0001B4B1B885A0637D51A49A7E7B889002012
:1067C000B09A00200024F448ECC605081C6B0608AB
:1067D00084350020ACC527376A3D0608753D06089C
:1067E00088350020823D06089C4006088C3D06083E
:1067F000E0360020D83600209E3D0608A83D060859
:10680000AF3D0608F0050020293D0608B83D060802
:10681000C53D0608F0350020CF3D0608DA3D0608E4
:106820007C360020E53D060819F0800F19D0B8F934
:10683000A80698F8E630984213DBFBF72FFB98F890
:10684000CD207449002A0CBF0D220E22034600926F
:1068500020467A223AF0E8FE02232B70012333709F
:10686000AEE66D4B1B681B017CD519F0400F79D04B
:106870006A4B93F8009004AAC9F109094FEA590933
:10688000002310462021994521D1654948444FF005
:10689000000B45F032FE09F1030959465F4B1B78A6
:1068A0008B4202D9B9F10B0F15D908AB99440023DB
:1068B00009F8103CBBF1000F54D05A4904AA2046F5
:1068C0003AF0B2FE02232B700123337078E602F80F
:1068D000011B0133D7E7CBB2184603910293FAF7B5
:1068E000E3F8029B039903F1310C4F4B1B7813F033
:1068F00001035FFA8CFC029332D0B8F9E2E0BEF1FA
:10690000FF3F2DD08289642312FB03F2474B93F89B
:1069100022305B0892FBF3F39E45B4BF63465223DB
:1069200098F9E02012F1800F04D090F901E096452B
:10693000A8BF5423029A42B1B8F9E420B2F1FF3F54
:1069400003D040689042A8BF432304AA9C4509F89D
:10695000023018BF0BF1010B013109F101099DE76C
:106960006346DDE7D8F8D49019F0040F0BD0BAF1E4
:10697000010F08D12E4920463AF056FE02232B7013
:1069800086F800A01CE619F4807F08D0264B1B78FF
:10699000DA0704D5274B1B780BB92749B6E619F45B
:1069A000803F0CD0204B1B78DB0708D5B8F8C830E7
:1069B0002BB1224A9268934201DC2149A6E619F0E4
:1069C000020F14D0184B98F809231B7803F0030327
:1069D00013430CD121F0DAF81A4B5B8A834206D9B3
:1069E000194920463AF020FE01232B70E8E519F002
:1069F000100F3FF4E5AD97F8D831002B3FF4E0AD30
:106A0000124920463AF010FE01232B70002387F82C
:106A1000D831D5E5EE3D060878360020B42B0020AD
:106A2000C73B06081C6B0608843500200C3200208A
:106A3000FD3D0608CC620020093E06086C360020A9
:106A4000153E0608503600201E3E06082A3E06085F
:106A500007B5002300F10D020DF1070140688DF824
:106A60000730FFF751FD9DF80730084A43B1D2F8CF
:106A7000D03643F40013C2F8D03603B05DF804FBFF
:106A8000D2F8D03623F40013F5E700BFB889002010
:106A900010B5084B0022D3F884108833914201D1FD
:106AA000002010BD13F8014B844201D00132F5E7FC
:106AB0000120F6E7B8890020F0B404780A4E049F5C
:106AC000650906EB850604F01F04012505FA04F4A8
:106AD000D6F8D05604972C428068F0BC18BF43F01B
:106AE000800332F0D3BD00BFB88900201D4B2DE9D3
:106AF000F04303EB81038FB0D3F8E08206460D46E6
:106B0000B8F1000F2AD0184B03EB41031C221C895B
:106B10000023194604F01F07C4F344190DEB0200CB
:106B2000A413069345F0C5FC01228DF80B4006AC7A
:106B30008DF81420CDE903468DF808508DF80970C2
:106B40008DF80A9002A8C0479DF8142000232AB1AE
:106B500000944A46394602A8FFF7AEFF0FB0BDE8E1
:106B6000F08300BFECC60508B88900202DE9F04F7E
:106B70001D4D90F801808678DFF870B06FF4917346
:106B800085B004462F1D05EB03094FF4FA6A15F989
:106B9000013B002B1EDB09EB8303D3EDAE7AFDEE48
:106BA000E77A4FF47A7317EE902AA2F57A720AFB0D
:106BB00002F292FBF3F202ABA2F57A725946184642
:106BC0003AF032FD02AB00933246002341462046A4
:106BD000FFF772FF0136BD42F6B2D8D1002323730E
:106BE00005B0BDE8F08F00BFDB8A0020493B0608F6
:106BF0002DE9FF47314B477893F82C2193F82D81ED
:106C0000436885781E2AA8BF1E22022AB8BF022226
:106C1000B8F1100FA8BF4FF01008B8F1020F4FF0F5
:106C20000B01B8BF4FF0020804461970D6B25FFAE4
:106C300088F90121501E4FF0170C8842636826DC4A
:106C400013440B2103F8011C616800238B54626814
:106C5000009239462A4620463E44FFF72DFF013E6A
:106C60004FF0010AF6B208F1FF33534513DC05EB90
:106C7000090263680093013A0023D2B239462046E4
:106C8000FFF71AFF0023237304B0BDE8F08703F871
:106C900001C00131D1E705EB0A02D2B21623394611
:106CA00020460392F7F7CEFC039A1623314620467E
:106CB000F7F7C8FC0AF1010AD5E700BFB889002040
:106CC00070B52A4B9FED2A7A2DED028B93ED7F8ACA
:106CD000F0EEC87AF4EEC77AF1EE10FA84B004460A
:106CE0003ED5D3ED7E7AF0EEE76AF4EEC76AF1EEB8
:106CF00010FA35D51F4B02931F4B03931F4BDFED4B
:106D0000208AB3F902309FED1F7A002BD8BFF1EE35
:106D1000677A77EEA87ABAEE0C0AA7EE870AD6BF92
:106D200000250125B1EE488A38EE288A44F0BCF8E7
:106D3000DFED157A6378BAEE000AA8EE270A1E186E
:106D400044F0B2F8A378184404AB03EB8505C2B253
:106D500055F8083C0093F1B200232046FFF7ACFE43
:106D60000023237304B0BDEC028B70BDB09A0020E9
:106D70006C61D83E343E0608CE3B0608D83600206B
:106D8000DB0F493F539A8E4183F922412DE9F04FA1
:106D9000184F91F8018091F80290DFF85CA0DFF8BD
:106DA0005CB085B006460C4600253B78AB4204DC5F
:106DB0000023237305B0BDE8F08F2846B04702AB2F
:106DC000504502465946A8BF524618463AF02CFC98
:106DD00004AB1844002109EB050202AB00F8081CC3
:106DE000D2B2009320460B464146FFF765FE0135BF
:106DF000DBE700BFB42B00209F8601000F8C060844
:106E000001460148C2E700BF451F0108014601488D
:106E1000BCE700BFCD1E01082DE9F0413A4C3B4ACA
:106E200021683B4D012382F8003211F0020F4FF030
:106E30000003C5F88430904608D00320FAF736FAEC
:106E40002A20FAF733FA3C20FAF730FA314F0026BD
:106E500017F8010B0136FAF729FA312EF8D1236819
:106E6000990617D50E20FAF721FA0D20FAF71EFA27
:106E70001820FAF71BFA1720FAF718FA1F20FAF76A
:106E800015FA1E20FAF712FA2F20FAF70FFA3A2015
:106E9000FAF70CFA204C23681A011ED41F4B9B7979
:106EA0000BBB3B20FAF702FA98F801324BB31C4BAC
:106EB0001C4F1C680121204632F0DEFB01212046D8
:106EC00032F00AFC0026D5F884309E4212D32046C8
:106ED0000021BDE8F04132F0CFBB2320FAF7E6F9FC
:106EE00023681B01DAD52420FAF7E0F93320FAF7FA
:106EF000DDF9D6E717F8011B2046FFF7F7FD01364D
:106F0000E1E7BDE8F08100BFE0360020B09A002044
:106F1000B8890020C4CA0508783600200C32002049
:106F2000DC660020408A0020074B032883F8E80035
:106F300003D8064A012308B913706DE7013803FA34
:106F400000F01070F9E700BFB8890020F0050020BC
:106F50002DE9F04F8E4CDFF8648294F83461082EEE
:106F600099B00546274600F09F84012388F8023235
:106F70000D2E00F20786DFE816F00E000506F10080
:106F80002501E102200361039C030506D8042B05BB
:106F9000FE00DE05ED05DFF82892D9F80000036851
:106FA0001B6C4C468BB10021984770B998F803329E
:106FB000042B06D1D9F8000032F064FB19B0BDE80B
:106FC000F08F012388F80032F8E7724B724A1B7881
:106FD000206803F0010388F804320023C7F8D03694
:106FE000536003681B6B002B00F0B18001219847B0
:106FF000002188F80502206832F03EFB2068F7F790
:1070000097F80DF120092068012132F065FBF7F7B0
:10701000FBFA624A624948463AF006FBCDF8009016
:10702000002306221421206832F030FB5D4B0093D0
:10703000082200230721206832F028FB5A4B0093D6
:10704000092200230B21206832F020FB574B0093CC
:10705000206800230A220B210DF1400932F016FBB3
:107060004846FCF753FE38B1CDF800902068002365
:107070000C22052132F00AFB2CF05AFE97F8E8307A
:1070800000F5741000F51060032BC8F8080204D84E
:1070900047490122002B5CD10A7098F8053288F824
:1070A00001320023C7F88430B7F82E3107EE903A4A
:1070B000F8EEE77AF7EE006A86EEA77A3D4B0022FB
:1070C0001A60DFED3D7A77EE277AC7EE276AC3EDC7
:1070D000016AFFF7A1FE206832F0D4FA0C2387F88A
:1070E00034313446354F97F80032FBB92CF020FE8E
:1070F0002F4B93F82D30CBB90A2EA0EB05000AD107
:1071000007EB4404B4F86032B0EB132F40F23E8535
:107110000302A4F8603207EB4606B6F89034B0EBF1
:10712000132F40F23B850502A6F89054184B93F8B4
:1071300034310A2B40F03A8597F88E3407EB43033D
:10714000B3F860321B0A0733C7F8AC3436E7184689
:107150004EE7013B02FA03F30B709EE7184B1868E9
:107160000368DB69984708B10024BBE70B2384F868
:1071700034310446B6E7124B186803681B6A984717
:1071800000287FF41BAF032384F834310446A9E7B9
:10719000B889002084350020889000208C3E0608A5
:1071A000363E06083A3E0608473E0608523E0608A6
:1071B000F00500203491002083F9A23EB09A00200F
:1071C000DC660020C94A98F80412137803F0010322
:1071D0009942914667D0002B00F00A810023C4F841
:1071E0006C36A4F87036C4F85C36C4F86436A4F87B
:1071F0007836C4F87C3688F80C3288F80D3294F86A
:10720000BC36BB4AC4F86026002B0CBF6323642342
:10721000A4F880366322142384F86826A4F8823602
:10722000B44AB54C002191612068012132F054FA32
:1072300097F82A31012BA24607D0022B40F0D680C6
:1072400099F800309C0700F1D180F7F7DDF997F845
:107250002B319FEDAA7A07EE903AF8EEE77A67EEC7
:10726000877AFDEEE77A17EE904AA54B0093DAF89D
:107270000000002307220C2132F008FA97F810339F
:1072800043B1A04B00930822DAF800000023114616
:1072900032F0FCF92C44C8F8084299F8003003F0A9
:1072A000010388F8043299F8004014F0010400F05A
:1072B000E28097F8CB26944B002A00F0C480B3F903
:1072C0000C30B7F960269A42B8BFA7F86036FAF7D3
:1072D000D7FDB7F9623600B283428C4BC8BFA7F81E
:1072E000620664221B6893FBF2F3B7F966261BB2B1
:1072F0009A42B8BFA7F866360FF070F897F868366C
:10730000D7F86C268342D7F81C3788BF87F8680601
:107310009A42B8BFC7F86C367D4BD3ED007A13EDB7
:10732000297AB4EEE77ABC3BF1EE10FA48BFC3ED20
:10733000067A0FF03BF8B7F8802603B29A42754BF5
:10734000B7F98226B3F90C30C8BFA7F880069A4275
:10735000C8BFA7F88236704B1B7803F00303032BDA
:1073600007D16E4BB7F970261B889A42B8BFA7F8B1
:1073700070366B4B1B6813F0006309D0D7F8D82622
:10738000B7F9781692F901209142B8BFA7F878268C
:10739000644A9179104600295FD0634B634C1A7898
:1073A00000210B46914251DBB3FBF2F2C823534359
:1073B00090F82220B3FBF2F3D7F87C269A42B8BFAC
:1073C000C7F87C36D8F81032D7F85826C8F81052CB
:1073D000EB1A1A44C7F85826D7F85C261344C7F8A6
:1073E0005C36052387F8343100247BE6504C3CE7BB
:1073F000D4F8DC30002B3FF450AF98F80E32002B5D
:107400007FF44BAF4B4BDB78002B7FF446AFD4F8C7
:107410000C3313F0600F07D03E4B628E1B7803EAEB
:10742000D22358077FF439AF012388F80C32424B3E
:107430002B44C8F80832FAF723FD0023A7F86406A6
:1074400087F8903729E7B3F90E303AE704EB810C5F
:107450000131BCF80CC06344A4E7002BACD0D7F8D2
:10746000D83692F822209B89642113FB01F352083D
:1074700093FBF2F3A0E798F80C32A3B31E4BD3F8BA
:107480000090B9F1000F0CD099F90F30002B08DDF6
:1074900088F80C42C8F80842C7F85C46C8F8105291
:1074A0009FE70E2018F090F998F80D3248B1D3B14B
:1074B0000021484688F80D1232F00EF9C8F8105233
:1074C0008FE763B9012388F80D3205F5742303F5BE
:1074D0001073C8E98453042387F8343102E6D8F8DE
:1074E00014329D42F1D2C8F810527AE78435002058
:1074F0000000881314900020DC6600200050C34771
:10750000333B06089C400608F43500206C3600200A
:10751000D0900020F0050020F03500200C3600202F
:10752000783600200C320020B42B00208C8F0020F5
:1075300020A10700883500200087930398F81832AF
:10754000022B20D0032B2CD0012B12D097F8903790
:107550000024A34214BF0323012388F81832C44B2C
:1075600087F88E47186887F88F47214632F0B4F8BD
:10757000B8E5FCF705FC00283FF4F6AD022388F8D7
:1075800018320024AEE5BA4B0024186887F88E47FD
:10759000214687F88F4732F09FF8032388F8183286
:1075A000A0E5FCF7EDFB00283FF4DEAD0024052349
:1075B00088F8184287F8343194E5AD4C2068F6F726
:1075C000B7FDD8F808327BB3EB1A002B1EDAA94BB3
:1075D0001B78D90715D4DFEDA87A97EDB17AB4EE10
:1075E000E77AF1EE10FA0ADC97EDAF7AB4EEE77ABB
:1075F000F1EE10FA03DC1B2018F0E6F808B1C8F829
:107600000852062387F8343100246BE520680021F6
:1076100032F062F80023C8F8083288F80C32C7F854
:107620005C36012388F80032944B1B681A01E8D5B8
:10763000FF20F9F739FAC7F8D806E2E7904B1B6844
:107640009B0725D58F4BB4F85C201B7803EAD22327
:10765000D4F8DC2003F0070302F48042134317D070
:10766000894B98ED877AD3ED007A884AE7EE077A5E
:1076700098ED887AE7EE077A98ED897AE7EE077A4F
:10768000B1EEE77AD2ED007A67EE877AC3ED007A41
:10769000774B1B681BB193F90F30002B04DC0723D9
:1076A00087F8343100241DE50C2387F83431002499
:1076B00018E5D4F81C07F9F79BFEDFED757A20EE8C
:1076C000270AFDEEC07A17EE90AA0EF087FE97F813
:1076D000CC30D4F8D04683428CBF44F0010424F06F
:1076E0000104C7F8D0460EF061FEB7F81E21D7F8A6
:1076F000D43682428CBF43F4804323F48043C7F8DE
:10770000D43697F80933002B46D124F4800424F0B2
:107710000204604BC7F8D0461A7812F0020F99465F
:107720000BD05D4B1B7D042B07D998F844229A425D
:1077300045D91AF055F9002841D044F48044C7F8DF
:10774000D046B7F8CE4004F00F00FAF702FC534BD6
:10775000240A5C4325D1D7F8D03623F02003B7F8AC
:10776000D040C7F8D03604F00F00FAF7F2FB4B4BCD
:10777000240A5C431CD1D7F8D03623F04003484A92
:10778000B7F8C8009268D7F8D41690421ADD23F0F3
:10779000102321F0200119E044F4800444F0020495
:1077A000B7E7A042D7F8D036D5D343F02003D6E7C9
:1077B000A042D7F8D036DED343F04003DFE724F40D
:1077C0008044BCE743F0102341F02001B7F8CA2001
:1077D000C7F8D416924539DB264A1278D40735D536
:1077E00043F40043264A1268900632D5214A1278A3
:1077F000D2072ED599F8002002F00302032A28D1DF
:10780000B7F828212AB327480088904221D343F0B3
:107810000043C7F8D036194B1B681B010ED597F9EA
:10782000E03013F1800F19D0D7F8D82692F9012053
:107830009A4213DB41F00801C7F8D416D8F8084281
:107840008CB10D2387F8343100244BE423F400433A
:10785000C8E723F00043C7F8D036DCE721F0080181
:10786000C7F8D416EAE7082387F834313AE400BFB2
:10787000DC6600208435002000C0DA447836002021
:10788000E0360020F0050020D09000208036002057
:107890000AD7233CF0350020F435002000879303FD
:1078A0006C3600200C3600200E2017F08DFFC64BE2
:1078B0000146186839B1002131F00EFF0C2384F81D
:1078C000343100240EE498F8053253B303689B6BFF
:1078D0000BB101229847BD4B98F858221B68C3F39F
:1078E00040139A4203D088F85832FFF795FAD8F837
:1078F0005C32B7F82E210133B3EB920FC8F85C323B
:1079000009D1B34A0023C8F85C3292F82C3083F0D6
:10791000010382F82C30092387F834310024FFF763
:10792000E1BB194631F0D8FED5E7AA4B94F88400A4
:1079300003F17C023E24002133F802CB22F8021B23
:10794000BCF5F05F04F1FF3488BF23F8021C14F08B
:10795000FF04F1D12246A44682420AD3002388F8CC
:107960008E3400283FF4A0AE0A2387F83431FFF7A5
:10797000B9BB08EB4C034FEA4C0EB3F8DC1208EB32
